:100000000C94830B0C94A4990C94D5990C94069A97
:100010000C94379A0C94689A0C94999A0C94CA9AF6
:100020000C94FB9A0C94B40B0C94B40B0C94B40B7E
:100030000C94B40B0C94B40B0C94B40B0C94B40B44
:100040000C94B40B0C94F40E0C94B40B0C94B40BF1
:100050000C94B40B0C94B40B0C94EB760C94D49CD1
:100060000C94B40B0C942F780C94B40B0C94B40B2C
:100070000C94B40B0C94B40B0C94B40B0C94B40B04
:100080000C94B40B0C94B40B0C94B40B0C94B40BF4
:100090000C94B40B0C94B40B0C94B40B0C94B40BE4
:1000A0000C94B40B0C94B40B0C94B40B0C94B40BD4
:1000B0000C94B40B0C94B40B0C94B40B0C94B40BC4
:1000C0000C94B40B0C94B40B0C94B40B0C94B40BB4
:1000D0000C94B40B0C94B40B0C94B40B0C94B40BA4
:1000E0000C94B40B084AD73B3BCE016E84BCBFFDD9
:1000F000C12F3D6C74319ABD56833DDA3D00C77FF8
:1001000011BED9E4BB4C3E916BAAAABE0000008090
:100110003F05A84CCDB2D44EB93836A9020C50B91F
:10012000918688083CA6AAAA2ABE000000803F65E6
:1001300063686F3A00656E6473746F7073206869EA
:10014000743A200020583A0020593A00205A3A00C8
:1001500024F404D9201BC40C5C0E9804C4095F026B
:1001600065077101F405F900FB04B300480487003A
:10017000C10369005803550003034500BE023A005D
:100180008402310053022A002902250004022000C3
:10019000E4011C00C8011900AF0117009801140008
:1001A00084011300710110006101100051010E0063
:1001B00043010D0036010B002B010B0020010B0049
:1001C000150109000C01090003010800FB000800EB
:1001D000F3000800EB000700E4000600DE00060064
:1001E000D8000600D2000600CC000500C7000500BC
:1001F000C2000500BD000400B9000400B500040001
:10020000B1000400AD000400A9000400A500030033
:10021000A20003009F0004009B000300980003005D
:100220009500020093000300900003008D0002007F
:100230008B00030088000200860002008400030097
:10024000810002007F0002007D0002007B000200AE
:1002500079000200770001007600020074000200BD
:1002600072000100710002006F0002006D000100C9
:100270006C0002006A0001006900020067000100D2
:1002800066000100650001006400020062000100D8
:1002900061000100600001005F0002005D000100DC
:1002A0005C0001005B0001005A00010059000100E0
:1002B00058000100570001005600010055000100E0
:1002C00054000100530000005300010052000100DF
:1002D00051000100500001004F0001004E000000DD
:1002E0004E0001004D0001004C0001004B000000D9
:1002F0004B0001004A0001004900010048000000D5
:1003000048000100470001004600000046000100CF
:1003100045000000450001004400010043000000CA
:1003200043000100420000004200010041000000C3
:1003300041000100400001003F0000003F000100BB
:100340003E0000003E0001003D0000003D000100B5
:100350003C0000003C0000003C0001003B000000AD
:100360003B0001003A0000003A00010039000000A3
:10037000390001003800000038000000380001009A
:100380003700000037000100360000003600000092
:100390003600010035000000350000003500010086
:1003A000340000003400000034000100330000007D
:1003B0003300000033000100320000003200000072
:1003C0003200010031000000310000003100010066
:1003D0003000000030000000300001002F0000005D
:1003E0002F0000002F0000002F0001002E00000051
:1003F0002E0000002E0001002D0000002D00000046
:100400002D0000002D0001002C0000002C00000039
:100410002C0000002C0001002B0000002B0000002D
:100420002B0000002B0001002A0000002A00000021
:100430002A0000002A000100290000002900000015
:100440002900000029000000290001002800000008
:1004500028000000280000002800000028000100FB
:1004600027000000270000002700000027000000F0
:1004700027000100260000002600000026000000E2
:1004800026000000260001002500000025000000D5
:1004900025000000250000002500000025000100C7
:1004A00024000000240000002400000024000000BC
:1004B00024000100230000002300000023000000AE
:1004C000230000002300000023000000230001009F
:1004D0002200000022000000220000002200000094
:1004E0002200000022000100210000002100000085
:1004F0002100000021000000210000002100000078
:100500002100010020000000200000002000000069
:10051000200000002000000020000000200000005B
:10052000200001001F0000001F0000001F0000004D
:100530001F0000001F0000001F0000001F0001003E
:100540001E0000001E0000001E0000001E00000033
:1005500024F4D43050C38E20C2A24017828B701175
:10056000127A910D816CD90AA861E108C758660713
:10057000615143061E4B5D05C145A7041A41110494
:10058000093D9803713931034036DB02653391022E
:10059000D4305402802E1D02632CEE01752AC50151
:1005A000B028A001102781018F2564012B244B0165
:1005B000E0223401AC211F018D200D01801FFC00C1
:1005C000841EED00971DDF00B81CD200E61BC6009C
:1005D000201BBC00641AB200B219A8000A19A000BE
:1005E0006A189900D117910040178B00B516840046
:1005F00031167E00B31579003A157300C7146F00E9
:1006000058146A00EE1366008813630025135E0019
:10061000C7125B006C12570015125400C111510033
:1006200070114F0021114B00D61049008D1047006A
:100630004610440002104200C00F4000800F3E00F0
:10064000420F3C00060F3B00CB0E3800930E3700E4
:100650005C0E3500270E3400F30D3200C10D310061
:10066000900D3000600D2E00320D2D00050D2C0078
:10067000D90C2B00AE0C2900850C29005C0C27003E
:10068000350C27000E0C2600E80B2400C40B2400B8
:10069000A00B23007D0B23005A0B2100390B2100F6
:1006A000180B2000F80A1F00D90A1E00BB0A1E0002
:1006B0009D0A1D00800A1D00630A1C00470A1B00DA
:1006C0002C0A1B00110A1A00F7091A00DD0919008B
:1006D000C4091900AB091900920917007B09180019
:1006E000630917004C091600360916002009160088
:1006F0000A091500F5081500E0081400CC081400DC
:10070000B8081400A4081400900813007D08120013
:100710006B08130058081200460812003408110034
:10072000230811001208110001081100F007100041
:10073000E0071000D0071000C0071000B0070F003E
:10074000A107100091070E0083070F0074070F0028
:1007500065070E0057070E0049070E003B070D0006
:100760002E070E0020070D0013070D0006070D00D1
:10077000F9060C00ED060D00E0060C00D4060C0096
:10078000C8060C00BC060C00B0060C00A4060B004A
:1007900099060C008D060B0082060B0077060B00F5
:1007A0006C060B0061060A0057060B004C060A0097
:1007B00042060A0038060A002E060A0024060A002D
:1007C0001A060A001006090007060A00FD050900BE
:1007D000F4050900EB050900E2050900D905090047
:1007E000D0050900C7050900BE050900B5050800C8
:1007F000AD050800A50509009C0508009405080042
:100800008C050800840508007C05080074050800B4
:100810006C050700650508005D0507005605080022
:100820004E0507004705070040050800380507008A
:10083000310507002A050700230507001C050600EF
:10084000160507000F05070008050600020507004A
:10085000FB040600F5040700EE040600E8040600A9
:10086000E2040700DB040600D5040600CF040600FE
:10087000C9040600C3040600BD040600B704060050
:10088000B1040500AC040600A6040600A00405009F
:100890009B04060095040500900406008A040500E8
:1008A00085040500800406007A040500750405002F
:1008B000700405006B040500660405006104050072
:1008C0005C04050057040500520405004D040500B2
:1008D00048040500430405003E0404003A040500F2
:1008E00035040500300404002C040500270404002E
:1008F000230405001E0404001A0404001604050065
:10090000110404000D04040009040500040404009B
:1009100000040400FC030400F8030400F4030400D2
:10092000F0030400EC030400E8030400E403040003
:10093000E0030400DC030400D8030400D403040033
:10094000D0030400CC030400C8030300C503030064
:1009500052656C65617365642E007C3C3E5E2B3D88
:100960003F2F5B5D3B2C2A225C006563686F3A0079
:10097000656E717565696E6720220022007374616F
:10098000727400506F7765725570002045787465F9
:10099000726E616C205265736574002042726F77CD
:1009A0006E206F75742052657365740020576174F2
:1009B0006368646F672052657365740020536F66C7
:1009C0007477617265205265736574004D61726C55
:1009D000696E3A2000312E302E30205243320020F2
:1009E0004C61737420557064617465643A20004DE5
:1009F00061726C696E2D5468752C20313220417003
:100A00007220323031322031343A30313A333020B2
:100A10002B30323030202D203431343430386232B3
:100A20006430666564343238623535343435663462
:100A30003862303164303039333261376139326392
:100A400000207C20417574686F723A2000427569FD
:100A50006C642D4D652D4D61726C696E002046727F
:100A60006565204D656D6F72793A20002020506CCD
:100A7000616E6E6572427566666572427974657301
:100A80003A200053746F7265642073657474696EE4
:100A90006773207265747265697665643A00537491
:100AA0006570732070657220756E69743A0020203D
:100AB0004D3932205800205900205A002045004D61
:100AC0006178696D756D20666565647261746573C2
:100AD00020286D6D2F73293A0020204D32303320AD
:100AE0005800205900205A002045004D6178696D5A
:100AF000756D20416363656C65726174696F6E200A
:100B0000286D6D2F7332293A0020204D323031206C
:100B10005800205900205A00204500416363656C4D
:100B200065726174696F6E3A20533D616363656CF1
:100B300065726174696F6E2C20543D7265747261C8
:100B4000637420616363656C65726174696F6E00C4
:100B500020204D323034205300205400416476610F
:100B60006E636564207661726961626C65733A20B8
:100B7000533D4D696E206665656472617465202819
:100B80006D6D2F73292C20543D4D696E2074726158
:100B900076656C20666565647261746520286D6D8C
:100BA0002F73292C20423D6D696E696D756D207320
:100BB00065676D656E742074696D6520286D732995
:100BC0002C20583D6D6178696D756D207859206ACB
:100BD00065726B20286D6D2F73292C20205A3D6D76
:100BE0006178696D756D205A206A65726B20286D79
:100BF0006D2F73290020204D3230352053002054B2
:100C000000204200205800205A002045005049444E
:100C10002073657474696E67733A002020204D3329
:100C200030312050002049002044006F6B00446F99
:100C30006E6520736176696E672066696C652E004B
:100C40004572726F723A004C696E65204E756D6226
:100C50006572206973206E6F74204C617374204C30
:100C6000696E65204E756D6265722B312C204C616A
:100C70007374204C696E653A00636865636B7375C5
:100C80006D206D69736D617463682C204C617374A1
:100C9000204C696E653A004E6F20436865636B7344
:100CA000756D2077697468206C696E65206E756D4E
:100CB0006265722C204C617374204C696E653A0039
:100CC0004E6F204C696E65204E756D62657220779F
:100CD00069746820636865636B73756D2C204C6163
:100CE0007374204C696E653A006F6B005072696EC8
:100CF0007465722073746F7070656420646575200C
:100D0000746F206572726F72732E2046697820743A
:100D10006865206572726F7220616E6420757365FC
:100D2000204D39393920746F207265737461727483
:100D3000212E202854656D7065726174757265206E
:100D400069732072657365742E205365742069740D
:100D5000206265666F726520726573746172746972
:100D60006E67290053544F505045442E2000446F65
:100D70006E65207072696E74696E672066696C6555
:100D8000004457454C4C2E2E2E004E6F206D6F7632
:100D9000652E00426567696E2066696C65206C6926
:100DA000737400456E642066696C65206C697374A9
:100DB000006F6B20543A0020423A0020403A00482D
:100DC000656174696E672E2E2E00543A0020453AF4
:100DD0000020573A0048656174696E6720646F6E41
:100DE000652E004265642048656174696E672E0057
:100DF000543A0020453A0020423A0042656420649B
:100E00006F6E652E005061727469616C2052656C62
:100E100065617365004649524D574152455F4E41E9
:100E20004D453A4D61726C696E2056313B205370CE
:100E300072696E7465722F6772626C206D6173687F
:100E4000757020666F722067656E36204649524D78
:100E5000574152455F55524C3A687474703A2F2F7F
:100E60007777772E6D656E64656C2D706172747323
:100E70002E636F6D2050524F544F434F4C5F564579
:100E80005253494F4E3A312E30204D414348494E3E
:100E9000455F545950453A4D656E64656C20455820
:100EA0005452554445525F434F554E543A310A000F
:100EB000583A00593A005A3A00453A0020436F75B3
:100EC0006E7420583A00593A005A3A00785F6D69BA
:100ED0006E3A00785F6D61783A00795F6D696E3ABD
:100EE00000795F6D61783A007A5F6D696E3A007AD9
:100EF0005F6D61783A00556E6B6E6F776E20636F31
:100F00006D6D616E643A2200220053657474696EDF
:100F100067732053746F72656400526573656E6405
:100F20003A006F6B005072696E7465722068616C74
:100F30007465642E206B696C6C28292063616C6C6D
:100F40006564202121004B494C4C45442E20005023
:100F500072696E7465722073746F7070656420645A
:100F6000657520746F206572726F72732E204669EA
:100F70007820746865206572726F7220616E6420DB
:100F8000757365204D39393920746F20726573741B
:100F9000617274212E202854656D706572617475BC
:100FA00072652069732072657365742E20536574B1
:100FB000206974206265666F726520726573746162
:100FC0007274696E67290053544F505045442E2067
:100FD000005072696E7465722052656164792E00EA
:100FE000022D2D2D2F2D2D2D0120006820006D00AC
:100FF0005A3A0025200025534400204D61696E2097
:101000000300204175746F73746172740020446929
:101010007361626C65205374657070657273002033
:101020004175746F20486F6D650020536574204FC3
:10103000726967696E00205072656865617420503E
:101040004C41002050726568656174204142530034
:1010500020436F6F6C646F776E00204D6F76652054
:10106000417869732020202020207E002050726566
:101070007061726520030020583A0020593A002020
:101080005A3A00204578747275646500204D616994
:101090006E2003002053706565643A0020024E6F95
:1010A0007A7A6C653A0020024265643A0020466113
:1010B0006E2073706565643A0020466C6F773A0065
:1010C00020436F6E74726F6C20030020024E6F7AA3
:1010D0007A6C653A0020024265643A002046616EEF
:1010E0002073706565643A00205049442D503A20C1
:1010F00000205049442D493A2000205049442D44B5
:101100003A2000205049442D433A200020436F6E7E
:1011100074726F6C200300204163633A003030002A
:10112000303000205678792D6A65726B3A200020A5
:10113000566D61782000783A00793A007A3A006575
:101140003A0020566D696E3A00205654726176203E
:101150006D696E3A0020416D61782000783A00791F
:101160003A007A3A00653A003030003030002041D1
:101170002D726574726163743A0030300030300053
:10118000205873746570732F6D6D3A002059737415
:101190006570732F6D6D3A00205A73746570732FEC
:1011A0006D6D3A00204573746570732F6D6D3A0054
:1011B000204D61696E202020202020202003002067
:1011C00054656D7065726174757265207E00204D86
:1011D0006F74696F6E2020202020207E00205374C1
:1011E0006F7265204550524F4D00204C6F61642056
:1011F0004550524F4D0020526573746F7265204602
:1012000061696C7361666500204D61696E20030041
:10121000045265667265736800200020576174632C
:101220006820202003002050726570617265207E66
:10123000002054756E65202020207E0020436F6EB4
:1012400074726F6C207E002053746F70205072692E
:101250006E742020207E002043617264204D656EF4
:1012600075202020207E00204E6F20436172640094
:101270004361726420696E736572746564004361D2
:1012800072642072656D6F766564002062696173B7
:101290003A200020643A2000206D696E3A20002038
:1012A0006D61783A2000204B753A20002054753A41
:1012B000200020436C617369632050494420002062
:1012C0004B703A2000204B693A2000204B643A20B2
:1012D0000020536F6D65206F76657273686F6F7451
:1012E0002000204B703A2000204B693A2000204B10
:1012F000643A2000204E6F206F76657273686F6FBE
:10130000742000204B703A2000204B693A200020C6
:101310004B643A2000504944204175746F74756ED7
:1013200065206661696C656420212C2054656D70B0
:101330006572617475726520746F206869676800F2
:101340006F6B20543A0020403A004572726F723A37
:1013500000202D20496E76616C6964206578747276
:1013600075646572206E756D6265722100202D2096
:10137000496E76616C696420657874727564657213
:10138000206E756D6265722021003A204578747276
:1013900075646572207377697463686564206F662D
:1013A000662E204D415854454D5020747269676730
:1013B000657265642021003A204578747275646511
:1013C00072207377697463686564206F66662E2087
:1013D0004D494E54454D502074726967676572657A
:1013E0006420210054656D706572617475726520AA
:1013F00068656174656420626564207377697463ED
:10140000686564206F66662E204D415854454D50E6
:1014100020747269676765726564202121006563C5
:10142000686F3A00534420696E6974206661696C84
:10143000004572726F723A00766F6C756D652E6939
:101440006E6974206661696C6564006F70656E52C8
:101450006F6F74206661696C65640053442063613A
:101460007264206F6B006F70656E206661696C65D9
:10147000642C2046696C653A20002E0046696C6534
:10148000206F70656E65643A002053697A653A0092
:1014900046696C652073656C6563746564006F7084
:1014A000656E206661696C65642C2046696C653ADE
:1014B00020002E006F70656E206661696C65642C7B
:1014C0002046696C653A20002E0057726974696E77
:1014D0006720746F2066696C653A20006F70656ED6
:1014E000206661696C65642C2046696C653A200051
:1014F0002E0046696C652064656C657465643A000D
:1015000044656C6574696F6E206661696C65642CF6
:101510002046696C653A20002E00534420707269A1
:101520006E74696E67206279746520002F004E6FBB
:1015300074205344207072696E74696E670065721E
:10154000726F722077726974696E6720746F20669B
:10155000696C650043616E6E6F7420656E746572B0
:10156000207375626469723A006563686F3A00209F
:10157000636F6C6420657874727573696F6E207028
:10158000726576656E7465640020746F6F206C6F91
:101590006E6720657874727573696F6E20707265FE
:1015A00076656E746564000000090A02080B0C0D74
:1015B0000706030401000000000000000000000016
:1015C000000000000000000000000000000000001B
:1015D00000000011100F00000000000000000000DB
:1015E00000000000000000000000000000010210E8
:1015F000202008081020401020408002010201082D
:1016000004020101020408102040808040201008DC
:101610000402018004020180402010080402010835
:101620000402010102040810204080010204081095
:101630002040800505050507050808080802020284
:10164000020A0A080804040404010101010101015D
:10165000010303030303030303040707070C0C0C34
:101660000C0C0C0C0C02020202060606060606060C
:10167000060B0B0B0B0B0B0B0B00002000230026A3
:101680000029002C002F0032000001000003010699
:1016900001090100002200250028002B002E003146
:1016A00000340002010000050108010B01000021C7
:1016B00000240027002A002D003000330001010023
:1016C00000040107010A01494E46494E4954594E4A
:1016D000414E000020410000C84200401C4620BC92
:1016E000BE4CCA1B0E5AAEC59D74CDCCCC3D0AD79C
:1016F000233C17B7D13877CC2B329595E6241FB110
:101700004F0A2A6D2F6D11241FBECFEFD1E2DEBF2D
:10171000CDBF00E00CBF14E0A0E0B2E0E0E4F7E5EC
:1017200001E00BBF02C007900D92AC38B107D9F7AA
:1017300010E1ACE8B4E001C01D92A635B107E1F7B5
:1017400017E1C4E0D7E100E006C022970109FE01DD
:101750000BBF0E944AA5C230D10780E00807A9F755
:101760000E94EF9D0C948EAB0C940000282F30E06B
:10177000A9015595479540654CBD80FD03C091E09A
:10178000863009F490E09DBD08958FEF8EBD0DB4B5
:1017900007FEFDCF8EB508958EBD0DB407FEFDCFBB
:1017A0000895FC01808161E00E949D9C0895CF9383
:1017B000DF93EC018A810E94B60B888160E00E9471
:1017C0009D9CDF91CF910895CF92DF92EF92FF928F
:1017D0000F931F93CF93DF93EC016B018A010E945B
:1017E0001E9DDC01CB017C010AC00E941E9D6E196A
:1017F0007F0981E06D32780710F081E108C00E9416
:10180000C50B8B838F3F89F38E3F39F08FE089833F
:10181000CE010E94D10B80E027C0980121503040BA
:1018200001151105C9F08FEF8EBDF60180E090E043
:101830004FEF07C00DB407FEFDCF5EB551934EBD0F
:10184000019682179307B0F30DB407FEFDCF8EB556
:101850002C0D3D1DF90180830E94C50B0E94C50B14
:10186000CE010E94D10B81E0DF91CF911F910F91AA
:10187000FF90EF90DF90CF9008950F931F93CF9339
:10188000DF93EB010E941E9D8B019C0107C00E940B
:101890001E9D601B710B6C177D0730F40E94C50BF9
:1018A0008F3FA9F781E001C080E0DF91CF911F91C8
:1018B0000F9108958F929F92AF92BF92EF92FF92F5
:1018C0000F931F93CF937C01C62F49015A010E94A9
:1018D000D70BC7016CE271E00E943D0C8C2F806435
:1018E0000E94CC0B08E110E0D501C401002E04C019
:1018F000B695A795979587950A94D2F70E94CC0B39
:10190000085010408FEF083F180771F7CC2321F0E3
:10191000C83021F08FEF03C085E901C087E80E943D
:10192000CC0BCC3011F40E94C50BC0E00E94C50B5B
:10193000F701838387FF04C0CF3F11F0CF5FF6CF5D
:10194000CF911F910F91FF90EF90BF90AF909F901C
:101950008F900895CF92DF92EF92FF920F931F9393
:10196000CF93DF93EC016A017B0189018C81833085
:1019700039F0A9E0CC0CDD1CEE1CFF1CAA95D1F7B8
:10198000CE0161E1A70196010E945A0C882339F02B
:1019900084E08983CE010E94D10B80E006C0CE0195
:1019A000B80140E052E00E94E40BDF91CF911F911B
:1019B0000F91FF90EF90DF90CF900895AF92BF927C
:1019C000CF92DF92EF92FF920F931F93CF93DF930B
:1019D000EC01162F1C82198248830E941E9DDC0197
:1019E000CB015C01888161E00E947C9CCE010E9459
:1019F000D10B82E360E00E947C9C83E361E00E9463
:101A00007C9C84E361E00E947C9C85E361E00E9411
:101A10007C9C85E361E00E949D9C85E08A830E9416
:101A2000B60B0AE08FEF0E94CC0B0150D9F70AC029
:101A30000E941E9D6A197B0987E0613D780710F0BE
:101A400081E05AC0CE0160E020E030E040E050E0AC
:101A50000E945A0C082F8B83813051F7CE0168E029
:101A60002AEA31E040E050E00E945A0C82FF02C0B6
:101A70000C830CC004E00E94C50B8B830150D9F786
:101A80008A3A11F082E038C082E08C838C81823007
:101A900031F4C12CD12CE12CB0E4FB2E0EC0CC24AF
:101AA000DD2476010AC00E941E9D6A197B0987E029
:101AB000613D780710F08AE01FC0CE0167E320E0A7
:101AC00030E040E050E00E945A0CCE0169E2A701EC
:101AD00096010E945A0C8B83882329F78C818230CF
:101AE000E9F4CE016AE320E030E040E050E00E94FB
:101AF0005A0C882331F088E08983CE010E94D10BF3
:101B000018C00E94C50B807C803C11F483E08C835C
:101B10000E94C50B0E94C50B0E94C50BCE010E94FE
:101B2000D10B173018F088E1898303C01A8381E054
:101B300001C080E0DF91CF911F910F91FF90EF9056
:101B4000DF90CF90BF90AF900895CF93DF93EC01DB
:101B50006EBDFA0180E090E00DB407FEFDCF20815C
:101B60002EBD0DB407FEFDCF21812EBD029632960B
:101B700022E08030920781F70DB407FEFDCF8FEF92
:101B80000E94CC0B8FEF0E94CC0B0E94C50B8B8365
:101B90008F71853039F083E18983CE010E94D10BAA
:101BA00080E001C081E0DF91CF910895CF92DF9274
:101BB000EF92FF920F931F93CF93DF93EC016A0193
:101BC0007B0189018C81833039F089E0CC0CDD1CEC
:101BD000EE1CFF1C8A95D1F7CE0168E1A7019601A2
:101BE0000E945A0C882311F086E01FC0CE016EEFD0
:101BF000A8010E94A50D8823C9F0CE0168E572E016
:101C00000E943D0C882311F487E10FC0CE016DE0E6
:101C100020E030E040E050E00E945A0C882321F49C
:101C20000E94C50B882379F086E18983CE010E944A
:101C3000D10B80E0DF91CF911F910F91FF90EF903A
:101C4000DF90CF900895CE010E94D10B81E0F2CFBA
:101C500080919E04882349F480919D04882329F46F
:101C600080919C04882309F4AEC0EFE2F1E007C044
:101C70009091C00095FFFCCF8093C600319684916F
:101C80008823B1F7E5E3F1E007C09091C00095FF2C
:101C9000FCCF8093C600319684918823B1F7809160
:101CA0009E04882349F1E4E4F1E007C09091C0006C
:101CB00095FFFCCF8093C600319684918823B1F7BD
:101CC00060919F047091A0048091A1049091A2045E
:101CD0000E94CEA12091FF0F309100104091011081
:101CE000509102100E9433A1AB01BC018BE59AE038
:101CF00022E030E00E948F7A80919D04882349F190
:101D0000E8E4F1E007C09091C00095FFFCCF80931C
:101D1000C600319684918823B1F76091A304709135
:101D2000A4048091A5049091A6040E94CEA12091C4
:101D300003103091041040910510509106100E943C
:101D400033A1AB01BC018BE59AE022E030E00E94B8
:101D50008F7A80919C04882349F1ECE4F1E007C07C
:101D60009091C00095FFFCCF8093C600319684917E
:101D70008823B1F76091A7047091A8048091A90409
:101D80009091AA040E94CEA12091071030910810D2
:101D90004091091050910A100E9433A1AB01BC017F
:101DA0008BE59AE022E030E00E948F7A8091C000BB
:101DB00085FFFCCF8AE08093C60010929E041092AB
:101DC0009D0410929C04089510929E0410929D040C
:101DD00010929C040895809307040895EFE6F0E0C4
:101DE00080818260808308951F920F920FB60F92B8
:101DF0000BB60F9211240F931F932F933F934F9382
:101E00005F936F937F938F939F93AF93BF93CF9382
:101E1000DF93EF93FF938091AF049091B00400970C
:101E200009F082C19091E20A8091E10A9817A1F02D
:101E30002091E10A30E08DE490E0289FF001299F95
:101E4000F00D389FF00D1124ED51F54FDF01A45B2B
:101E5000BF4F81E08C9302C0E0E0F0E0F093B0046B
:101E6000E093AF04309709F459C11092B104109275
:101E7000B2041092B3041092B40464AD75AD7093C3
:101E8000B6046093B5042CE96134720728F48EE43B
:101E90006132780748F002C060E47CE97695679586
:101EA0007695679584E007C0E7E261317E0730F000
:101EB0007695679582E08093B70408C081E08093AF
:101EC000B7046032710510F460E270E06052704057
:101ED000F8E060307F07E0F0272F30E0220F331F5B
:101EE000220F331F205B3E4FF9013296859194916A
:101EF000AA27699FE001689FC10DDA1F0694CA1FD7
:101F0000DA1F1124F901459154914C1B5D0B1FC040
:101F1000CB01969587958C7F805B9A4FFC0145910C
:101F200054910296FC01A591B491862F90E08770A0
:101F30009070A89F9001A99F300DB89F300D11247B
:101F4000D3E036952795DA95E1F7421B530B4436DB
:101F50005105A0F4E0E0F2E006C09091C00095FFCA
:101F6000FCCF8093C60081918823B9F78BE59AE076
:101F70004AE050E00E94B47944E650E0CA01A0E093
:101F8000B0E08093B8049093B904A093BA04B093DE
:101F9000BB045093890040938800E091AF04F09116
:101FA000B00460AD71AD2CE96134720728F48EE4A1
:101FB0006132780748F002C060E47CE97695679565
:101FC0007695679584E007C0E7E261317E0730F0DF
:101FD0007695679582E08093B70408C081E080938E
:101FE000B7046032710510F460E270E06052704036
:101FF000F8E060307F07E0F0272F30E0220F331F3A
:10200000220F331F205B3E4FF90132968591949148
:10201000AA27699FE001689FC10DDA1F0694CA1FB5
:10202000DA1F1124F901459154914C1B5D0B1FC01F
:10203000CB01969587958C7F805B9A4FFC014591EB
:1020400054910296FC01A591B491862F90E087707F
:102050009070A89F9001A99F300DB89F300D11245A
:10206000E3E036952795EA95E1F7421B530B44369A
:102070005105A0F4E0E0F2E006C09091C00095FFA9
:10208000FCCF8093C60081918823B9F78BE59AE055
:102090004AE050E00E94B47944E650E05093BD0419
:1020A0004093BC04E091AF04F091B0048089918921
:1020B000A289B389B695A79597958795B095A09570
:1020C000909581959F4FAF4FBF4F8093BE049093E3
:1020D000BF04A093C004B093C1048093C204909342
:1020E000C304A093C404B093C5048093C604909322
:1020F000C704A093C804B093C9048093CA04909302
:10210000CB04A093CC04B093CD041092AB041092F6
:10211000AC041092AD041092AE0406C080ED97E0BE
:102120009093890080938800E091AF04F091B0040F
:10213000309709F41AC580A18093CE0480FF37C080
:10214000119A8FEF8093030420B1217031E023278F
:1021500059F18091CF04882339F180819181A28146
:10216000B381181619061A061B06F4F480918C0424
:1021700090918D04A0918E04B0918F0480939F0460
:102180009093A004A093A104B093A20430939E0462
:1021900080899189A289B3898093AB049093AC0420
:1021A000A093AD04B093AE042093CF0436C0119831
:1021B00081E08093030421E0029B02C020E02BC059
:1021C0008091D004882339F180819181A281B381EB
:1021D000181619061A061B06F4F480918C049091C7
:1021E0008D04A0918E04B0918F0480939F049093EE
:1021F000A004A093A104B093A20420939E0480891C
:102200009189A289B3898093AB049093AC04A09385
:10221000AD04B093AE042093D0048091CE0481FF2E
:102220003BC044988FEF8093040421E0049B02C0DC
:1022300020E02FC08091D104882359F1E091AF04B0
:10224000F091B00484819581A681B7811816190692
:102250001A061B06F4F48091900490919104A091C9
:102260009204B09193048093A3049093A404A09348
:10227000A504B093A60420939D0480899189A28926
:10228000B3898093AB049093AC04A093AD04B09356
:10229000AE042093D1043AC0449A81E080930404B0
:1022A00021E0069B02C020E02FC08091D204882349
:1022B00059F1E091AF04F091B00484819581A68139
:1022C000B781181619061A061B06F4F480919004BB
:1022D00090919104A0919204B09193048093A304EF
:1022E0009093A404A093A504B093A60420939D0406
:1022F00080899189A289B3898093AB049093AC04BF
:10230000A093AD04B093AE042093D2048091CE0488
:1023100082FF3DC0A29A8FEF8093050426B12095DD
:10232000221F2227221F81F18091D304882361F18B
:10233000E091AF04F091B00480859185A285B385CA
:10234000181619061A061B06FCF480919404909145
:102350009504A0919604B09197048093A70490935C
:10236000A804A093A904B093AA0481E080939C04DC
:1023700080899189A289B3898093AB049093AC043E
:10238000A093AD04B093AE042093D3043AC0A298B6
:1023900081E08093050421E0359B02C020E02FC03E
:1023A0008091D404882359F1E091AF04F091B004F6
:1023B00080859185A285B385181619061A061B0615
:1023C000F4F48091940490919504A0919604B091B6
:1023D00097048093A7049093A804A093A904B093B2
:1023E000AA0420939C0480899189A289B38980934F
:1023F000AB049093AC04A093AD04B093AE042093CF
:10240000D4048091CE049FB7F89483FF08C08091D4
:102410000B018F7E80930B019FBF8FEF07C08091D0
:102420000B01806180930B019FBF81E080930604C4
:10243000C0E0D0E086C18091C00087FF1AC06091E3
:10244000C6008091DC0A9091DD0AAC014F5F5F4FBE
:102450004F7750702091DE0A3091DF0A4217530700
:1024600041F0845A954FFC0160835093DD0A4093FC
:10247000DC0AE091AF04F091B0044091BE045091A9
:10248000BF046091C0047091C10480819181A281D8
:10249000B381480F591F6A1F7B1F4093BE0450939E
:1024A000BF046093C0047093C10414161506160689
:1024B000170644F5139A80899189A289B389481B2C
:1024C000590B6A0B7B0B4093BE045093BF0460937F
:1024D000C0047093C104139880918C0490918D0472
:1024E000A0918E04B0918F0420910304820F911D5E
:1024F000A11DB11D80938C0490938D04A0938E0434
:10250000B0938F04E091AF04F091B0044091C20405
:102510005091C3046091C4047091C5048481958175
:10252000A681B781480F591F6A1F7B1F4093C204C1
:102530005093C3046093C4047093C5041416150625
:102540001606170644F5469A80899189A289B389AF
:10255000481B590B6A0B7B0B4093C2045093C30476
:102560006093C4047093C504469880919004909140
:102570009104A0919204B091930420910404820FDD
:10258000911DA11DB11D8093900490939104A0937F
:102590009204B0939304E091AF04F091B0044091A1
:1025A000C6045091C7046091C8047091C904808525
:1025B0009185A285B385480F591F6A1F7B1F4093E1
:1025C000C6045093C7046093C8047093C9041416DA
:1025D00015061606170644F5409A80899189A28946
:1025E000B389481B590B6A0B7B0B4093C60450936D
:1025F000C7046093C8047093C90440988091940400
:1026000090919504A0919604B091970420910504AF
:10261000820F911DA11DB11D809394049093950488
:10262000A0939604B0939704E091AF04F091B004A6
:102630008091CA049091CB04A091CC04B091CD04B8
:102640004485558566857785840F951FA61FB71F1E
:102650008093CA049093CB04A093CC04B093CD0490
:10266000181619061A061B060CF042C09FB7F894FC
:1026700080910B01806480930B019FBFE091AF04B8
:10268000F091B0048091CA049091CB04A091CC0445
:10269000B091CD044089518962897389841B950B5F
:1026A000A60BB70B8093CA049093CB04A093CC04E1
:1026B000B093CD049FB7F89480910B018F7B8093EA
:1026C0000B019FBF8091980490919904A0919A0466
:1026D000B0919B0420910604820F911DA11DB11D94
:1026E0008093980490939904A0939A04B0939B04C8
:1026F0008091AB049091AC04A091AD04B091AE0474
:102700000196A11DB11D8093AB049093AC04A093DE
:10271000AD04B093AE048091AB049091AC04A09151
:10272000AD04B091AE042196E091AF04F091B004F5
:10273000408951896289738984179507A607B7076D
:1027400038F48091B70490E0C817D9070CF473CE21
:102750004091AB045091AC046091AD047091AE0413
:10276000E091AF04F091B00484899589A689B78976
:1027700084179507A607B70708F4DCC00091B804D2
:102780001091B9042091BA043091BB04448D558D49
:10279000668D778DAA27059FB12D169FC001269FB4
:1027A000900D259F800D911D069FB00D811D9A1FD4
:1027B000159FB00D811D9A1F249FB00D811D9A1F7A
:1027C000149FB10D8A1F9A1FB6958A1F9A1F112454
:1027D00024AD35AD280F391F3093B6042093B504CE
:1027E00080AD91ADA2ADB3ADA90160E070E08417FA
:1027F0009507A607B70720F49093B6048093B50415
:102800006091B5047091B604FCE961347F0728F447
:102810002EE46132720748F002C060E47CE97695EC
:1028200067957695679584E007C087E26131780700
:1028300030F07695679582E08093B70408C081E018
:102840008093B7046032710510F460E270E060526A
:102850007040E8E060307E07E0F0272F30E0220F84
:10286000331F220F331F205B3E4FF90132968591B3
:102870009491AA27699FE001689FC10DDA1F069411
:10288000CA1FDA1F1124F901459154914C1B5D0BAD
:102890001FC0CB01969587958C7F805B9A4FFC017A
:1028A000459154910296FC01A591B491862F90E038
:1028B00087709070A89F9001A99F300DB89F300D30
:1028C0001124D3E036952795DA95E1F7421B530B97
:1028D00044365105A0F4E0E0F2E006C09091C0005B
:1028E00095FFFCCF8093C60081918823B9F78BE5D3
:1028F0009AE04AE050E00E94B47944E650E05093F8
:1029000089004093880060E070E08091B804909165
:10291000B904A091BA04B091BB04840F951FA61FFF
:10292000B71F8093B8049093B904A093BA04B093EE
:10293000BB04F6C04091AB045091AC046091AD046F
:102940007091AE04808D918DA28DB38D8417950703
:10295000A607B70708F0DCC00091B1041091B204DB
:102960002091B3043091B404448D558D668D778DDC
:10297000AA27059FB12D169FE001269FD00D259F08
:10298000C00DD11D069FB00DC11DDA1F159FB00DE2
:10299000C11DDA1F249FB00DC11DDA1F149FB10D98
:1029A000CA1FDA1FB695CA1FDA1F11248091B50419
:1029B0009091B604E05CFF4F8C179D0718F480815E
:1029C000918102C08C1B9D0B40815181628173817A
:1029D0008C0120E030E0041715072607370708F4BC
:1029E000CA01FCE981349F0728F42EE48132920762
:1029F00048F002C080E49CE9969587959695879566
:102A000024E007C0E7E281319E0730F09695879574
:102A100022E02093B70408C021E02093B70480325D
:102A2000910510F480E290E0BC0160527040F8E043
:102A300060307F07E0F0272F30E0220F331F220F96
:102A4000331F205B3E4FF901329685919491AA275E
:102A5000699FE001689FC10DDA1F0694CA1FDA1F43
:102A60001124F901459154914C1B5D0B1FC0CB0102
:102A7000969587958C7F805B9A4FFC014591549188
:102A80000296FC01A591B491862F90E0877090701A
:102A9000A89F9001A99F300DB89F300D1124E3E04D
:102AA00036952795EA95E1F7421B530B44365105BD
:102AB000A0F4E0E0F2E006C09091C00095FFFCCFEA
:102AC0008093C60081918823B9F78BE59AE04AE0AC
:102AD00050E00E94B47944E650E05093890040935E
:102AE000880060E070E08091B1049091B204A09100
:102AF000B304B091B404840F951FA61FB71F809331
:102B0000B1049093B204A093B304B093B40408C08A
:102B10008091BC049091BD049093890080938800BB
:102B20004091AB045091AC046091AD047091AE043F
:102B3000E091AF04F091B00480899189A289B389B2
:102B4000481759076A077B0780F01092B00410926B
:102B5000AF049091E20A8091E10A981731F08091D8
:102B6000E10A8F5F8F708093E10AFF91EF91DF910F
:102B7000CF91BF91AF919F918F917F916F915F9115
:102B80004F913F912F911F910F910F900BBE0F907E
:102B90000FBE0F901F901895099A3C9A9A9AEAE0F6
:102BA000F1E08081806180838081846080830D9AE0
:102BB000159A0F9A179A3A9A429A989AA09A229A34
:102BC0002A9A0898109A0A98129A0C98149A0E98B1
:102BD000169A3F98479A3D98459A0B9A159A3E9AAD
:102BE000179A389A429A808180648083A09A808163
:102BF000816080832A9AA1E8B0E08C918F7E8C93CB
:102C00008C9188608C93E0E8F0E080818D7F8083F8
:102C100080818E7F808380818F73808380818F7C91
:102C200080838C91887F82608C9380E090E4909385
:102C30008900809388001092850010928400EFE64E
:102C4000F0E080818260808381E080930704789443
:102C500008959091E20A8091E10A981741F00E944C
:102C6000EF6D81E00E94882C0E946358F2CF089596
:102C7000CF93DF93EFB7F894EC0188819981AA8113
:102C8000BB8180938C0490938D04A0938E04B093A9
:102C90008F04EB0188819981AA81BB818093900484
:102CA00090939104A0939204B0939304EA018881D5
:102CB0009981AA81BB818093940490939504A093F9
:102CC0009604B0939704E90188819981AA81BB8118
:102CD0008093980490939904A0939A04B0939B04D2
:102CE000EFBFDF91CF9108952FB7F894FC01808159
:102CF0009181A281B3818093980490939904A093C9
:102D00009A04B0939B042FBF08950F931F939FB70E
:102D1000F894E82FF0E0EE0FFF1FEE0FFF1FE457CF
:102D2000FB4F00811181228133819FBFB801C9010E
:102D30001F910F9108950E94291680E599E00E9445
:102D4000022C159A179A429AA09A089580916F00C2
:102D50008D7F80936F0006C08091E10A8F5F8F7036
:102D60008093E10A9091E20A8091E10A981751F468
:102D70001092B0041092AF0480916F008260809333
:102D80006F0008959091E20A8091E10A981751F33B
:102D9000E3CFCF93DF93EC019C012C5F3F4F898DF4
:102DA0009A8D41E050E060E070E00E94DC218823D1
:102DB000A1F08D899E89AF89B88D0097A105B105D5
:102DC00071F48C819D81AE81BF818D8B9E8BAF8B89
:102DD000B88F89818068898302C080E001C081E06A
:102DE000DF91CF910895CF92DF92EF92FF920F93F0
:102DF0001F93CF938C01FC0181899289A389B489A7
:102E0000803EFFEF9F07FFE1AF07F0E0BF0708F04C
:102E100079C0C8010E94C916882309F473C00E94B2
:102E2000DC1F882309F46EC0D8015996ED91FC91FE
:102E30005A971496CD90DD90ED90FC9017978EEFF9
:102E40009FEFAFEFBFEFC80ED91EEA1EFB1E058431
:102E500004C0CC0CDD1CEE1CFF1C0A94D2F7868546
:102E60009785A089B189C80ED91EEA1EFB1E81E094
:102E70008093DB04C092DE06D092DF06E092E0068B
:102E8000F092E10680E092E0EEEDF4E0DF019C01DB
:102E90001D9221503040E1F7C1E011C0B701A601F9
:102EA0004C0F511D611D711D8091DC049091DD045A
:102EB0002EED34E00E94D60D882321F1CF5FD8019A
:102EC0005996ED91FC915A978481C81738F380E0A8
:102ED00092E0A0E0B0E0058404C0880F991FAA1F0B
:102EE000BB1F0A94D2F7F80141895289638974891A
:102EF000480F591F6A1F7B1F418B528B638B748B4A
:102F000081E001C080E0CF911F910F91FF90EF9081
:102F1000DF90CF900895CF93DF93EC018C859D8552
:102F2000AE85BF8541E0662309F440E0BC01CD01D8
:102F30000E941920882351F0888990E025E0880FAD
:102F4000991F2A95E1F782529B4F02C080E090E0E2
:102F5000DF91CF910895FC0190E080E02EE2308176
:102F6000303269F0983029F4DB01A80FB11D2C93A1
:102F70008F5F3081DB01A80FB11D3C938F5F9F5F96
:102F800031969B3061F7680F711DFB011082089527
:102F9000CF93DF93EB01FC012381222389F02250A0
:102FA000223020F48FE28883198208C060E00E94FA
:102FB0008B17009729F0BE010E94AB1781E001C07A
:102FC00080E0DF91CF910895CF93DF93EA01FB0179
:102FD0002BE030E231932150E9F7DC0130E047E0AB
:102FE0001CC04A3069F138E04AE017C0E21741F1ED
:102FF000FC010196E491EE23C9F7431708F1213251
:10300000F8F02F37E8F4FB01E30FF11D822F815612
:103010008A3108F4205220833F5F9A2F8B2F2D9105
:10302000222339F02F3229F02E32D9F28AE599E0A5
:10303000DFCF9883898381E0FB019081903209F48E
:1030400080E0DF91CF9108950F931F93CF93DF938B
:10305000EC018B018B81882309F040C0FB0187893B
:10306000803109F041C082E08B831D8A1E8A1F8A4D
:10307000188E808D918DA0E0B0E035E0880F991F0B
:10308000AA1FBB1F3A95D1F7898B9A8BAB8BBC8B50
:1030900013C083E08B83F801428D538D648D758D51
:1030A0004D8B5E8B6F8B788F9E012F5E3F4FC801DB
:1030B0000E94D620882391F01A8F098F81E089839E
:1030C0001C821D821E821F82188619861A861B8604
:1030D0001C861D861E861F86188A01C080E0DF912F
:1030E000CF911F910F9108958032C1F7D2CF2F92C7
:1030F0003F924F925F926F927F928F929F92AF9288
:10310000BF92CF92DF92EF92FF920F931F93CF93D4
:10311000DF9300D000D0CDB7DEB79C838B83662EC3
:10312000272E2A01DC0113968C911397882309F42A
:10313000D2C011968C91119780FFCDC0E7C02A01B3
:10314000481A590A5201862C922CEB81FC81349644
:10315000FA83E983212C02E0302EB7C0EB81FC8199
:1031600080859185A285B3857FEF672E71E0772EEC
:103170006822792223816C017D0119E0F694E7949D
:10318000D794C7941A95D1F7418D528D5E834D83A4
:10319000223061F4DA015A964D915D916D917C91E6
:1031A0005D974C0D5D1D6E1D7F1D4EC0ED81FE8136
:1031B000048101500C216114710411F5002301F503
:1031C0000097A105B10559F4EB81FC8185899689A9
:1031D000A789B08D84839583A683B78311C0AB8103
:1031E000BC8114964D915D916D917C9117978D8165
:1031F0009E8129813A810E945320882309F46BC063
:10320000AB81BC815996ED91FC915A9714964D91E2
:103210005D916D917C911797425050406040704095
:10322000058404C0440F551F661F771F0A94D2F708
:1032300086859785A089B189480F591F6A1F7B1F12
:10324000400F511D611D711DC1018619970985012E
:103250008A159B0508F48C01B2E000301B0709F0C9
:1032600073C08091DE069091DF06A091E006B091D8
:10327000E106481759076A077B0709F465C0809182
:10328000DC049091DD0494010E94AA0C882341F48F
:1032900022C0B30162527B4FC401A8010E9441A821
:1032A000800E911EA80160E070E0EB81FC818085BA
:1032B0009185A285B385840F951FA61FB71F8087B0
:1032C0009187A287B387A01AB10AA114B10409F0AB
:1032D00045CFC20102C08FEF9FEF26960FB6F8943C
:1032E000DEBF0FBECDBFDF91CF911F910F91FF9039
:1032F000EF90DF90CF90BF90AF909F908F907F9096
:103300006F905F904F903F902F900895AB81BC815C
:1033100051964D915D916D917C91549718968D9138
:103320009D910D90BC91A02D820120E030E06A01BA
:103330007B01C81AD90AEA0AFB0A0C151D052E05DD
:103340003F0508F0FCCEFECECB01BA0140E00E9462
:103350001920882309F09DCFBECFCF93DF930F9222
:10336000CDB7DEB7BE016F5F7F4F41E050E00E94F6
:1033700077188130910519F4898190E002C08FEFB0
:103380009FEF0F90DF91CF9108950F931F93CF93ED
:10339000DF938C01EB01FC018381823020F1808579
:1033A0009185A285B3858F719070A070B0700097E1
:1033B000A105B105C1F4C801BE0140E250E00E9480
:1033C00077188032910519F0009769F40EC0888152
:1033D000882359F0853E79F38E3269F38B8583FD1E
:1033E000EACF80E203C08FEF01C080E0DF91CF9190
:1033F0001F910F910895CF92DF92EF92FF92CF939A
:10340000DF93EC018B81823038F1C884D984EA845F
:10341000FB84CE010E94AD1997FD1EC08885998559
:10342000AA85BB854F96A11DB11D88879987AA875C
:10343000BB87D701C60125E0B695A79597958795D7
:103440002A95D1F78F7090E035E0880F991F3A9553
:10345000E1F782529B4F02C080E090E0DF91CF9174
:10346000FF90EF90DF90CF9008958F929F92AF9250
:10347000BF92CF92DF92EF92FF920F931F93CF9361
:10348000DF93EC014A015B012B81222309F475C013
:1034900089899A89AB89BC8984179507A607B707DC
:1034A00008F46BC078C081149104A104B10449F4FC
:1034B0001C821D821E821F82188619861A861B8610
:1034C0005AC0488559856A857B85E98DFA8D2585A1
:1034D00030E0275F3F4FDB01CA010197A109B10925
:1034E000022E04C0B695A795979587950A94D2F7B2
:1034F000750164010894C108D108E108F10804C00D
:10350000F694E794D794C7942A95D2F7C816D906AB
:10351000EA06FB0628F0411551056105710549F4DD
:103520008D899E89AF89B88D8C839D83AE83BF833F
:1035300016C0C81AD90AEA0AFB0A11C04C815D817B
:103540006E817F81898D9A8D98010E945320089405
:10355000C108D108E108F108882321F40EC08E01CA
:103560000C5F1F4FC114D104E104F10439F78886C0
:103570009986AA86BB8681E001C080E0DF91CF9169
:103580001F910F91FF90EF90DF90CF90BF90AF9081
:103590009F908F900895223009F085CFE8CF40E0CA
:1035A00050E060E070E00E94351A08950F931F9379
:1035B000CF93DF938C01FC0183818823C9F1818142
:1035C00087FF33C0C80161E00E948B17EC010097B0
:1035D00079F18881853E61F1F8018381823040F480
:1035E00081899289A389B4898C8F9D8FAE8FBF8F7B
:1035F000F80185899689A789B08D9B8F8A8FBD8BAD
:10360000AC8BE091D504F091D604309751F0BE0117
:103610006A5E7F4FCE0148961995888D998D9B8B58
:103620008A8BF80181818F7781830E94DC1F04C01F
:1036300081E0F801808380E0DF91CF911F910F91AD
:103640000895CF93DF93EC010E94D61A1B82DF917D
:10365000CF910895CF93DF93EC018B81882321F0E4
:10366000CE010E94D61A1B82DF91CF9108954F920E
:103670005F926F927F928F929F92AF92BF92EF92E2
:10368000FF920F931F93CF93DF9300D00F92CDB78C
:10369000DEB77C014A015B01FC018381813009F0C6
:1036A00085C0818181FF82C095C00097A105B105C9
:1036B00009F47AC0F7014084518462847384C7019D
:1036C000B501A4010E94351A882309F46FC0F701DF
:1036D000818D928D81149104A104B10479F44589FE
:1036E00056896789708D0E94ED22882309F45EC097
:1036F000F701158A168A178A108E3CC0F70144819B
:103700005581668177819E012F5F3F4F0E94532034
:10371000882309F44BC0F701818D928D49815A812C
:103720006B817C81FC012789203149F4483FFFEF00
:103730005F07F0E06F07F0E07F07E0F408C0483F64
:103740002FEF52072FEF62072FE0720798F40E94C5
:10375000ED22882359F1F7014481558166817781F3
:10376000818D928D0FEF1FEF2FEF3FE00E944421DC
:103770008823E1F0F701818A928AA38AB48A818141
:1037800080688183C7010E94D61A882379F0B50129
:10379000A401481459046A047B0410F4B301A20183
:1037A000C7010E94351A03C081E001C080E00F907C
:1037B0000F900F900F90DF91CF911F910F91FF907D
:1037C000EF90BF90AF909F908F907F906F905F90A1
:1037D0004F900895F70181899289A389B48984174C
:1037E0009507A607B70708F060CFE0CFCF93DF9328
:1037F000EC0140E050E060E070E00E94371B88235D
:1038000069F0CE0161E00E948B17009739F025EE38
:10381000FC0120831B820E94DC1F01C080E0DF913D
:10382000CF9108951F93CF93DF93EC01142FE62FD0
:10383000F0E035E0EE0FFF1F3A95E1F7E252FB4F63
:103840008385817121F0842F827109F05DC08091A0
:10385000DE069091DF06A091E006B091E1068C872C
:103860009D87AE87BF87688B4489558960E070E08B
:10387000BA0155274427828D938DA0E0B0E0482BF4
:10388000592B6A2B7B2B4D8B5E8B6F8B788F8385AF
:1038900090E088719070009751F4848D958DA68D7D
:1038A000B78D898B9A8BAB8BBC8B81E00DC080313F
:1038B000910551F59E012F5E3F4F898D9A8D0E9493
:1038C000D620882309F184E08B83812F8F70898330
:1038D0001C821D821E821F82188619861A861B86EC
:1038E00014FF18C0CE0140E050E060E070E00E949C
:1038F000371B882351F00EC049895A896B897C890E
:10390000CE010E94351A02C01B8280E0DF91CF9168
:103910001F91089515FDF0CF81E0F8CF7F928F922F
:103920009F92AF92BF92CF92DF92EF92FF920F934E
:103930001F93CF93DF935C01EB01942E852E722EA3
:10394000898D9A8DF501928F818FCB010E94CF1ABC
:1039500010E037C0CE010E94FB19BC01009709F4AA
:1039600090C0D701C60135E0B695A7959795879584
:103970003A95D1F7082F0F70FB018081882311F051
:10398000853EB1F4112379F48091DE069091DF0633
:10399000A091E006B091E106F50184879587A6879E
:1039A000B787008B11E0FB018081882351F417C099
:1039B000892D982D4BE050E00E9434A8009709F41F
:1039C0006FC0C884D984EA84FB8489899A89AB89C9
:1039D000BC89C816D906EA06FB0608F4BBCF76FEFA
:1039E00050C071FE4EC0112351F0F5010089C50190
:1039F00061E00E948B17EC01009769F442C08B8153
:103A0000823009F43EC0CE010E94F3168823C9F12A
:103A1000CEEDD4E000E080E2FE0111928A95E9F754
:103A2000FE01A92DB82D8BE00D9001928150E1F798
:103A3000E091D504F091D604309739F0BE01625F71
:103A40007F4FCE014096199508C081E298E2998B8C
:103A5000888B80E098E09F878E87888999899B8BE7
:103A60008A8B998F888F8E859F859F8B8E8B0E94E6
:103A7000DC1F882331F0C501602F472D0E94121CE6
:103A800001C080E0DF91CF911F910F91FF90EF90E7
:103A9000DF90CF90BF90AF909F908F907F900895D0
:103AA00077FEE9CFEECF5F926F927F928F929F92D7
:103AB000AF92BF92CF92DF92EF92FF920F931F933C
:103AC000CF93DF93CDB7DEB7C354D0400FB6F89491
:103AD000DEBF0FBECDBF4C016B0124965FAF4EAF72
:103AE0002497522E1FA21AA61C861F8661157105E7
:103AF00009F47AC0FC018381882309F075C0FA01BA
:103B000080818F3291F405C031962496FFAFEEAFDD
:103B100024972496EEADFFAD249780818F32A1F3D8
:103B2000F60183818250823050F4860157E2E52EFF
:103B3000F12CEC0EFD1E3701BE2CAF2C11C0F6018E
:103B4000618D728DCE010C960E942418882309F491
:103B50004BC08E01045F1F4FE9CF8701EB2CFA2C7D
:103B600024968EAD9FAD2497BE016F5F7F4FAE014F
:103B70004E5B5F4F0E94E417882331F435C03196C5
:103B80002496FFAFEEAF24972496EEADFFAD2497B9
:103B900080818F32A1F38823E9F0C701B801AE011B
:103BA0004F5F5F4F21E00E948E1C8823E9F00C15C7
:103BB0001D0529F0C8010E94D61AF8011382E614E7
:103BC000F70459F64CE0E42EF12CEC0EFD1E0B2D03
:103BD0001A2DC6CFC401B801AE014F5F5F4F252D2E
:103BE0000E948E1C082F01C000E0CE010C960E949E
:103BF0002A1BCE0187960E942A1B802FCD5BDF4FA8
:103C00000FB6F894DEBF0FBECDBFDF91CF911F91ED
:103C10000F91FF90EF90DF90CF90BF90AF909F906B
:103C20008F907F906F905F9008951F93CF93DF9355
:103C3000CDB7DEB76B970FB6F894DEBF0FBECDBF22
:103C40009C01AB0119821C82CE010196B90122E0D0
:103C50000E94531D882331F0CE0101960E94F61B6D
:103C6000182F01C010E0CE0101960E942A1B812F5F
:103C70006B960FB6F894DEBF0FBECDBFDF91CF912C
:103C80001F9108952F923F924F925F926F927F9271
:103C90008F929F92BF92CF92DF92EF92FF920F93FB
:103CA0001F93CF93DF9300D000D0CDB7DEB78C0148
:103CB000B62EC72E5E834D83DC0113968C9113972D
:103CC000813009F059C111968C91119781FF54C12F
:103CD00070C1F80141895289638974898085918511
:103CE000A285B38584179507A607B70731F0C801E9
:103CF0000E94351A882309F43FC14D805E802B2C29
:103D00003C2C07C1F801218D328DF901B480BA94A1
:103D1000AC01BD01032E39E076956795579547951F
:103D20003A95D1F7302DB4224FEF642E41E0742E36
:103D300068227922BB2009F04BC06114710409F09C
:103D400047C0D80114964D915D916D917C91179764
:103D5000411551056105710559F455968D919D9157
:103D60000D90BC91A02D0097A105B10561F525C06E
:103D7000C9019E012F5F3F4F0E945320882309F401
:103D8000FBC089819A81AB81BC81F801218D328D84
:103D9000F9012789203149F4883FFFEF9F07F0E0C0
:103DA000AF07F0E0BF0748F40EC0883F2FEF92073F
:103DB0002FEFA2072FE0B20730F0C8010E94C9160A
:103DC000882331F4D9C0F80184839583A683B7830F
:103DD00080E092E08619970942018415950508F460
:103DE0004C01D8015996ED91FC915A971496CD90BB
:103DF000DD90ED90FC9017978EEF9FEFAFEFBFEF48
:103E0000C80ED91EEA1EFB1E058404C0CC0CDD1CA6
:103E1000EE1CFF1C0A94D2F786859785A089B1898C
:103E2000C80ED91EEA1EFB1ECB0CD11CE11CF11CD6
:103E300090E0891692E0990639F58091DE0690911E
:103E4000DF06A091E006B091E1068C159D05AE0558
:103E5000BF0571F41092DB048FEF9FEFAFEFBFEF60
:103E60008093DE069093DF06A093E006B093E10610
:103E70008091DC049091DD04B701A60191010E94BC
:103E8000D60D882391F578C061147104F9F4F80116
:103E900080859185A285B38541895289638974891A
:103EA00084179507A607B70788F00E94DC1F8823B0
:103EB00009F462C081E08093DB04C092DE06D092F8
:103EC000DF06E092E006F092E10608C0C701B60105
:103ED00041E00E941920882309F44EC0C301825298
:103EE0009B4FB101A4010E9441A8A40160E070E0D1
:103EF000F80180859185A285B385840F951FA61F43
:103F0000B71F80879187A287B387280C391C481870
:103F10005908F80180859185A285B3854114510423
:103F200009F0F0CE4189528963897489481759078D
:103F30006A077B0740F4818B928BA38BB48B8181C2
:103F4000806881830DC08091D5049091D60400973C
:103F500039F08D819E81009719F08181806881837D
:103F6000F801818183FF05C0C8010E94D61A882309
:103F700019F08D819E8105C081E0D8018C938FEF6F
:103F80009FEF26960FB6F894DEBF0FBECDBFDF9130
:103F9000CF911F910F91FF90EF90DF90CF90BF9046
:103FA0009F908F907F906F905F904F903F902F9059
:103FB000089582FD8ECEA1CE8091DB04882399F1F5
:103FC0004091DE065091DF066091E0067091E106B7
:103FD0008091DC049091DD042EED34E00E94D60D3A
:103FE000882319F14091D7045091D8046091D904E5
:103FF0007091DA04411551056105710591F08091C8
:10400000DC049091DD042EED34E00E94D60D88236F
:1040100071F01092D7041092D8041092D904109223
:10402000DA041092DB0481E0089580E0089580E0D6
:104030000895CF92DF92EF92FF92CF936B017C01B4
:10404000C42F8091DE069091DF06A091E006B0912A
:10405000E1068C159D05AE05BF05C1F00E94DC1F71
:104060008823D1F08091DC049091DD04B701A60192
:104070002EED34E00E94AA0C882371F0C092DE0677
:10408000D092DF06E092E006F092E10681E0CC23D8
:1040900021F08093DB0401C080E0CF91FF90EF908E
:1040A000DF90CF900895CF92DF92EF92FF920F931F
:1040B0001F93CF93DF93EC016A017B01890189850E
:1040C0009A85AB85BC850196A11DB11D8417950706
:1040D000A607B70708F460C08F89803129F4BB2791
:1040E000AF2D9E2D8D2D0CC0803209F055C0DB0107
:1040F000CA0147E0B695A795979587954A95D1F758
:104100004B895C896D897E89840F951FA61FB71F17
:104110004091DE065091DF066091E0067091E10665
:1041200084179507A607B70739F0BC01CD0140E019
:104130000E941920882381F18F89803191F48FEFBB
:1041400090E0A0E0B0E0C822D922EA22FB22F601EA
:10415000EE0FFF1FE252FB4F80819181A0E0B0E0A3
:1041600014C08FE790E0A0E0B0E0C822D922EA2294
:10417000FB22F601EE0FFF1FEE0FFF1FE252FB4F77
:1041800080819181A281B381BF70F8018083918386
:10419000A283B38381E001C080E0DF91CF911F91C2
:1041A0000F91FF90EF90DF90CF9008956F927F92E4
:1041B0008F929F92AF92BF92CF92DF92EF92FF9237
:1041C0000F931F93CF93DF9300D00F92CDB7DEB73D
:1041D0008C0149835A836B837C833901CC24DD2491
:1041E0007601812CE2E09E2EA12CB12C49815A81CE
:1041F0006B817C81C8019E012F5F3F4F0E9453203D
:10420000882371F1D501C401F801058404C0880F29
:10421000991FAA1FBB1F0A94D2F7C80ED91EEA1E07
:10422000FB1E89819A81AB81BC812789203149F4A9
:10423000883FFFEF9F07F0E0AF07F0E0BF0748F4CB
:10424000D5CF883F2FEF92072FEFA2072FE0B207BD
:1042500068F2F301C082D182E282F38281E001C080
:1042600080E00F900F900F900F90DF91CF911F91F2
:104270000F91FF90EF90DF90CF90BF90AF909F9005
:104280008F907F906F9008954F925F926F927F9280
:104290008F929F92AF92BF92CF92DF92EF92FF9256
:1042A0000F931F93CF93DF93EC014A015B01280129
:1042B0003901423051056105710508F46BC08985EB
:1042C0009A85AB85BC850196A11DB11D8417950704
:1042D000A607B70708F45EC08F89803129F4C52E80
:1042E000D62EE72EFF240CC0803209F053C06A019D
:1042F0007B0187E0F694E794D794C7948A95D1F729
:104300008B899C89AD89BE89C80ED91EEA1EFB1E09
:10431000C701B60141E00E9419208823D9F18F8995
:10432000803181F48FEF90E0A0E0B0E08822992204
:10433000AA22BB22F401EE0FFF1FE252FB4F518273
:10434000408213C08FE790E0A0E0B0E0882299227D
:10435000AA22BB22F401EE0FFF1FEE0FFF1FE25255
:10436000FB4F40825182628273828A89823080F060
:104370008D819E81AF81B8858C0D9D1DAE1DBF1DA9
:104380008093D7049093D804A093D904B093DA040F
:1043900081E001C080E0DF91CF911F910F91FF90EC
:1043A000EF90DF90CF90BF90AF909F908F907F90D5
:1043B0006F905F904F9008952F923F924F925F922F
:1043C0006F927F928F929F92AF92BF92CF92DF9225
:1043D000EF92FF920F931F93CF93DF93CDB7DEB78A
:1043E0002F970FB6F894DEBF0FBECDBF1C014C87D0
:1043F0005D876E877F873B872A87DC0119962D9121
:104400003D914D915C911C972F5F3F4F4F4F5F4FF8
:104410002E833F8348875987EA85FB8540805180FA
:1044200062807380411451046104710431F0089476
:10443000411C511C611C711C10C0DC014D905D9031
:104440006D907C90B1E0BD832C853D854E855F8568
:10445000213031054105510509F01D82530142010A
:10446000CC24DD247601F10181859285A385B48574
:10447000C816D906EA06FB0608F093C02E813F81D4
:1044800048855985281539054A055B0550F422E011
:10449000822E912CA12CB12C32E0432E512C612C78
:1044A000712CC101B501A4019E012F5F3F4F0E94F5
:1044B0005320882309F475C049815A816B817C811E
:1044C000D501C4010196A11DB11D4115510561051C
:1044D000710519F02C013D010DC084199509A6093B
:1044E000B7092C853D854E855F8582179307A40704
:1044F000B50759F00894C11CD11CE11CF11C0894AB
:10450000811C911CA11CB11CAECFC101A401B5013D
:104510000FEF1FEF2FEF3FE00E944421882391F41B
:1045200040C0680179010894C108D108E108F10888
:10453000C101B701A6010E944421882391F197018E
:10454000860102C095018401401651066206730679
:1045500040F3AA85BB854D915D916D917C91139738
:10456000411551056105710539F0C10193018201C1
:104570000E9444218823A9F0EA85FB85408251826C
:1045800062827382FD81FF2371F00894411C511CEB
:10459000611C711CD1014D925D926D927C921397BA
:1045A00002C080E001C081E02F960FB6F894DEBF14
:1045B0000FBECDBFDF91CF911F910F91FF90EF9074
:1045C000DF90CF90BF90AF909F908F907F906F9033
:1045D0005F904F903F902F900895AF92BF92CF92EF
:1045E000DF92EF92FF920F931F93CF93DF9300D050
:1045F0000F92CDB7DEB75C016A017B0182E090E0EB
:10460000A0E0B0E0F50180839183A283B383C5016C
:10461000B701A6019E012F5F3F4F0E9453208823C0
:1046200041F1C501B701A60100E010E020E030E053
:104630000E9444218823E9F0C980DA80EB80FC8065
:10464000F5018789803151F4F8EFCF16FFEFDF06CF
:10465000F0E0EF06F0E0FF0650F4D9CF88EFC8167F
:104660008FEFD8068FEFE8068FE0F80680F281E042
:1046700001C080E00F900F900F900F90DF91CF91CD
:104680001F910F91FF90EF90DF90CF90BF90AF9070
:1046900008956F927F928F929F92AF92BF92CF9226
:1046A000DF92EF92FF921F93CF93DF93EC01142FD1
:1046B0007093DD046093DC041F8A82E090E0A0E048
:1046C000B0E088839983AA83BB831092DB041092A5
:1046D000D7041092D8041092D9041092DA048FEF04
:1046E0009FEFAFEFBFEF8093DE069093DF06A093BE
:1046F000E006B093E106442389F1453008F008C193
:1047000060E070E080E090E040E00E9419208823A3
:1047100009F4FEC0E12FF0E0A4E0EE0FFF1FAA9520
:10472000E1F7E457F94F808190E08F779070009720
:1047300009F0EEC084859585A685B78584369105F8
:10474000A105B10508F4E4C080849184A284B384F7
:1047500081149104A104B10421F4DAC088249924BD
:104760005401C501B40140E00E941920882309F4D6
:10477000CFC08091E9049091EA0422E08030920752
:1047800009F0C6C03091EE04332309F4C1C0809112
:10479000EC049091ED04009709F4BAC02091EB0469
:1047A000222309F4B5C03A8B2C831D8630E041E00A
:1047B00050E006C0812F8F5F8D87183008F0A8C0A9
:1047C0001D85CA01012E02C0880F991F0A94E2F7C5
:1047D0002817390779F78091F4049091F504009730
:1047E00019F0A0E0B0E008C08091020590910305A7
:1047F000A0910405B09105058D839E83AF83B88792
:104800002091EC043091ED046901EE24FF24C80CE2
:10481000D91CEA1CFB1CCB8ADC8AED8AFE8A6090DC
:10482000EF047090F004798E688E2091EE0430E0F1
:1048300040E050E0BC01CD010E94C7A4DC01CB01E7
:104840008C0D9D1DAE1DBF1D8A8F9B8FAC8FBD8FA4
:10485000A301E5E0440F551FEA95E1F741505E4F93
:10486000452F5527469560E070E0480F591F6A1F95
:104870007B1F4E875F87688B798B8091F1049091C5
:10488000F204009719F0A0E0B0E008C08091FE04A7
:104890009091FF04A0910005B0910105841A950A3A
:1048A000A60AB70A880E991EAA1EBB1E04C0B6949B
:1048B000A794979487941A95D2F789869A86AB869F
:1048C000BC8685EF88168FE0980680E0A80680E019
:1048D000B80618F48CE08F8B1BC025EF82162FEFE3
:1048E000920620E0A20620E0B20610F480E10DC09E
:1048F00080910A0590910B05A0910C05B0910D05D2
:104900008A8F9B8FAC8FBD8F80E28F8B81E001C03F
:1049100080E0DF91CF911F91FF90EF90DF90CF90DB
:10492000BF90AF909F908F907F906F900895CF939E
:10493000DF930F92CDB7DEB769830496BE016F5F38
:104940007F4F41E050E00E94421E0F90DF91CF91D7
:104950000895DB010D900020E9F7AD014150504072
:10496000461B570B04960E94421E0895CF93DF9377
:10497000CAE6D9E0FE0107C09091C00095FFFCCFC8
:104980008093C600319684918823B1F7EEE9FAE06E
:1049900007C09091C00095FFFCCF8093C600319670
:1049A00084918823B1F78091C00085FFFCCF8AE015
:1049B0008093C600FE018491EAE6F9E008C0909178
:1049C000C00095FFFCCF8093C60031968491882368
:1049D000B1F7EEEAFAE007C09091C00095FFFCCF76
:1049E0008093C600319684918823B1F74091FF0FE0
:1049F0005091001060910110709102108BE59AE0C7
:104A000022E030E00E948F7AE6EBFAE007C0909156
:104A1000C00095FFFCCF8093C60031968491882317
:104A2000B1F74091031050910410609105107091FE
:104A300006108BE59AE022E030E00E948F7AE9EBE5
:104A4000FAE007C09091C00095FFFCCF8093C600AC
:104A5000319684918823B1F7409107105091081046
:104A60006091091070910A108BE59AE022E030E025
:104A70000E948F7AECEBFAE007C09091C00095FF9E
:104A8000FCCF8093C600319684918823B1F7409182
:104A90000B1050910C1060910D1070910E108BE561
:104AA0009AE022E030E00E948F7A8091C00085FF7A
:104AB000FCCF8AE08093C600FE018491EAE6F9E02B
:104AC00008C09091C00095FFFCCF8093C60031963E
:104AD00084918823B1F7EFEBFAE007C09091C00012
:104AE00095FFFCCF8093C600319684918823B1F75F
:104AF0008091C00085FFFCCF8AE08093C600FE0154
:104B00008491EAE6F9E008C09091C00095FFFCCFDF
:104B10008093C600319684918823B1F7E9EDFAE0DD
:104B200007C09091C00095FFFCCF8093C6003196DE
:104B300084918823B1F740910F105091101060912B
:104B40001110709112108BE59AE022E030E00E9483
:104B50008F7AE2EEFAE007C09091C00095FFFCCF9B
:104B60008093C600319684918823B1F74091131049
:104B70005091141060911510709116108BE59AE009
:104B800022E030E00E948F7AE5EEFAE007C09091D3
:104B9000C00095FFFCCF8093C60031968491882396
:104BA000B1F7409117105091181060911910709141
:104BB0001A108BE59AE022E030E00E948F7AE8EE4E
:104BC000FAE007C09091C00095FFFCCF8093C6002B
:104BD000319684918823B1F740911B1050911C109D
:104BE00060911D1070911E108BE59AE022E030E07C
:104BF0000E948F7A8091C00085FFFCCF8AE080936D
:104C0000C600FE018491EAE6F9E008C09091C00078
:104C100095FFFCCF8093C600319684918823B1F72D
:104C2000EBEEFAE007C09091C00095FFFCCF8093B7
:104C3000C600319684918823B1F78091C00085FF2A
:104C4000FCCF8AE08093C600FE018491EAE6F9E099
:104C500008C09091C00095FFFCCF8093C6003196AC
:104C600084918823B1F7E9E0FBE007C09091C00090
:104C700095FFFCCF8093C600319684918823B1F7CD
:104C80004091EF0F5091F00F6091F10F7091F20F82
:104C90008BE59AE02AE030E00E944979E2E1FBE00E
:104CA00007C09091C00095FFFCCF8093C60031965D
:104CB00084918823B1F74091F30F5091F40F6091E4
:104CC000F50F7091F60F8BE59AE02AE030E00E9434
:104CD0004979E5E1FBE007C09091C00095FFFCCF6A
:104CE0008093C600319684918823B1F74091F70FE5
:104CF0005091F80F6091F90F7091FA0F8BE59AE0DF
:104D00002AE030E00E944979E8E1FBE007C0909199
:104D1000C00095FFFCCF8093C60031968491882314
:104D2000B1F74091FB0F5091FC0F6091FD0F709116
:104D3000FE0F8BE59AE02AE030E00E9449798091ED
:104D4000C00085FFFCCF8AE08093C600FE018491FD
:104D5000EAE6F9E008C09091C00095FFFCCF80938F
:104D6000C600319684918823B1F7EBE1FBE007C0E0
:104D70009091C00095FFFCCF8093C600319684913E
:104D80008823B1F78091C00085FFFCCF8AE0809333
:104D9000C600FE018491EAE6F9E008C09091C000E7
:104DA00095FFFCCF8093C600319684918823B1F79C
:104DB000E0E5FBE007C09091C00095FFFCCF809339
:104DC000C600319684918823B1F74091E70F509146
:104DD000E80F6091E90F7091EA0F8BE59AE022E00D
:104DE00030E00E948F7AE9E5FBE007C09091C000B7
:104DF00095FFFCCF8093C600319684918823B1F74C
:104E00004091E30F5091E40F6091E50F7091E60F30
:104E10008BE59AE022E030E00E948F7A8091C0001A
:104E200085FFFCCF8AE08093C600FE018491EAE60C
:104E3000F9E008C09091C00095FFFCCF8093C600B8
:104E4000319684918823B1F7ECE5FBE007C090919F
:104E5000C00095FFFCCF8093C600319684918823D3
:104E6000B1F78091C00085FFFCCF8AE08093C60037
:104E7000FE018491EAE6F9E008C09091C00095FF38
:104E8000FCCF8093C600319684918823B1F7E5EF7B
:104E9000FBE007C09091C00095FFFCCF8093C60057
:104EA000319684918823B1F74091EB0F5091EC0F2C
:104EB0006091ED0F7091EE0F8BE59AE022E030E00B
:104EC0000E948F7AEEEFFBE007C09091C00095FF43
:104ED000FCCF8093C600319684918823B1F740912E
:104EE000D30F5091D40F6091D50F7091D60F8BE5F1
:104EF0009AE022E030E00E948F7AE1E0FCE007C017
:104F00009091C00095FFFCCF8093C60031968491AC
:104F10008823B1F740911F1050912010609121100B
:104F2000709122108BE59AE02AE030E00E944979E6
:104F3000E4E0FCE007C09091C00095FFFCCF8093B7
:104F4000C600319684918823B1F74091DF0F5091CC
:104F5000E00F6091E10F7091E20F8BE59AE022E0A3
:104F600030E00E948F7AE7E0FCE007C09091C0003B
:104F700095FFFCCF8093C600319684918823B1F7CA
:104F80004091DB0F5091DC0F6091DD0F7091DE0FCF
:104F90008BE59AE022E030E00E948F7AEAE0FCE0C4
:104FA00007C09091C00095FFFCCF8093C60031965A
:104FB00084918823B1F74091D70F5091D80F609119
:104FC000D90F7091DA0F8BE59AE022E030E00E9471
:104FD0008F7A8091C00085FFFCCF8AE08093C60065
:104FE000FE018491EAE6F9E008C09091C00095FFC7
:104FF000FCCF8093C600319684918823B1F7EDE011
:10500000FCE007C09091C00095FFFCCF8093C600E4
:10501000319684918823B1F78091C00085FFFCCF41
:105020008AE08093C600FE01C491EAE6F9E008C078
:105030008091C00085FFFCCFC093C6003196C4911B
:10504000CC23B1F7EBE1FCE007C09091C00095FFE5
:10505000FCCF8093C600319684918823B1F74091AC
:1050600036045091370460913804709139048BE50F
:105070009AE022E030E00E948F7AE5E2FCE007C08F
:105080009091C00095FFFCCF8093C600319684912B
:105090008823B1F760913204709133048091340415
:1050A000909135042FE632E143E05EE30E9433A1A4
:1050B000AB01BC018BE59AE022E030E00E948F7AE0
:1050C000E8E2FCE007C09091C00095FFFCCF809320
:1050D000C600319684918823B1F760912E047091B7
:1050E0002F0480913004909131042FE632E143E0A7
:1050F0005EE30E9401A4AB01BC018BE59AE022E0D3
:1051000030E00E948F7A8091C00085FFFCCF8AE05A
:105110008093C600DF91CF910895CF93DF930F92D4
:105120000F92CDB7DEB780915010909151109E0133
:105130002F5F3F4F009719F42655304102C0281BBE
:10514000390B3A83298389819A810F900F90DF91DF
:10515000CF910895BC018091060890910708843092
:1051600091050CF06EC0209108083091090840E6C6
:1051700050E0249FC001259F900D349F900D112475
:10518000865F974F0E9460A8EAE6F9E007C0909119
:10519000C00095FFFCCF8093C60031968491882390
:1051A000B1F7E0E7F9E007C09091C00095FFFCCFB0
:1051B0008093C600319684918823B1F72091080826
:1051C0003091090880E690E0289FF001299FF00DBA
:1051D000389FF00D1124E65FF74F06C09091C00094
:1051E00095FFFCCF8093C60081918823B9F7EBE748
:1051F000F9E007C09091C00095FFFCCF8093C600F6
:10520000319684918823B1F78091C00085FFFCCF4F
:105210008AE08093C6008091080890910908019661
:1052200064E070E00E94FAA4909309088093080853
:105230008091060890910708019690930708809343
:1052400006080895809A889A0895809A8898089503
:105250008091940990919509019660E070E00E9418
:105260004EA5462F572F682F792FCB01BA010895ED
:105270008091940990919509019660E070E04AE070
:1052800050E00E94CDA60895682FE0918E09F0911C
:105290008F0940E650E0E49F9001E59F300DF49FB8
:1052A000300D1124C901865F974F70E00E9455A808
:1052B0009C01909395098093940981E02115310513
:1052C00009F480E008950E941E9DDC01CB018093CB
:1052D000A6099093A709A093A809B093A909E09102
:1052E0008E09F0918F09E657F64F80818823A1F44B
:1052F000E2E2FFE007C09091C00095FFFCCF8093F1
:10530000C600319684918823B1F78091C00085FF53
:10531000FCCF8AE08093C60008958BE59AE00E9456
:10532000C278EAE1FFE007C09091C00095FFFCCF92
:105330008093C600319684918823B1F740919A09F1
:1053400050919B0960919C0970919D094F5F5F4F3F
:105350006F4F7F4F8BE59AE02AE030E00E945E7944
:105360008091C00085FFFCCF8AE08093C6000E9438
:10537000632908956F927F928F929F92AF92BF920E
:10538000CF92DF92EF92FF920F931F93CF9385E41A
:10539000682E84E0782E0BE017E09EEAC92E99E093
:1053A000D92E2EE1E22E27E0F22EC0E0F30181910A
:1053B0003F010E944429882309F10E9428294B01BA
:1053C0005C01F7018081882319F46091BE0901C056
:1053D00061E070E080E090E00E94CEA1F8012081C1
:1053E0003181428153810E9401A49B01AC01C5011E
:1053F000B4010E9453A0DC01CB0105C0F8018081FB
:105400009181A281B381F60180839183A283B383CA
:10541000CF5F0C5F1F4F84E090E0C80ED91E089448
:10542000E11CF11CC43011F686E40E944429882353
:10543000E1F00E9428296B017C016093C8097093F8
:10544000C9098093CA099093CB0920E030E040E07D
:1054500050E00E942FA3181644F4C0921C04D0926E
:105460001D04E0921E04F0921F04CF911F910F9132
:10547000FF90EF90DF90CF90BF90AF909F908F9074
:105480007F906F9008950E94BA2989E40E94442970
:10549000882329F00E942829DC01CB0104C080E088
:1054A00090E0A0E0B0E08093CC099093CD09A09368
:1054B000CE09B093CF098AE40E944429882329F0B9
:1054C0000E942829DC01CB0104C080E090E0A0E02C
:1054D000B0E08093D0099093D109A093D209B09302
:1054E000D30908958F929F92AF92BF92CF92DF928D
:1054F000EF92FF920F931F93CF93DF930E941E9D15
:10550000DC01CB018093A6099093A709A093A80979
:10551000B093A90960910A0470910B04CEEAD9E016
:1055200034E0C32ED12CCC0EDD1E48E0A42EB12CCD
:10553000AC0EBD1E5CE0852E912C8C0E9D1E882726
:1055400077FD8095982F0E94CEA120911C04309168
:105550001D0440911E0450911F040E9401A420E0EC
:1055600030E040E752E40E9433A120E030E048EC14
:1055700052E40E9433A17B018C01CE01B601A5014A
:105580009401EEEFCE2EE6E0DE2E0E946D8D80912E
:10559000AE099091AF09A091B009B091B109809383
:1055A0000B0790930C07A0930D07B0930E07809103
:1055B000B2099091B309A091B409B091B509809353
:1055C0000F0790931007A0931107B09312078091D3
:1055D000B6099091B709A091B809B091B909809323
:1055E000130790931407A0931507B09316078091A3
:1055F000BA099091BB09A091BC09B091BD098093F3
:10560000170790931807A0931907B0931A07DF9113
:10561000CF911F910F91FF90EF90DF90CF90BF90AF
:10562000AF909F908F9008954F925F926F927F926C
:10563000AF92BF92CF92DF92EF920F931F93CF93CF
:10564000C82F6091CC097091CD098091CE099091BD
:10565000CF092091D0093091D1094091D2095091C0
:10566000D3090E943CA32B013C0160910A04709174
:105670000B0400D000D00DB71EB70F5F1F4F882757
:1056800077FD8095982F0E94CEA120911C04309127
:105690001D0440911E0450911F040E9401A420E0AB
:1056A00030E040E752E40E9433A120E030E048ECD3
:1056B00052E40E9433A15B016C01F80140825182E7
:1056C00062827382C4838091FE0685838BE097E0BB
:1056D0006EEA79E04CEC59E020E001E0A2E0EA2E2D
:1056E0000E947E848091AE099091AF09A091B0098B
:1056F000B091B10980930B0790930C07A0930D070D
:10570000B0930E078091B2099091B309A091B409AA
:10571000B091B50980930F0790931007A0931107DC
:10572000B09312078091B6099091B709A091B8097A
:10573000B091B9098093130790931407A0931507AC
:10574000B09316078091BA099091BB09A091BC094A
:10575000B091BD098093170790931807A09319077C
:10576000B0931A078DB79EB706960FB6F8949EBFF2
:105770000FBE8DBF0E941E9DDC01CB018093A60948
:105780009093A709A093A809B093A909CF911F915D
:105790000F91EF90DF90CF90BF90AF907F906F9080
:1057A0005F904F9008958091FC060895CF93DF930A
:1057B000EC0105C082EE96E00E94359E2196FE0126
:1057C00064916623B9F7DF91CF9108950F931F93EA
:1057D000CF93DF938C01C8EDD9E0CE01B80144E14D
:1057E00050E00E9475A8F80101900020E9F7319778
:1057F000E01BF10BEC0FFD1F1082DF91CF911F9189
:105800000F910895FC01349120E0A8EDB9E08A1BC6
:105810009B0B332349F0243139F03D932F5FFD0179
:10582000E80FF91F3491F5CF1C9208950E94717012
:105830008091FC068823C1F581E08093FC0680916D
:105840009A0990919B09A0919C09B0919D09809320
:10585000C4099093C509A093C609B093C709E0E4B1
:10586000FCE007C09091C00095FFFCCF8093C6007C
:10587000319684918823B1F7EFE4FFE007C090915F
:10588000C00095FFFCCF8093C60031968491882399
:10589000B1F78091C00085FFFCCF8AE08093C600FD
:1058A00087EC9FE00E94022C0895F8940E9471708A
:1058B000159A179A429AA09A8CE060E00E947C9C0C
:1058C000E0E4FCE007C09091C00095FFFCCF80931E
:1058D000C600319684918823B1F7E5E2FFE007C066
:1058E0009091C00095FFFCCF8093C60031968491C3
:1058F0008823B1F78091C00085FFFCCF8AE08093B8
:10590000C60086E49FE00E94022C0E942529FFCF5A
:105910000F931F930E941E9DDC01CB014091C00993
:105920005091C1096091C2097091C3090091A60903
:105930001091A7092091A8093091A909801B910B0A
:10594000A20BB30B481759076A077B0738F44115B8
:1059500051056105710511F00E94552C80912104BB
:1059600090912204A0912304B09124040097A105F2
:10597000B10539F10E941E9DDC01CB014091A609C1
:105980005091A7096091A8097091A909841B950BF2
:10599000A60BB70B4091210450912204609123047F
:1059A00070912404481759076A077B0750F49091B7
:1059B000E20A8091E10A981721F4159A179A429AFF
:1059C000A09A0E94168D1F910F9108952F923F92D9
:1059D0004F925F926F927F928F929F92AF92BF92FF
:1059E000CF92DF92EF92FF920F931F93CF93DF93AB
:1059F000CDB7DEB76E970FB6F894DEBF0FBECDBF42
:105A000030E6632E712CECEEFCE034904AE0542E2C
:105A1000E9EEFCE044901CC28D3051F08A3321F451
:105A200090919109992321F04F3551050CF4F1C162
:105A30004115510509F4F5C28091080890910908B3
:105A4000869D7001879DF00C969DF00C11244E0DE3
:105A50005F1D465F574FFA01108220919109222362
:105A600009F0D2C1109291098657964FFC0110821D
:105A70008701065F174FC8016EE470E00E9455A8C9
:105A8000009709F410C19093950980939409801BA5
:105A9000910B8E0D9F1D855F974F60E070E04AE08F
:105AA00050E00E94CDA6DC01CB0180939609909333
:105AB0009709A0939809B093990980909A099090BA
:105AC0009B09A0909C09B0909D09B501A4014F5F6E
:105AD0005F4F6F4F7F4F84179507A607B70709F4ED
:105AE0003AC02091080830910908269DC001279DE1
:105AF000900D369D900D1124865F974F64E172E002
:105B00000E9484A8009739F5E0E4FCE007C090917A
:105B1000C00095FFFCCF8093C60031968491882306
:105B2000B1F7E7E4FCE007C09091C00095FFFCCF1F
:105B30008093C600319684918823B1F78BE59AE073
:105B4000B501A4012AE030E00E945E798091C00096
:105B500085FFFCCF91C08091080890910908869D2F
:105B60007001879DF00C969DF00C11242AE0C22E46
:105B700028E0D22ECE0CDF1CC6016AE270E00E9443
:105B800055A8009721F452C003272F5F02C020E0E0
:105B900000E0F701E20FF11DE65FF74F30813A3286
:105BA00099F790939509809394098C199D098E0D0E
:105BB0009F1D855F974F60E070E00E944EA50E9498
:105BC0009BA1AB01BC01802F90E08417950709F4DD
:105BD00059C0E0E4FCE007C09091C00095FFFCCF05
:105BE0008093C600319684918823B1F7E9E7FCE001
:105BF00007C09091C00095FFFCCF8093C6003196FE
:105C000084918823B1F740919A0950919B09609142
:105C10009C0970919D098BE59AE02AE030E00E9492
:105C20005E798091C00085FFFCCF26C0E0E4FCE0F7
:105C300007C09091C00095FFFCCF8093C6003196BD
:105C400084918823B1F7E7E9FCE007C09091C00098
:105C500095FFFCCF8093C600319684918823B1F7DD
:105C60008BE59AE0B501A4012AE030E00E945E795C
:105C70008091C00085FFFCCF8AE08093C6000E941F
:105C80008D2947C08091960990919709A091980914
:105C9000B091990980939A0990939B09A0939C09CC
:105CA000B0939D093BC0C8016AE270E00E9455A80C
:105CB0000097A1F1E0E4FCE007C09091C00095FFDF
:105CC000FCCF8093C600319684918823B1F7E0EC35
:105CD000FCE007C09091C00095FFFCCF8093C60008
:105CE000319684918823B1F740919A0950919B098C
:105CF00060919C0970919D098BE59AE02AE030E063
:105D00000E945E798091C00085FFFCCF8AE080937D
:105D1000C600109293091092920924C2809108083B
:105D200090910908869D7001879DF00C969DF00C5E
:105D300011248701065F174FC80167E470E00E94D5
:105D400055A8009709F44AC0909395098093940947
:105D5000801B910B8E0D9F1D855F974F60E070E05B
:105D60000E944EA50E949BA1DC01CB0184309105CD
:105D7000A8F58091FC068823C9F480912207882326
:105D800069F5842DE9EEFCE008C09091C00095FF14
:105D9000FCCF8093C600319684918823B1F780911F
:105DA000C00085FFFCCF5092C60018C0832DECEEDA
:105DB000FCE008C09091C00095FFFCCF8093C60026
:105DC000319684918823B1F78091C00085FFFCCF84
:105DD0005092C60084E69DE00E94022C8091080843
:105DE00090910908019664E070E00E94FAA49093F3
:105DF0000908809308088091060890910708019689
:105E000090930708809306081092930910929209C4
:105E10001FC08B3319F491E09093910990919109EF
:105E20009923B1F42091080830910908269DF001CA
:105E3000279DF00D369DF00D1124E40FF51FE65F50
:105E4000F74F80834F5F5F4F5093930940939209C0
:105E50008091DC0A9091DD0A2091DE0A3091DF0A00
:105E6000821B930B8F779070009709F476C1809115
:105E7000060890910708843091050CF06EC18BE5FF
:105E80009AE00E94A67880939009409192095091DF
:105E900093098A3009F0C0CDCBCD809192099091C1
:105EA0009309009709F40DC15DC14D3091F04A335B
:105EB00021F420919109222361F0209192093091DF
:105EC00093092F3531052CF4FFEF8F3F9F0709F021
:105ED000D9C08091FC079091FD07A091FE07B09179
:105EE000FF074091F4075091F5076091F607709114
:105EF000F70784179507A607B70708F48CC0862D07
:105F0000EEE6FDE008C09091C00095FFFCCF8093C5
:105F1000C600319684918823B1F78091C00085FF37
:105F2000FCCFE092C6000E941E9DDC01CB01809355
:105F30009E0990939F09A093A009B093A109409155
:105F4000A2095091A3096091A4097091A509841B2D
:105F5000950BA60BB70BBC01CD0128EE33E040E05A
:105F600050E00E940DA58DB79EB708970FB6F89424
:105F70009EBF0FBE8DBF0DB71EB70F5F1F4FEDB792
:105F8000FEB792828182F80133822282CA01B9016E
:105F90002CE330E040E050E00E940DA5DC01CB0195
:105FA000F80135832483978386830E949EA8852DDC
:105FB0002DB73EB7285F3F4F0FB6F8943EBF0FBED8
:105FC0002DBFEAE6F9E008C09091C00095FFFCCF34
:105FD0008093C600319684918823B1F7F40106C0FE
:105FE0009091C00095FFFCCF8093C60081918823DB
:105FF000B9F78091C00085FFFCCFE092C600C401D4
:106000000E94E62B82E297E00E946F8482E297E092
:1060100061E00E94D3818091920990919309009749
:1060200019F4109291099EC0209108083091090836
:106030002A9DF0012B9DF00D3A9DF00D1124E80FE3
:10604000F91FE65FF74F1082F901E657F64FC0825D
:106050008091060890910708019690930708809315
:106060000608C901019664E070E00E94FAA49093CA
:1060700009088093080810929109109293091092D0
:10608000920934C04B3311F4C09291098091910967
:10609000882361F580910808909109088A9DF00194
:1060A0008B9DF00D9A9DF00D1124E20FF31FE65F1A
:1060B000F74F40832F5F3F4F30939309209392090E
:1060C00015C0B0E6AB2EB12CCC24C394EEE6FDE0B7
:1060D00064901AE0E12E4E010894811C911C09E1A4
:1060E000202E02E0302EEAE6F9E054908091FC0781
:1060F0009091FD07A091FE07B091FF074091F40732
:106100005091F5076091F6077091F707841795078E
:10611000A607B70738F580910608909107088430E4
:10612000910504F58091E1079091E207A091E307C2
:10613000B091E4078093FC079093FD07A093FE07BE
:10614000B093FF0789ED97E00E94AD19482F809327
:1061500090098A3009F0A9CEBCCE8091230788230C
:1061600009F09BCE6E960FB6F894DEBF0FBECDBF82
:10617000DF91CF911F910F91FF90EF90DF90CF9023
:10618000BF90AF909F908F907F906F905F904F9057
:106190003F902F900895CF93DF93CDB7DEB7A897A8
:1061A0000FB6F894DEBF0FBECDBFDE019196E8E2D8
:1061B000F2E088E001900D928150E1F7DE015996FE
:1061C000E0E3F2E088E001900D928150E1F7DE011A
:1061D0005196E8E3F2E088E001900D928150E1F7FA
:1061E000DE011996E0E4F2E088E001900D92815022
:1061F000E1F7DE011196E8E4F2E088E001900D920B
:106200008150E1F782EE96E064E144E020E00E94F4
:10621000699F82EE96E061E0AE014F5D5F4F0E94A4
:10622000F19E82EE96E062E0AE01475E5F4F0E9413
:10623000F19E82EE96E063E0AE014F5E5F4F0E94FA
:10624000F19E82EE96E064E0AE01475F5F4F0E94F0
:10625000F19E82EE96E065E0AE014F5F5F4F0E94D7
:10626000F19E81ED9FE00E94022CA8960FB6F89453
:10627000DEBF0FBECDBFDF91CF910895CF9382E1F6
:1062800061E00E947C9CC4E15B9A65E070E080E084
:1062900090E00E945A9D5B9865E070E080E090E09D
:1062A0000E945A9DC15081F7CF910895CF9382E10A
:1062B00061E00E947C9CCAE05B9A63E070E080E051
:1062C00090E00E945A9D5B9863E070E080E090E06F
:1062D0000E945A9DC15081F7CF91089588E260E0F5
:1062E0000E947C9C8AE260E00E947C9C83E160E0EA
:1062F0000E947C9C86E260E00E947C9CA19A9FB7F1
:10630000F894EBE0F1E08081806880839FBF5A9A27
:106310005F9A0895CF92DF92EF92FF92CF93C1E000
:106320009199C0E08091090187FFC260C090EC099B
:10633000D090ED09E090EE09F090EF090E941E9DCB
:10634000DC01CB01C816D906EA06FB0610F44A9B0D
:10635000C460C093FB064091FB0641708091FB0630
:1063600081FD4260842F90E02091F7063091F8067D
:106370008217930791F1423059F0433081F0413058
:10638000A9F021303105A9F02230310531F51BC0CB
:106390002115310571F023303105F9F414C0223094
:1063A000310539F021303105C1F40DC023303105FC
:1063B00039F42091F9063091FA062F5F3F4F09C05A
:1063C0002115310551F42091F9063091FA0621503A
:1063D00030403093FA062093F9069093F8068093A4
:1063E000F706CF91FF90EF90DF90CF900895CF9375
:1063F000DF93EC0119821A82188281E08B830E945C
:106400006E310E94CB3018861986DF91CF910895A6
:10641000CF92DF92EF92FF920F931F93CF93DF9370
:106420008C01FC0197818681981719F48381882358
:1064300039F081E0F801838382EE96E00E94619F4B
:10644000F801D681EE24FF24CD2EDD24C7FCD094A4
:1064500031C2443009F4EAC045307CF4413009F4DB
:1064600048C042301CF44423A9F021C2423009F450
:106470007BC0433009F01BC2A7C0463009F44BC1B2
:1064800046300CF403C1473009F495C1483009F097
:106490000EC2DCC1F8018381882351F082EE96E0C0
:1064A00060E04E2D0E94339F8AEF9FE00E94D62B22
:1064B000F8012081332727FD30958C2F90E0281795
:1064C000390709F0F4C18091FB0682FFF0C10E94F8
:1064D0001E9DDC01CB018C509E4FAF4FBF4F809370
:1064E000EC099093ED09A093EE09B093EF0981E0D8
:1064F000DAC1F8018381882351F082EE96E060E0F2
:106500004E2D0E94339F82E090E10E94D62BF8012D
:106510002081332727FD30958C2F90E028173907ED
:1065200009F0C5C18091FB0682FFC1C10E941E9D7A
:10653000DC01CB018C509E4FAF4FBF4F8093EC09D5
:106540009093ED09A093EE09B093EF0910923307F1
:106550001092320782E297E00E94AC7D82E297E0DF
:1065600061E00E94D381A1C1F8018381882351F0A9
:1065700082EE96E060E04E2D0E94339F8DE090E128
:106580000E94D62BF8012081332727FD30958C2FD0
:1065900090E02817390709F08AC18091FB0682FF35
:1065A00086C10E941E9DDC01CB018C509E4FAF4FD7
:1065B000BF4F8093EC099093ED09A093EE09B0933F
:1065C000EF0980E592E02FC0F8018381882351F024
:1065D00082EE96E060E04E2D0E94339F8FE190E1C5
:1065E0000E94D62BF8012081332727FD30958C2F70
:1065F00090E02817390709F05AC18091FB0682FF05
:1066000056C10E941E9DDC01CB018C509E4FAF4FA6
:10661000BF4F8093EC099093ED09A093EE09B093DE
:10662000EF0984E592E00E94AA283FC1F801838126
:10663000882351F082EE96E060E04E2D0E94339F59
:106640008AE290E10E94D62BF8012081332727FDB2
:1066500030958C2F90E02817390709F028C18091D8
:10666000FB0682FF24C10E941E9DDC01CB018C50E1
:106670009E4FAF4FBF4F8093EC099093ED09A093CD
:10668000EE09B093EF0988E592E0CDCFF801838160
:10669000882351F082EE96E060E04E2D0E94339FF9
:1066A00086E390E10E94D62BF8012081332727FD55
:1066B00030958C2F90E02817390709F0F8C08091A9
:1066C000FB0682FFF4C00E941E9DDC01CB018C50B2
:1066D0009E4FAF4FBF4F8093EC099093ED09A0936D
:1066E000EE09B093EF0984EB90E060E00E94536DF7
:1066F00090931F0A80931E0A80E090E0A4E3B3E425
:106700008093140A9093150AA093160AB093170A5F
:1067100086E490E044C0F8018381882351F082EE42
:1067200096E060E04E2D0E94339F83E490E10E944A
:10673000D62BF8012081332727FD30958C2F90E050
:106740002817390709F0B3C08091FB0682FFAFC05C
:106750000E941E9DDC01CB018C509E4FAF4FBF4F5E
:106760008093EC099093ED09A093EE09B093EF09A3
:1067700080EF90E060E00E94536D90931F0A809339
:106780001E0A80E090E0A0E7B3E48093140A90939F
:10679000150AA093160AB093170A84E690E00E94A7
:1067A0009B6D90931D0A80931C0A87E06FEF70E049
:1067B0000E942C9B7AC0F8018381882351F082EEDD
:1067C00096E060E04E2D0E94339F80E590E10E94AC
:1067D000D62BF8012081332727FD30958C2F90E0B0
:1067E0002817390709F063C08091FB0682FF5FC05C
:1067F0000E941E9DDC01CB018C509E4FAF4FBF4FBE
:106800008093EC099093ED09A093EE09B093EF0902
:1068100080E090E060E00E94536D90931F0A8093A7
:106820001E0A80E090E0A0E0B0E08093140A90930C
:10683000150AA093160AB093170A80E090E00E9410
:106840009B6D90931D0A80931C0A2FC0F8018381D1
:10685000882351F082EE96E060E04E2D0E94339F37
:106860008AE590E10E94D62BF8012081332727FD8D
:1068700030958C2F90E028173907C9F48091FB06DA
:1068800082FF15C00E941E9DDC01CB018C509E4FE3
:10689000AF4FBF4F8093EC099093ED09A093EE09A1
:1068A000B093EF0983E0F80181830E945631089488
:1068B000E11CF11CCE2D4E2D4D0FF8015681852F78
:1068C000992787FD9095039697012C0D3D1D821702
:1068D00093070CF0BECD8085882309F06FC05783E5
:1068E000C091F906D091FA061382848195819E01A8
:1068F000281B390BC90104968930910508F05EC048
:1069000082EE96E060E040810E94339F82EE96E046
:1069100060E20E94359EF8018681D7FF06C0815053
:10692000868387FF48C0168246C0C531D1054CF02A
:106930008F5FF8018683863014F085E08683CFE090
:10694000D0E0D093FA06C093F906F801D583C4834A
:10695000CE0165E070E00E94FAA46083643011F417
:1069600083E08083F8018081893014F088E080839F
:10697000F80197818681981711F081E0838382EE78
:1069800096E060E0F80140810E94339FF801808129
:10699000992787FD90952681332727FD3095820F13
:1069A000931F009711F06EE301C063E082EE96E062
:1069B0000E94359E03C0C4E0D0E0C3CFDF91CF91E9
:1069C0001F910F91FF90EF90DF90CF9008952F923D
:1069D0003F924F925F926F927F928F929F92AF926F
:1069E000BF92CF92DF92EF92FF920F931F93CF93BC
:1069F000DF93CDB7DEB7A2970FB6F894DEBF0FBE18
:106A0000CDBF7C01DC0117969C91179716968C914F
:106A10001697981729F413968C911397882339F0B9
:106A200081E0F701838382EE96E00E94619FD701A7
:106A300013968C911397882379F0809124078823EB
:106A400039F082E297E00E9447838093050A04C0F0
:106A50001092050AF7011682D7011696BC90169778
:106A600088249924AA242B2D332727FD309538A379
:106A70002F8F215030403AA329A365E2662E67E0AC
:106A8000762E362C272C2E010894411C511C5BC1FC
:106A9000BB2029F031E0B31609F090C036C0D70111
:106AA00013968C911397882351F082EE96E060E064
:106AB000482D0E94339F88E092E10E94D62BF70177
:106AC0002081332727FD3095802F90E02817390744
:106AD00009F035C18091FB0682FF31C10E941E9DE5
:106AE000DC01CB018C509E4FAF4FBF4F8093EC0920
:106AF0009093ED09A093EE09B093EF0981E0D701DF
:106B000011968C930E9456311AC1F7018381882314
:106B100069F182EE96E060E0482D0E94339F82EE9C
:106B200096E065E672E00E94249E89E597E065E2C2
:106B300077E00E94C817809125078F3229F480E101
:106B400092E10E94D62B12C082EE96E067E672E0D8
:106B50000E94249E82EE96E065E277E00E94249EE9
:106B600082EE96E069E672E00E94249ED7012C91A5
:106B7000332727FD3095802F90E02817390709F03B
:106B8000DEC08091FB0682FFDAC00E941E9DDC0100
:106B9000CB018C509E4FAF4FBF4F8093EC09909329
:106BA000ED09A093EE09B093EF0982E297E00E940D
:106BB0004084F70116820E9456317EC029A13AA175
:106BC000280D391D8091050A90E0821793070CF477
:106BD000B6C0D70113968C911397882301F16B2DC2
:106BE000625082E297E00E94FD8282EE96E060E0D1
:106BF000482D0E94339F89E192E10E94D62B80911B
:106C00003107882331F082EE96E067E672E00E9459
:106C1000249E82EE96E065E277E00E94249EF701D2
:106C20002081332727FD3095802F90E028173907E2
:106C300009F085C08091FB0682FF81C00E941E9DE5
:106C4000DC01CB018C509E4FAF4FBF4F8093EC09BE
:106C50009093ED09A093EE09B093EF096B2D62506C
:106C600082E297E00E94FD828091310705E217E001
:106C7000CC24DD24882349F42AC0D8018C9190E0EB
:106C80000E9414A8F80181938F01C601F3010190BD
:106C90000020E9F7E652F7400894C11CD11C8E177A
:106CA0009F0758F382E297E065E277E00E949683BF
:106CB000D70116961C921697AA24A39440C0F801F7
:106CC000808190E00E9414A8D8018D938D01C601A7
:106CD000F30101900020E9F7E652F7400894C11C47
:106CE000D11C8E179F0758F300D000D0EDB7FEB728
:106CF0003196ADB7BEB712965C924E9211972DE6C3
:106D000032E033832283348225820E949EA88DB78D
:106D10009EB706960FB6F8949EBF0FBE8DBFC201F8
:106D20000E94AA2884E792E00E94AA280E943E318D
:106D3000D70111961C9285E297E00E94E62BB3944E
:106D40000894811C911C082DF7014681842F9927F6
:106D500087FD909503962F8D38A1280D391D821738
:106D600093070CF095CEC090050A8085882309F022
:106D70008FC047830091F9061091FA06138284812F
:106D800095819801281B390BC9010496893091051A
:106D900008F07EC0DC2CD39482EE96E060E0408167
:106DA0000E94339F82EE96E060E20E94359ED701FA
:106DB00016968C91169717FF0AC0815016968C93E1
:106DC000169787FF6DC016961C92169769C00531FD
:106DD0001105ECF08F5FF70186832D2D30E0A901BE
:106DE00042505040992787FD9095841795071CF0D5
:106DF0008C2D825086838901000F111F000F111FF7
:106E0000020F131F0F30110514F00FE010E0109364
:106E1000FA060093F906D70115961C930E93149762
:106E2000C80165E070E00E94FAA4F7016083643055
:106E300011F483E08083D7012C91332727FD30950F
:106E40008D2D90E0821793070CF4DC92F701978167
:106E50008681981711F081E0838382EE96E060E0EE
:106E6000D7014C910E94339FF7018081992787FDBC
:106E700090952681332727FD3095820F931F009729
:106E800011F06EE301C063E082EE96E00E94359E51
:106E9000AA2049F081E0D70113968C93139703C081
:106EA00004E010E0B4CFA2960FB6F894DEBF0FBE98
:106EB000CDBFDF91CF911F910F91FF90EF90DF90A9
:106EC000CF90BF90AF909F908F907F906F905F908A
:106ED0004F903F902F900895FF920F931F93CF9361
:106EE000DF93EC018985882361F00E949A998823B9
:106EF00099F480912307882379F481E08B831986A4
:106F00000BC00E949A99882321F48091230788233B
:106F100019F081E08B8389879F818E81981719F4FE
:106F20008B81882331F081E08B8382EE96E00E9492
:106F3000619F00E074E0F72E15E08B81023009F4C8
:106F400058C0033009F47BC0013031F1882351F07F
:106F500082EE96E060E040E00E94339F8BE192E198
:106F60000E94D62B8881882309F0A1C08091FB065E
:106F700082FF9DC00E941E9DDC01CB018C509E4F64
:106F8000AF4FBF4F8093EC099093ED09A093EE09AA
:106F9000B093EF09198289C0882381F082EE96E0D0
:106FA00060E041E00E94339F8985882319F486E2DE
:106FB00092E102C081E392E10E94D62B8881813068
:106FC00009F075C08091FB0682FF71C00E941E9D72
:106FD000DC01CB018C509E4FAF4FBF4F8093EC092B
:106FE0009093ED09A093EE09B093EF0982E08983B5
:106FF0005CC0882351F082EE96E060E042E00E949F
:10700000339F8CE392E10E94D62B8881823009F075
:107010004EC08091FB0682FF4AC00E941E9DDC018B
:10702000CB018C509E4FAF4FBF4F8093EC09909394
:10703000ED09A093EE09B093EF09F98236C08823D9
:10704000B1F082EE96E060E043E00E94339F4F99FA
:107050000AC080912307882319F087E492E105C0D4
:1070600087E592E102C087E692E10E94D62B4F9914
:107070001EC088818330D9F48091FB0682FF17C03F
:1070800082E297E00E946F840E941E9DDC01CB018A
:107090008C509E4FAF4FBF4F8093EC099093ED09FA
:1070A000A093EE09B093EF0919830E9456310F5F48
:1070B000043009F042CF8885882309F068C08E81AA
:1070C0008F830091F9061091FA061B828C819D81B5
:1070D0009801281B390BC90104968930910508F0E5
:1070E00056C082EE96E060E048810E94339F82EEB7
:1070F00096E060E20E94359E8E8117FF06C08150A7
:107100008E8387FF41C01E823FC0053111053CF0D0
:107110008F5F8E8318160CF41E820FE010E0109320
:10712000FA060093F9061D830C83C80165E070E040
:107130000E94FAA46883643011F483E08883888114
:10714000843014F083E088839F818E81981711F03A
:1071500081E08B8382EE96E060E048810E94339F5D
:107160008881992787FD90952E81332727FD3095BB
:10717000820F931F009711F06EE301C063E082EE6F
:1071800096E00E94359E03C004E010E0C8CFDF9176
:10719000CF911F910F91FF900895FC016081718143
:1071A000828193810E949BA1DC01CB01FC0164E6FA
:1071B00070E00E94FAA4CB012AE030E0B9010E94FD
:1071C000FAA4805D80930B0ACF01B9010E94FAA452
:1071D000482FCB01B9010E94FAA4805D80930C0A6C
:1071E000405D40930D0A10920E0A8BE09AE00895DC
:1071F000FC0180812AE030E090E0B9010E94FAA40D
:10720000482FCB01B9010E94FAA4805D80930B0A3C
:10721000405D40930C0A10920D0A8BE09AE00895AD
:10722000FC018081918164E670E00E94FAA4CB01A8
:107230002AE030E0B9010E94FAA4805D80930B0A35
:1072400080819181B9010E94FAA4CB01B9010E9409
:10725000FAA4805D80930C0A80819181B9010E941B
:10726000FAA4805D80930D0A10920E0A8BE09AE0DA
:107270000895FC018081918168EE73E00E94FAA478
:10728000CB012AE030E0B9010E94FAA4805D80932E
:107290000B0A8081918164E670E00E94FAA4CB0120
:1072A000B9010E94FAA4805D80930C0A80819181CB
:1072B000B9010E94FAA4CB01B9010E94FAA4805D31
:1072C00080930D0A80819181B9010E94FAA4805DAA
:1072D00080930E0A10920F0A8BE09AE008952F9285
:1072E0003F924F925F926F927F928F929F92AF9256
:1072F000BF92CF92DF92EF92FF920F931F93CF93A3
:10730000DF93CDB7DEB764970FB6F894DEBF0FBE3C
:10731000CDBF5C01FC0197818681981719F48381A8
:10732000882339F081E0F501838382EE96E00E94A4
:10733000619FF501868022243324282D332727FDE1
:1073400030953C8B2B8B71C3423009F497C243308C
:1073500034F4442371F0413009F064C33DC044303B
:1073600009F443C144300CF4CBC0453009F05AC392
:10737000F2C1F5018381882351F082EE96E060E04E
:10738000422D0E94339F8CE890E10E94D62BF5019C
:107390002081332727FD3095892D90E02817390764
:1073A00009F040C38091FB0682FF3CC30E941E9DF2
:1073B000DC01CB018C509E4FAF4FBF4F8093EC0947
:1073C0009093ED09A093EE09B093EF0981E0F501E8
:1073D00081830E94563126C3F5018381882349F1B8
:1073E00082EE96E060E0422D0E94339F84E990E1B6
:1073F0000E94D62B82EE96E06DE0422D0E94339FD4
:1074000060910A0470910B04882777FD8095982F6E
:107410000E94CEA1DC01CB018F87988BA98BBA8B00
:10742000CE010F960E94CD38BC0182EE96E00E94FC
:10743000249EF5012081332727FD3095892D90E08A
:107440002817390709F0EEC28091FB0682FF2CC095
:10745000808591E089278087882349F080910A04FC
:1074600090910B049093FA068093F9060DC0C90120
:10747000880F991F880F991F820F931F9093FA0608
:107480008093F9060E9456310E941E9DDC01CB01BB
:107490008C509E4FAF4FBF4F8093EC099093ED09F6
:1074A000A093EE09B093EF09F5018085882309F4D4
:1074B000B9C28091F9069091FA061816190634F0AF
:1074C00081E090E09093FA068093F9068091F906A6
:1074D0009091FA06F1E081399F0734F080E991E05C
:1074E0009093FA068093F9068091F9069091FA0636
:1074F00090930B0480930A0481E080931B07B3C12F
:10750000F50183818823A1F182EE96E060E0422DAF
:107510000E94339F8CE990E10E94D62B82EE96E088
:107520006DE0422D0E94339F80911E0A90911F0AA8
:1075300060E00E949E6D20E030E040E05FE30E944A
:1075400053A00E949BA1882777FD8095982F0E94C9
:10755000CEA1DC01CB018B879C87AD87BE87CE0196
:107560000B960E94CD38BC0182EE96E00E94249ECC
:10757000F5018081992787FD9095292D30E08217AC
:10758000930709F04FC28091FB0682FFC5C080853A
:1075900091E089278087882341F080911E0A90918D
:1075A0001F0A60E00E949E6D72C06091F9067091A2
:1075B000FA06882777FD8095982F0E94CEA16B014F
:1075C0007C010E949BA1DC01CB0160E00E94536D15
:1075D00090931F0A80931E0AC092140AD092150A33
:1075E000E092160AF092170A75C0F501838188238C
:1075F00099F182EE96E060E0422D0E94339F86EA88
:1076000090E10E94D62B82EE96E06DE0422D0E9422
:10761000339F80911C0A90911D0A0E940E7020E0F9
:1076200030E040E05FE30E9453A00E949BA18827C6
:1076300077FD8095982F0E94CEA1DC01CB018F832E
:107640009887A987BA87CE0107960E94CD38BC01DA
:1076500082EE96E00E94249EF5018081992787FDA5
:107660009095292D30E08217930709F0DBC18091B6
:10767000FB0682FF51C0808591E08927808788239F
:10768000A9F080911C0A90911D0A0E940E7020E0C2
:1076900030E040E05FE30E9453A00E949BA1DC0128
:1076A000CB019093FA068093F90626C06091F90603
:1076B0007091FA06882777FD8095982F0E94CEA1B9
:1076C0000E949BA1DC01CB010E949B6D90931D0A3F
:1076D00080931C0AF5012081332727FD3095C901CD
:1076E000880F991F880F991F820F931F9093FA0696
:1076F0008093F9060E9456310E941E9DDC01CB0149
:107700008C509E4FAF4FBF4F8093EC099093ED0983
:10771000A093EE09B093EF09F5018085882309F461
:1077200081C18091F9069091FA0697FF04C01092EA
:10773000FA061092F9068091F9069091FA06F1E0A6
:1077400085309F070CF48FC084E091E09093FA0697
:107750008093F90688C0F5018381882331F182EE98
:1077600096E060E0422D0E94339F8DEA90E10E94F6
:10777000D62B82EE96E06DE0422D0E94339F609101
:10778000FD0670E080E090E00E94CCA1DC01CB011E
:107790008B839C83AD83BE83CE0103960E94CD383C
:1077A000BC0182EE96E00E94249EF50120813327E1
:1077B00027FD3095892D90E02817390709F032C14F
:1077C0008091FB0682FF2AC0808591E0892780870F
:1077D000882339F08091FD068093F9061092FA060D
:1077E0000DC0C901880F991F880F991F820F931F21
:1077F0009093FA068093F9060E9456310E941E9DCE
:10780000DC01CB018C509E4FAF4FBF4F8093EC09F2
:107810009093ED09A093EE09B093EF09F5018085EF
:10782000882309F4FFC08091F9069091FA0697FF2A
:1078300004C01092FA061092F9068091F906909110
:10784000FA068F3F910539F034F08FEF90E0909376
:10785000FA068093F9066091F9066093FD0687E0C9
:1078600070E00E942C9B82EE96E06DE0492D0E9414
:10787000339F89EF96E00E941039CFC0F5018381D4
:10788000882339F182EE96E060E0422D0E94339F1A
:1078900089EB90E10E94D62B82EE96E06DE0422DBE
:1078A0000E94339F60910B1070910C1080910D100D
:1078B00090910E100E949BA1DC01CB019A838983D9
:1078C000CE0101960E943939BC0182EE96E00E94F9
:1078D000249EF5010081112707FD1095892D90E068
:1078E0000817190709F09EC08091FB0682FF6CC043
:1078F000808591E089278087882369F060910B104B
:1079000070910C1080910D1090910E100E949BA10F
:10791000DC01CB0143C06091F9067091FA0688271B
:1079200077FD8095982F0E94CEA16B017C0160911C
:10793000BF0F7091C00F8091C10F9091C20F0E9434
:10794000CEA12B013C01C701B60120910B10309153
:107950000C1040910D1050910E100E9433A19B010C
:10796000AC01C301B2010E9401A40E94D1A36093A3
:10797000BF0F7093C00F8093C10F9093C20FC0923E
:107980000B10D0920C10E0920D10F0920E10C80166
:10799000880F991F880F991F800F911F9093FA06E7
:1079A0008093F9060E941E9DDC01CB018C509E4FF6
:1079B000AF4FBF4F8093EC099093ED09A093EE0970
:1079C000B093EF090E945631F5018085882351F16B
:1079D0008091F9069091FA068530910534F485E09E
:1079E00090E09093FA068093F9068091F9069091C1
:1079F000FA06F7E280319F0734F08FE097E2909328
:107A0000FA068093F90682EE96E06DE0492D0E9419
:107A1000339F89EF96E00E943939BC0182EE96E0EF
:107A20000E94249E0894211C311C922C422D480D4A
:107A3000F5015681852F992787FD909503962B890F
:107A40003C89220D331D821793070CF07DCC808575
:107A5000882309F06FC057830091F9061091FA0648
:107A60001382848195819801281B390BC9010496E2
:107A70008930910508F05EC082EE96E060E04081BA
:107A80000E94339F82EE96E060E20E94359EF501EF
:107A9000868117FF06C08150868387FF48C0168203
:107AA00046C0053111054CF08F5FF50186838330A8
:107AB00014F082E086830FE010E01093FA06009342
:107AC000F906F50115830483C80165E070E00E94A2
:107AD000FAA46083643011F483E08083F50180812F
:107AE000863014F085E08083F501978186819817B0
:107AF00011F081E0838382EE96E060E0F501408141
:107B00000E94339FF5018081992787FD90952681FA
:107B1000332727FD3095820F931F009711F06EE3F6
:107B200001C063E082EE96E00E94359E03C004E04F
:107B300010E0C3CF64960FB6F894DEBF0FBECDBF82
:107B4000DF91CF911F910F91FF90EF90DF90CF9039
:107B5000BF90AF909F908F907F906F905F904F906D
:107B60003F902F900895FC01608171818281938103
:107B700020E030E040E251E40E9401A40E949BA179
:107B80009B0177FD02C08BE201C08DE280930B0A5E
:107B900037FF03C0309521953F4FC90160E177E27F
:107BA0000E94FAA4CB01EAE0F0E0BF010E94FAA42F
:107BB000805D80930C0AC90168EE73E00E94FAA40C
:107BC000CB01BF010E94FAA4805D80930D0AC90118
:107BD00064E670E00E94FAA4CB01BF010E94FAA4FF
:107BE000805D80930E0AC901BF010E94FAA4282F6C
:107BF000CB01BF010E94FAA4805D80930F0A8EE240
:107C00008093100A205D2093110A1092120A8BE0D3
:107C10009AE008954F925F926F927F928F929F9217
:107C2000AF92BF92CF92DF92EF92FF920F931F938A
:107C3000CF93DF93CDB7DEB76A970FB6F894DEBF68
:107C40000FBECDBF5C01FC0197818681981719F4A6
:107C50008381882339F081E0F501838382EE96E009
:107C60000E94619FF501868066247724482C552464
:107C700047FC5094CEC4433009F472C144304CF4F4
:107C8000413009F446C042300CF0B8C0442371F0D2
:107C9000BDC4453009F47FC245300CF4EAC146301A
:107CA00009F453C3473009F0B1C407C4F501838117
:107CB000882351F082EE96E060E0462D0E94339FCB
:107CC00080EC90E10E94D62BF5012081332727FD1F
:107CD0003095892D90E02817390709F097C48091D5
:107CE000FB0682FF93C40E941E9DDC01CB018C50D9
:107CF0009E4FAF4FBF4F8093EC099093ED09A09337
:107D0000EE09B093EF0984E0F50181830E945631BA
:107D10007DC4F50183818823A1F182EE96E060E0C5
:107D2000462D0E94339F8BEC90E10E94D62B82EE71
:107D300096E06DE0462D0E94339F80911E0A90913F
:107D40001F0A60E00E949E6D20E030E040E05FE3AB
:107D50000E9453A00E949BA1882777FD8095982FB1
:107D60000E94CEA1DC01CB018F8B988FA98FBA8F97
:107D7000CE0147960E94CD38BC0182EE96E00E946B
:107D8000249EF5018081992787FD9095292D30E06B
:107D90008217930709F03AC48091FB0682FFC5C0A1
:107DA000808591E089278087882341F080911E0A91
:107DB00090911F0A60E00E949E6D72C06091F9066A
:107DC0007091FA06882777FD8095982F0E94CEA1A2
:107DD0006B017C010E949BA1DC01CB0160E00E9451
:107DE000536D90931F0A80931E0AC092140AD0927A
:107DF000150AE092160AF092170A75C0F501838100
:107E0000882399F182EE96E060E0462D0E94339F30
:107E100085ED90E10E94D62B82EE96E06DE0462D36
:107E20000E94339F80911C0A90911D0A0E940E703F
:107E300020E030E040E05FE30E9453A00E949BA15D
:107E4000882777FD8095982F0E94CEA1DC01CB0179
:107E50008B8B9C8BAD8BBE8BCE0143960E94CD3815
:107E6000BC0182EE96E00E94249EF5018081992754
:107E700087FD9095292D30E08217930709F0C6C33E
:107E80008091FB0682FF51C0808591E08927808721
:107E90008823A9F080911C0A90911D0A0E940E70FF
:107EA00020E030E040E05FE30E9453A00E949BA1ED
:107EB000DC01CB019093FA068093F90626C060910D
:107EC000F9067091FA06882777FD8095982F0E9411
:107ED000CEA10E949BA1DC01CB010E949B6D9093DF
:107EE0001D0A80931C0AF5012081332727FD309558
:107EF000C901880F991F880F991F820F931F9093B4
:107F0000FA068093F9060E9456310E941E9DDC01FC
:107F1000CB018C509E4FAF4FBF4F8093EC09909395
:107F2000ED09A093EE09B093EF09F5018085882350
:107F300009F46CC38091F9069091FA0697FF04C08A
:107F40001092FA061092F9068091F9069091FA06BD
:107F5000F1E085309F070CF44AC384E091E043C30D
:107F6000F5018381882331F182EE96E060E0462DB1
:107F70000E94339F8CED90E10E94D62B82EE96E01A
:107F80006DE0462D0E94339F6091FD0670E080E019
:107F900090E00E94CCA1DC01CB018F87988BA98B4C
:107FA000BA8BCE010F960E94CD38BC0182EE96E0CE
:107FB0000E94249EF5012081332727FD3095892DCD
:107FC00090E02817390709F021C38091FB0682FF52
:107FD0002AC0808591E089278087882339F08091A5
:107FE000FD068093F9061092FA060DC0C901880FAC
:107FF000991F880F991F820F931F9093FA06809301
:10800000F9060E9456310E941E9DDC01CB018C5066
:108010009E4FAF4FBF4F8093EC099093ED09A09313
:10802000EE09B093EF09F5018085882309F4EEC2CB
:108030008091F9069091FA0697FF04C01092FA0613
:108040001092F9068091F9069091FA068F3F9105FA
:1080500039F034F08FEF90E09093FA068093F906B0
:108060006091F9066093FD0687E070E00E942C9B0A
:10807000BEC2F5018381882339F182EE96E060E08B
:10808000462D0E94339F88EE90E10E94D62B82EE0F
:1080900096E06DE0462D0E94339F6091360470910A
:1080A000370480913804909139040E949BA1DC012F
:1080B000CB019E838D83CE0105960E943939BC0188
:1080C00082EE96E00E94249EF5010081112707FDB3
:1080D0001095892D90E00817190709F097C2809133
:1080E000FB0682FF44C0808591E089278087882332
:1080F00069F0609136047091370480913804909152
:1081000039040E949BA1DC01CB011BC06091F906E0
:108110007091FA06882777FD8095982F0E94CEA14E
:10812000DC01CB018093360490933704A09338048C
:10813000B0933904C801880F991F880F991F800FC9
:10814000911F9093FA068093F9060E941E9DDC0110
:10815000CB018C509E4FAF4FBF4F8093EC09909353
:10816000ED09A093EE09B093EF090E945631F50195
:108170008085882309F44AC28091F9069091FA0615
:10818000181619060CF480C181E090E09093FA066D
:108190008093F90679C1F5018381882369F182EE24
:1081A00096E060E0462D0E94339F81EF90E10E94AF
:1081B000D62B82EE96E06DE0462D0E94339F6091B3
:1081C00032047091330480913404909135042FE689
:1081D00032E143E05EE30E9433A1DC01CB018B87F7
:1081E0009C87AD87BE87CE010B960E94B33DBC0134
:1081F00082EE96E00E94249EF5010081112707FD82
:108200001095892D90E00817190709F0FFC180919A
:10821000FB0682FF5CC0808591E0892780878823E8
:10822000C9F06091320470913304809134049091CC
:10823000350420E030E040E251E40E9401A42FE642
:1082400032E143E05EE30E9433A10E949BA1DC0186
:10825000CB0127C06091F9067091FA06882777FD57
:108260008095982F0E94CEA120E030E040E251E4BA
:108270000E9433A12FE632E143E05EE30E9401A4B5
:10828000DC01CB018093320490933304A093340437
:10829000B0933504C801880F991F880F991F800F6C
:1082A000911F9093FA068093F9060E941E9DDC01AF
:1082B000CB018C509E4FAF4FBF4F8093EC099093F2
:1082C000ED09A093EE09B093EF090E945631F50134
:1082D0008085882309F49AC18091F9069091FA0665
:1082E00097FF04C01092FA061092F9068091F906E1
:1082F0009091FA06F7E287309F0734F086E097E224
:108300009093FA068093F90682EE96E06DE0492D8F
:108310000E94339F6091F9067091FA06882777FDD5
:108320008095982F0E94CEA120E030E040E251E4F9
:108330000E9433A1DC01CB018F839887A987BA877C
:10834000CE0107960E94B33D5CC1F501838188236D
:1083500069F182EE96E060E0462D0E94339F8AEF3D
:1083600090E10E94D62B82EE96E06DE0462D0E94B1
:10837000339F60912E0470912F048091300490916E
:1083800031042FE632E143E05EE30E9401A40E9443
:108390009BA1DC01CB019C838B83CE0103960E94C1
:1083A0003939BC0182EE96E00E94249EF5010081DD
:1083B000112707FD1095892D90E00817190709F07E
:1083C00025C18091FB0682FF50C0808591E08927FE
:1083D00080878823C9F060912E0470912F048091CA
:1083E00030049091310420E030E040EA50E40E94F3
:1083F00033A12FE632E143E05EE30E9433A10E9405
:108400009BA1DC01CB011BC06091F9067091FA06BB
:10841000882777FD8095982F0E94CEA1DC01CB01A3
:1084200080932E0490932F04A0933004B0933104D2
:10843000C801880F991F880F991F800F911F909373
:10844000FA068093F9060E941E9DDC01CB018C5038
:108450009E4FAF4FBF4F8093EC099093ED09A093CF
:10846000EE09B093EF090E945631F501808588230B
:1084700009F4CCC08091F9069091FA0697FF04C0E8
:108480001092FA061092F9068091F9069091FA0678
:10849000F7E287309F0734F086E097E29093FA0680
:1084A0008093F90682EE96E06DE0492D0E94339F9D
:1084B00089EF96E00E943939A4C0F50183818823B1
:1084C00039F182EE96E060E0462D0E94339F83E012
:1084D00091E10E94D62B82EE96E06DE0462D0E943F
:1084E000339F60912A0470912B0480912C04909109
:1084F0002D040E949BA1DC01CB019A838983CE01CC
:1085000001960E941039BC0182EE96E00E94249EE2
:10851000F5010081112707FD1095892D90E00817BE
:10852000190709F073C08091FB0682FF44C0808563
:1085300091E089278087882369F060912A047091EF
:108540002B0480912C0490912D040E949BA1DC01AE
:10855000CB011BC06091F9067091FA06882777FD60
:108560008095982F0E94CEA1DC01CB0180932A0434
:1085700090932B04A0932C04B0932D04C801880F72
:10858000991F880F991F800F911F9093FA0680936F
:10859000F9060E941E9DDC01CB018C509E4FAF4F0F
:1085A000BF4F8093EC099093ED09A093EE09B0932F
:1085B000EF090E945631F5018085882339F18091B9
:1085C000F9069091FA0697FF04C01092FA061092ED
:1085D000F9068091F9069091FA06F3E08F3D9F0726
:1085E00034F08EED93E09093FA068093F90682EED4
:1085F00096E06DE0492D0E94339F89EF96E00E943E
:108600001039BC0182EE96E00E94249E0894611C01
:10861000711C962C462D480DF5015681852F992702
:1086200087FD909503969301240D351D82179307BE
:108630000CF021CB8085882309F06FC0578300910F
:10864000F9061091FA061382848195819801281BFE
:10865000390BC90104968930910508F05EC082EE9D
:1086600096E060E040810E94339F82EE96E060E2F7
:108670000E94359EF501868117FF06C081508683D2
:1086800087FF48C0168246C0053111054CF08F5F48
:10869000F5018683853014F084E086830FE010E0D6
:1086A0001093FA060093F906F50115830483C801B7
:1086B00065E070E00E94FAA46083643011F483E006
:1086C0008083F5018081883014F087E08083F50194
:1086D00097818681981711F081E0838382EE96E07E
:1086E00060E0F50140810E94339FF5018081992768
:1086F00087FD90952681332727FD3095820F931FA4
:10870000009711F06EE301C063E082EE96E00E94F4
:10871000359E03C004E010E0C3CF6A960FB6F8940C
:10872000DEBF0FBECDBFDF91CF911F910F91FF90A4
:10873000EF90DF90CF90BF90AF909F908F907F9001
:108740006F905F904F900895FC01608171818281EC
:10875000938120E030E048EC52E40E9401A40E94A2
:108760009BA19B0177FD02C08BE201C08DE280934B
:108770000B0A37FF03C0309521953F4FC90160E1D7
:1087800077E20E94FAA4CB01EAE0F0E0BF010E9488
:10879000FAA4805D80930C0AC90168EE73E00E9420
:1087A000FAA4CB01BF010E94FAA4805D80930D0A58
:1087B000C90164E670E00E94FAA4CB01BF010E94E7
:1087C000FAA4805D80930E0A8EE280930F0AC9019D
:1087D000BF010E94FAA4282FCB01BF010E94FAA476
:1087E000805D8093100A205D2093110A1092120A76
:1087F0008BE09AE008952F923F924F925F926F9292
:108800007F928F929F92AF92BF92CF92DF92EF9220
:10881000FF920F931F93CF93DF93CDB7DEB7A89747
:108820000FB6F894DEBF0FBECDBF7C01FC0197816F
:108830008681981719F48381882339F081E0F70144
:10884000838382EE96E00E94619FF7016680262D69
:10885000332727FD309538A72FA3220F331F220F70
:10886000331F2553304F3CA32BA36FA178A5660F70
:10887000771F660F771F6D5F7F4E7EA36DA3222447
:1088800033243AA229A2262C37010C94F04C78E02C
:10889000271609F434C27215ACF082E0281609F4E8
:1088A0002DC1821544F0222039F191E0291611F0F2
:1088B0000C94DE4C58C0F3018381F6E0F2150CF005
:1088C0007BC17BC22EE0221609F4B6C422153CF00F
:1088D000F3018381FCE0F2150CF013C3E4C320E143
:1088E000221609F487C622160CF495C531E1231629
:1088F00011F00C94DE4C6DC7F3018381882351F095
:1089000082EE96E060E049A10E94339F8CE091E105
:108910000E94D62BF3012081332727FD30958C2D23
:1089200090E02817390711F00C94DE4C8091FB067B
:1089300082FD02C00C94DE4C0E941E9DDC01CB0126
:108940008C509E4FAF4FBF4F8093EC099093ED0931
:10895000A093EE09B093EF0984E0F30181830E94B4
:1089600056310C94DE4CF3018381882389F182EE29
:1089700096E060E049A10E94339F87E191E10E9467
:10898000D62B82EE96E06DE049A10E94339F609164
:10899000E70F7091E80F8091E90F9091EA0F20E0C6
:1089A00030E048EC52E40E9433A10E949BA1DC011C
:1089B000CB019C878B87CE010B960E941039BC019E
:1089C00082EE96E00E94249E8DE191E10E94D62BDA
:1089D000F3010081112707FD10958C2D90E00817F9
:1089E000190709F0EBC78091FB0682FF55C080850F
:1089F00091E0892780878823A9F06091E70F709123
:108A0000E80F8091E90F9091EA0F0E949BA1DC0191
:108A1000CB0164E670E00E94FAA47093FA066093BA
:108A2000F90628C08091F9069091FA0624E630E014
:108A3000829FB001839F700D929F700D1124882733
:108A400077FD8095982F0E94CEA1DC01CB01809309
:108A5000E70F9093E80FA093E90FB093EA0FC801D6
:108A6000880F991F880F991F800F911F9093FA0606
:108A70008093F9060E941E9DDC01CB018C509E4F15
:108A8000AF4FBF4F8093EC099093ED09A093EE098F
:108A9000B093EF090E945631F3018085882309F4D1
:108AA0008DC78091F9069091FA068530910534F4CE
:108AB00085E090E09093FA068093F9068091F9069C
:108AC0009091FA06F3E08F3D9F0734F08EED93E02E
:108AD0009093FA068093F90682EE96E06DE04C2DB5
:108AE0000E94339F89EF96E00E941039BC0182EE0C
:108AF00096E00E94249E80E291E1D2C2F30183813C
:108B0000882339F182EE96E060E049A10E94339F0C
:108B100083E291E10E94D62B82EE96E06DE049A1BE
:108B20000E94339F6091DF0F7091E00F8091E10F01
:108B30009091E20F0E949BA1DC01CB019A8789876B
:108B4000CE0109960E941039BC0182EE96E00E9487
:108B5000249EF3010081112707FD10958C2D90E0D4
:108B60000817190709F02AC78091FB0682FFB3C0D6
:108B7000808591E089278087882349F06091DF0F05
:108B80007091E00F8091E10F9091E20F70C06091C1
:108B9000F9067091FA06882777FD8095982F0E9434
:108BA000CEA1DC01CB018093DF0F9093E00FA09367
:108BB000E10FB093E20F72C08823F1F182EE96E0EC
:108BC00060E049A10E94339F8FE291E10E94D62B81
:108BD00023E0221619F486E391E111C034E0231654
:108BE00019F489E391E10BC065E0261619F48CE3D2
:108BF00091E105C076E0271621F48FE391E10E9410
:108C0000D62B82EE96E06DE04C2D0E94339FEDA1B5
:108C1000FEA160817181828193810E949BA1DC0110
:108C2000CB0198878F83CE0107960E941039BC0133
:108C300082EE96E00E94249EF3010081112707FD39
:108C400010958C2D90E00817190709F0B7C6809190
:108C5000FB0682FF40C0808591E0892780878823BA
:108C600059F0EDA1FEA160817181828193810E9402
:108C70009BA1DC01CB0119C06091F9067091FA0645
:108C8000882777FD8095982F0E94CEA1DC01CB012B
:108C9000EDA1FEA180839183A283B383C801880FD5
:108CA000991F880F991F800F911F9093FA06809348
:108CB000F9060E941E9DDC01CB018C509E4FAF4FE8
:108CC000BF4F8093EC099093ED09A093EE09B09308
:108CD000EF090E945631F3018085882309F46EC69E
:108CE0008091F9069091FA06181619060CF4F0C056
:108CF00081E090E09093FA068093F906E9C0F301D1
:108D00008381882339F182EE96E060E049A10E94D8
:108D1000339F82E491E10E94D62B82EE96E06DE0D3
:108D200049A10E94339F6091EB0F7091EC0F8091ED
:108D3000ED0F9091EE0F0E949BA1DC01CB019E8371
:108D40008D83CE0105960E941039BC0182EE96E01B
:108D50000E94249EF3010081112707FD10958C2DA0
:108D600090E00817190709F029C68091FB0682FFD9
:108D7000A0C0808591E089278087882349F0609191
:108D8000EB0F7091EC0F8091ED0F9091EE0F5BC0A7
:108D90006091F9067091FA06882777FD8095982FE3
:108DA0000E94CEA1DC01CB018093EB0F9093EC0FDE
:108DB000A093ED0FB093EE0F5FC0882339F182EEE0
:108DC00096E060E049A10E94339F89E491E10E940E
:108DD000D62B82EE96E06DE049A10E94339F609110
:108DE000D30F7091D40F8091D50F9091D60F0E9420
:108DF0009BA1DC01CB019C838B83CE0103960E9457
:108E00001039BC0182EE96E00E94249EF30100819D
:108E1000112707FD10958C2D90E00817190709F010
:108E2000CDC58091FB0682FF44C0808591E08927F3
:108E30008087882369F06091D30F7091D40F80915F
:108E4000D50F9091D60F0E949BA1DC01CB011BC0D6
:108E50006091F9067091FA06882777FD8095982F22
:108E60000E94CEA1DC01CB018093D30F9093D40F4D
:108E7000A093D50FB093D60FC801880F991F880F04
:108E8000991F800F911F9093FA068093F9060E9414
:108E90001E9DDC01CB018C509E4FAF4FBF4F809386
:108EA000EC099093ED09A093EE09B093EF090E94AD
:108EB0005631F3018085882309F480C58091F90635
:108EC0009091FA0697FF04C01092FA061092F906E4
:108ED0008091F9069091FA06F3E08F3D9F0734F0F8
:108EE0008EED93E09093FA068093F90682EE96E079
:108EF0006DE04C2D0E94339F89EF96E00E9410395F
:108F000058C5882309F444C082EE96E060E049A188
:108F10000E94339F85E591E10E94D62B29E022161D
:108F200019F48CE591E111C03AE0231619F48FE5AC
:108F300091E10BC06BE0261619F482E691E105C0C1
:108F40007CE0271621F485E691E10E94D62B82EE83
:108F500096E06DE04C2D0E94339FEBA1FCA1608157
:108F600071818281938124E630E040E050E00E94EC
:108F70000DA53A832983CE0101960E941039BC01C8
:108F800082EE96E00E94249E88E691E10E94D62B14
:108F9000F3016081772767FD70958C2D90E068174D
:108FA000790709F00BC58091FB0682FF48C08085D8
:108FB00091E089278087882369F0EBA1FCA180815B
:108FC000918164E670E00E94FAA47093FA066093BF
:108FD000F90623C08091F9069091FA0624E630E064
:108FE000829FA001839F500D929F500D1124CA01B2
:108FF000AA2797FDA095BA2FEBA1FCA180839183AE
:10900000A283B383CB01880F991F880F991F860F06
:10901000971F9093FA068093F9060E941E9DDC012B
:10902000CB018C509E4FAF4FBF4F8093EC09909374
:10903000ED09A093EE09B093EF090E945631F301B8
:109040008085882309F4BAC48091F9069091FA06C4
:109050001816190634F081E090E09093FA06809398
:10906000F9068091F9069091FA06F3E08F3D9F078B
:1090700034F08EED93E09093FA068093F90682EE39
:1090800096E06DE04C2D0E94339F89EF96E00E94A0
:109090001039BC0182EE96E00E94249E8BE691E19D
:1090A0000E94D62B8BC4882389F182EE96E060E083
:1090B00049A10E94339F8EE691E10E94D62B82EE59
:1090C00096E06DE049A10E94339F6091E30F70919B
:1090D000E40F8091E50F9091E60F20E030E048EC3E
:1090E00052E40E9433A1DC01CB018D8F9E8FAF8FA4
:1090F000B8A3CE014D960E94CD38BC0182EE96E019
:109100000E94249E8AE791E10E94D62BF301008100
:10911000112707FD10958C2D90E00817190709F00D
:109120004DC48091FB0682FF55C0808591E0892760
:1091300080878823A9F06091E30F7091E40F8091FC
:10914000E50F9091E60F0E949BA1DC01CB0164E644
:1091500070E00E94FAA47093FA066093F90628C0A2
:109160008091F9069091FA0624E630E0829FB001E2
:10917000839F700D929F700D1124882777FD809535
:10918000982F0E94CEA1DC01CB018093E30F909336
:10919000E40FA093E50FB093E60FC801880F991F65
:1091A000880F991F800F911F9093FA068093F906FC
:1091B0000E941E9DDC01CB018C509E4FAF4FBF4FD4
:1091C0008093EC099093ED09A093EE09B093EF0919
:1091D0000E945631F3018085882309F4EFC3809102
:1091E000F9069091FA068A30910534F48AE090E00D
:1091F0009093FA068093F9068091F9069091FA0609
:10920000F3E08F3D9F0734F08EED93E09093FA06E4
:109210008093F90682EE96E06DE04C2D0E94339F1C
:1092200089EF96E00E941039BC0182EE96E00E9420
:10923000249E8DE791E134CFF30183818823C9F027
:1092400082EE96E060E049A10E94339F80E891E1C0
:109250000E94D62B82EE96E06BE049A10E94339FDC
:109260008FEF9FE00E94A443BC0182EE96E00E9433
:10927000249EF3014080552447FC50948C2D90E0AF
:109280004816590609F09AC38091FB0682FF84C0F4
:10929000808591E089278087882399F06091FF0F6E
:1092A00070910010809101109091021020E030E048
:1092B00048EC52E40E9401A40E949BA1DC01CB0176
:1092C00055C06091F9067091FA06882777FD809560
:1092D000982F0E94CEA120E030E048EC52E40E949A
:1092E00033A1162F072FE82ED92E6091B30F70915E
:1092F000B40F8091B50F9091B60F0E94CEA14B0193
:109300005C01A801852F942FAE2DBD2DBC01CD0190
:109310002091FF0F309100104091011050910210E8
:109320000E9433A19B01AC01C501B4010E9401A4BC
:109330000E94D1A36093B30F7093B40F8093B50FC5
:109340009093B60FA801852F942FAE2DBD2D80933D
:10935000FF0F90930010A0930110B0930210C20170
:10936000880F991F880F991F840D951D9093FA06F9
:109370008093F9060E941E9DDC01CB018C509E4F0C
:10938000AF4FBF4F8093EC099093ED09A093EE0986
:10939000B093EF090E945631F3018085882309F4C8
:1093A0000DC38091F9069091FA068530910534F449
:1093B00085E090E09093FA068093F9068091F90693
:1093C0009091FA06FDE781309F0734F080E09DE739
:1093D0009093FA068093F90682EE96E06BE04C2DAE
:1093E0000E94339F6091F9067091FA06882777FDF5
:1093F0008095982F0E94CEA120E030E048EC52E406
:109400000E9433A1DC01CB01898F9A8FAB8FBC8F77
:10941000CE014996CCC2F30183818823C9F082EE44
:1094200096E060E049A10E94339F8CE891E10E94A0
:10943000D62B82EE96E06BE049A10E94339F83E039
:1094400090E10E94A443BC0182EE96E00E94249E1B
:10945000F3014080552447FC50948C2D90E0481631
:10946000590609F0ABC28091FB0682FF84C080855B
:1094700091E089278087882399F06091031070918B
:109480000410809105109091061020E030E048EC27
:1094900052E40E9401A40E949BA1DC01CB0155C0B3
:1094A0006091F9067091FA06882777FD8095982FCC
:1094B0000E94CEA120E030E048EC52E40E9433A1AB
:1094C000162F072FE82ED92E6091B70F7091B80F85
:1094D0008091B90F9091BA0F0E94CEA14B015C010F
:1094E000A801852F942FAE2DBD2DBC01CD0120915B
:1094F00003103091041040910510509106100E9405
:1095000033A19B01AC01C501B4010E9401A40E94DA
:10951000D1A36093B70F7093B80F8093B90F909356
:10952000BA0FA801852F942FAE2DBD2D8093031067
:1095300090930410A0930510B0930610C201880FF9
:10954000991F880F991F840D951D9093FA0680939B
:10955000F9060E941E9DDC01CB018C509E4FAF4F3F
:10956000BF4F8093EC099093ED09A093EE09B0935F
:10957000EF090E945631F3018085882309F41EC249
:109580008091F9069091FA068530910534F485E0D2
:1095900090E09093FA068093F9068091F9069091F5
:1095A000FA06F7E280319F0734F08FE097E290935C
:1095B000FA068093F90682EE96E06BE04C2D0E944D
:1095C000339F6091F9067091FA06882777FD8095A0
:1095D000982F0E94CEA120E030E048EC52E40E9497
:1095E00033A1DC01CB018D8B9E8BAF8BB88FCE016D
:1095F0004596DDC1F30183818823C9F082EE96E0B0
:1096000060E049A10E94339F88E991E10E94D62B36
:1096100082EE96E06BE049A10E94339F87E090E1E3
:109620000E94A443BC0182EE96E00E94249EF301B6
:109630004080552447FC50948C2D90E048165906E4
:1096400009F0BCC18091FB0682FF84C0808591E057
:1096500089278087882399F06091071070910810FE
:109660008091091090910A1020E030E048EC52E41B
:109670000E9401A40E949BA1DC01CB0155C0609116
:10968000F9067091FA06882777FD8095982F0E9439
:10969000CEA120E030E048EC52E40E9433A1162F26
:1096A000072FE82ED92E6091BB0F7091BC0F8091CF
:1096B000BD0F9091BE0F0E94CEA14B015C01A8018D
:1096C000852F942FAE2DBD2DBC01CD01209107100B
:1096D000309108104091091050910A100E9433A156
:1096E0009B01AC01C501B4010E9401A40E94D1A359
:1096F0006093BB0F7093BC0F8093BD0F9093BE0F10
:10970000A801852F942FAE2DBD2D80930710909327
:109710000810A0930910B0930A10C201880F991F76
:10972000880F991F840D951D9093FA068093F90672
:109730000E941E9DDC01CB018C509E4FAF4FBF4F4E
:109740008093EC099093ED09A093EE09B093EF0993
:109750000E945631F3018085882309F42FC180913E
:10976000F9069091FA068530910534F485E090E091
:109770009093FA068093F9068091F9069091FA0683
:10978000F7E280319F0734F08FE097E29093FA067A
:109790008093F90682EE96E06BE04C2D0E94339F99
:1097A0006091F9067091FA06882777FD8095982FC9
:1097B0000E94CEA120E030E048EC52E40E9433A1A8
:1097C000DC01CB01898B9A8BAB8BBC8BCE01419694
:1097D000EEC0F30183818823C9F082EE96E060E059
:1097E00049A10E94339F84EA91E10E94D62B82EE28
:1097F00096E06BE049A10E94339F8BE090E10E94CC
:10980000A443BC0182EE96E00E94249EF3014080B6
:10981000552447FC50948C2D90E04816590609F0C9
:10982000CDC08091FB0682FF84C0808591E08927AE
:109830008087882399F060910B1070910C108091B3
:109840000D1090910E1020E030E048EC52E40E94A0
:1098500001A40E949BA1DC01CB0155C06091F906D7
:109860007091FA06882777FD8095982F0E94CEA1E7
:1098700020E030E048EC52E40E9433A1162F072F7D
:10988000E82ED92E6091BF0F7091C00F8091C10F4B
:109890009091C20F0E94CEA14B015C01A801852FBF
:1098A000942FAE2DBD2DBC01CD0120910B10309118
:1098B0000C1040910D1050910E100E9433A19B018D
:1098C000AC01C501B4010E9401A40E94D1A3609320
:1098D000BF0F7093C00F8093C10F9093C20FA80168
:1098E000852F942FAE2DBD2D80930B1090930C10CF
:1098F000A0930D10B0930E10C201880F991F880F0E
:10990000991F840D951D9093FA068093F9060E9485
:109910001E9DDC01CB018C509E4FAF4FBF4F8093FB
:10992000EC099093ED09A093EE09B093EF090E9422
:109930005631F3018085882309F440C08091F906EF
:109940009091FA068530910534F485E090E090938B
:10995000FA068093F9068091F9069091FA06F7E2EB
:1099600080319F0734F08FE097E29093FA0680935E
:10997000F90682EE96E06BE04C2D0E94339F6091D9
:10998000F9067091FA06882777FD8095982F0E9436
:10999000CEA120E030E048EC52E40E9433A1DC018B
:1099A000CB018D879E87AF87B88BCE010D960E9425
:1099B000A443BC0182EE96E00E94249E239429A138
:1099C0003AA12F5F3F4F3AA329A36BA17CA16C5F03
:1099D0007F4F7CA36BA38DA19EA104969EA38DA314
:1099E000C9A0F3014681842F992787FD909503969E
:1099F00029A13AA16FA178A5260F371F82179307D7
:109A000014F00C94474473018085882309F06FC0DB
:109A100047830091F9061091FA061382848195819B
:109A20009801281B390BC90104968930910508F06B
:109A30005EC082EE96E060E040810E94339F82EE3D
:109A400096E060E20E94359EF301868117FF06C012
:109A50008150868387FF48C0168246C005311105B4
:109A60004CF08F5FF30186838F3014F08EE0868395
:109A70000FE010E01093FA060093F906F701158342
:109A80000483C80165E070E00E94FAA4608364303A
:109A900011F483E08083F7018081823114F081E149
:109AA0008083F70197818681981711F081E0838385
:109AB00082EE96E060E0F70140810E94339FF7015B
:109AC0008081992787FD90952681332727FD309542
:109AD000820F931F009711F06EE301C063E082EEE6
:109AE00096E00E94359E03C004E010E0C3CFA89624
:109AF0000FB6F894DEBF0FBECDBFDF91CF911F919F
:109B00000F91FF90EF90DF90CF90BF90AF909F901C
:109B10008F907F906F905F904F903F902F9008951F
:109B2000CF92DF92EF92FF920F931F93CF93DF9329
:109B30008C01FC0197818681981719F48381882311
:109B400039F081E0F801838382EE96E00E94619F04
:109B5000F801D681EE24FF24CD2EDD24C7FCD0945D
:109B600000C2423009F4BFC0433034F4442359F0FA
:109B7000413009F0F3C138C0433009F433C14430F7
:109B800009F0ECC1B5C1F8018381882351F082EE60
:109B900096E060E04E2D0E94339F8CE690E10E949B
:109BA000D62BF8012081332727FD30958C2F90E0AC
:109BB0002817390709F0D2C18091FB0682FFCEC178
:109BC0000E941E9DDC01CB018C509E4FAF4FBF4FBA
:109BD0008093EC099093ED09A093EE09B093EF09FF
:109BE00081E0F8018183B8C1F80183818823C9F03D
:109BF00082EE96E060E04E2D0E94339F87E790E171
:109C00000E94D62B82EE96E06BE04E2D0E94339F91
:109C10008BE097E00E94A443BC0182EE96E00E9494
:109C2000249EF8018081992787FD90952C2F30E0A4
:109C30008217930709F092C18091FB0682FF31C021
:109C4000808591E089278087882329F088E792E042
:109C50000E94AA2816C08CE792E00E94AA28F80168
:109C60002081332727FD3095C901880F991F880F60
:109C7000991F820F931F9093FA068093F9060E9412
:109C800056310E941E9DDC01CB018C509E4FAF4F80
:109C9000BF4F8093EC099093ED09A093EE09B09328
:109CA000EF09F8018085882309F458C18091F906ED
:109CB0009091FA06181619061CF480E892E004C088
:109CC000009741F08DE892E00E94AA281092FA06CF
:109CD0001092F90682EE96E06BE04C2F0E94339FC3
:109CE0008BE097E0FDC0F80183818823C9F082EE04
:109CF00096E060E04E2D0E94339F8BE790E10E943A
:109D0000D62B82EE96E06BE04E2D0E94339F8FE0C3
:109D100097E00E94A443BC0182EE96E00E94249E3C
:109D2000F8018081992787FD90952C2F30E08217CC
:109D3000930709F013C18091FB0682FF31C0808533
:109D400091E089278087882329F088E792E00E94A4
:109D5000AA2816C08CE792E00E94AA28F801208168
:109D6000332727FD3095C901880F991F880F991F48
:109D7000820F931F9093FA068093F9060E94563142
:109D80000E941E9DDC01CB018C509E4FAF4FBF4FF8
:109D90008093EC099093ED09A093EE09B093EF093D
:109DA000F8018085882309F4D9C08091F906909143
:109DB000FA06181619061CF48BE992E004C0009705
:109DC00041F088EA92E00E94AA281092FA061092C6
:109DD000F90682EE96E06BE04C2F0E94339F8FE0F5
:109DE00097E07EC0F80183818823C9F082EE96E077
:109DF00060E04E2D0E94339F8FE790E10E94D62BAA
:109E000082EE96E06BE04E2D0E94339F83E197E057
:109E10000E94A443BC0182EE96E00E94249EF801B9
:109E20008081992787FD90952C2F30E0821793072A
:109E300009F094C08091FB0682FF31C0808591E0DB
:109E400089278087882329F088E792E00E94AA2842
:109E500016C08CE792E00E94AA28F80120813327DF
:109E600027FD3095C901880F991F880F991F820F10
:109E7000931F9093FA068093F9060E9456310E9430
:109E80001E9DDC01CB018C509E4FAF4FBF4F809386
:109E9000EC099093ED09A093EE09B093EF09F80156
:109EA0008085882309F45AC08091F9069091FA06BA
:109EB000181619061CF486EB92E004C0009741F0D6
:109EC00082EC92E00E94AA281092FA061092F906FB
:109ED00082EE96E06BE04C2F0E94339F83E197E087
:109EE0000E94A443BC0182EE96E00E94249E36C0EC
:109EF000F8018381882351F082EE96E060E04E2DD8
:109F00000E94339F83E890E10E94D62BF8012081C4
:109F1000332727FD30958C2F90E028173907F1F46F
:109F20008091FB0682FF1AC00E941E9DDC01CB01BE
:109F30008C509E4FAF4FBF4F8093EC099093ED092B
:109F4000A093EE09B093EF098FEC92E00E94AA284B
:109F500086ED92E00E94AA280E9456310894E11CE6
:109F6000F11CCE2D4E2D4D0FF8015681852F9927CE
:109F700087FD9095039697012C0D3D1D8217930741
:109F80000CF0EFCD8085882309F06FC05783C09116
:109F9000F906D091FA061382848195819E01281BCF
:109FA000390BC90104968930910508F05EC082EE34
:109FB00096E060E040810E94339F82EE96E060E28E
:109FC0000E94359EF8018681D7FF06C081508683A6
:109FD00087FF48C0168246C0C531D1054CF08F5F5F
:109FE000F8018683823014F081E08683CFE0D0E0F0
:109FF000D093FA06C093F906F801D583C483CE0145
:10A0000065E070E00E94FAA46083643011F483E09C
:10A010008083F8018081853014F084E08083F8012A
:10A0200097818681981711F081E0838382EE96E014
:10A0300060E0F80140810E94339FF80180819927F8
:10A0400087FD90952681332727FD3095820F931F3A
:10A05000009711F06EE301C063E082EE96E00E948B
:10A06000359E03C0C4E0D0E0C3CFDF91CF911F91F4
:10A070000F91FF90EF90DF90CF9008952F923F9235
:10A080004F925F926F927F928F929F92AF92BF9208
:10A09000CF92DF92EF92FF920F931F93CF93DF93B4
:10A0A000CDB7DEB72E970FB6F894DEBF0FBECDBF8B
:10A0B0001C01FC0183818823B1F080910A049091F6
:10A0C0000B049093FA068093F90682EE96E00E94C4
:10A0D000619F82EE96E060E040E00E94339F80EE58
:10A0E0009FE00E94D62B80911A0A90911B0A60E093
:10A0F0000E949E6D20E030E040E05FE30E9453A0AC
:10A100000E949BA18B019C018091250490912604C3
:10A110000817190721F4F1018381882301F182EEE8
:10A1200096E061E040E00E94339FB801882777FD08
:10A130008095982F0E94CEA1DC01CB018B879C8754
:10A14000AD87BE87CE010B960E94CD38BC0182EE52
:10A1500096E00E94249E109326040093250480918B
:10A160001E0A90911F0A60E00E949E6D20E030E080
:10A1700040E05FE30E9453A00E949BA18B019C01E1
:10A1800080912704909128040817190721F4F10100
:10A190008381882301F182EE96E065E040E00E9431
:10A1A000339FB801882777FD8095982F0E94CEA114
:10A1B000DC01CB018F839887A987BA87CE010796E8
:10A1C0000E94CD38BC0182EE96E00E94249E10933E
:10A1D0002804009327048091A2099091A309A091DB
:10A1E000A409B091A5090097A105B10509F456C0CD
:10A1F00082EE96E060E041E00E94339F0E941E9D47
:10A200008090A2099090A309A090A409B090A509FC
:10A210000091FF091091000A20E030E080169106BD
:10A22000A206B306D9F1E0E6CE2EEAEEDE2EE12C50
:10A23000F12CA70196010E940DA529013A01C50143
:10A24000B401A70196010E940DA58201021B130B08
:10A25000C8016CE370E00E94E6A4C82E6A83CE01B8
:10A2600002960E94F838BC0182EE96E00E94249E7D
:10A270008BEE9FE00E94D62BC982CE0101960E94F0
:10A28000F838BC0182EE96E00E94249E8EEE9FE09C
:10A290000E94D62B1093000A0093FF0960911307C8
:10A2A00070911407809115079091160720E030E017
:10A2B00048EC52E40E9401A40E949BA18B019C01E6
:10A2C0008091010A9091020A0817190721F4F101FF
:10A2D00083818823B9F082EE96E06AE041E00E9433
:10A2E000339F80EF9FE00E94D62B83E197E00E948E
:10A2F000A443BC0182EE96E00E94249E1093020AC1
:10A300000093010A20910A0430910B043E832D83AF
:10A3100080911B07882331F010921B073093FA06B7
:10A320002093F9068091F9069091FA068217930717
:10A3300021F4F10123812223E9F09E838D838A3069
:10A34000910524F48AE090E09E838D838D819E8127
:10A35000F3E0883E9F0724F087EE93E09E838D8391
:10A360008D819E8190930B0480930A049093FA064A
:10A370008093F9068D819E812091030A3091040A11
:10A380008217930721F4F10123812223B9F09093DE
:10A39000040A8093030A82EE96E060E042E00E94A5
:10A3A000339FCE0105960E941039BC0182EE96E0E3
:10A3B0000E94249E83EF9FE00E94D62B08ED19E0B7
:10A3C0008091D809882339F182EE96E060E043E07D
:10A3D0000E94339F82EE96E0B8010E94249EF8010D
:10A3E00001900020E9F73197E01BF10BCC24DD242C
:10A3F00004E110E00E1B110909C082EE96E065E64B
:10A4000072E00E94249E0894C11CD11CC016D10683
:10A41000A4F31092D80980912307882339F1C090C2
:10A42000F407D090F507E090F607F090F707C11415
:10A43000D104E104F104D1F06091FC077091FD07B3
:10A440008091FE079091FF0724E630E040E050E065
:10A450000E94C7A4A70196010E940DA5022F2536D0
:10A4600031F4F1018381882311F416C000E082EEFB
:10A4700096E06AE042E00E94339F0B831C82CE018B
:10A4800003960E941039BC0182EE96E00E94249E41
:10A4900086EF9FE00E94D62BF10113822E960FB615
:10A4A000F894DEBF0FBECDBFDF91CF911F910F910A
:10A4B000FF90EF90DF90CF90BF90AF909F908F90E4
:10A4C0007F906F905F904F903F902F900895EF9204
:10A4D000FF920F931F93CF93DF937C018B01C4E016
:10A4E000D0E0F70120813181C901019691838083F9
:10A4F000F80161918F01C9010E94DDAA219789F7B6
:10A5000084E090E0DF91CF911F910F91FF90EF9049
:10A510000895EF92FF920F931F93CF93DF937C01E7
:10A520008B01C0E1D0E0F70120813181C9010196A2
:10A5300091838083F80161918F01C9010E94DDAA96
:10A54000219789F780E190E0DF91CF911F910F91E2
:10A55000FF90EF900895EF92FF920F931F93CF9388
:10A56000DF937C018B01C4E0D0E0F70120813181D1
:10A57000C901019691838083F80161918F01C9011E
:10A580000E94DDAA219789F784E090E0DF91CF91C6
:10A590001F910F91FF90EF9008950F931F93CF930A
:10A5A000DF93CDB7DEB72A970FB6F894DEBF0FBEA4
:10A5B000CDBF80E390E3A0E3B0E08F839887A987C5
:10A5C000BA8784E690E09A838983CE010196BE0122
:10A5D000695F7F4F0E946752CE0101966FEF7FE067
:10A5E0000E948952CE0101966FE070E10E9489526B
:10A5F0000FEE1FE089819A819C012F5F3F4F3A83C4
:10A600002983F80161918F010E94DDAAFFE00F3FCD
:10A610001F0781F7CE01019667EE7FE00E94AB52E3
:10A62000CE01019663EE7FE00E94AB52CE0101960F
:10A630006BEE7FE00E94AB52CE01019663ED7FE0AE
:10A640000E94AB520FE110E189819A819C012F5F3A
:10A650003F4F3A832983F80161918F010E94DDAA5F
:10A66000F0E103321F0781F7CE0101966FED7FE025
:10A670000E94AB52CE0101966BED7FE00E94AB527F
:10A68000CE01019667ED7FE00E94AB52CE010196AC
:10A6900066E374E00E94AB52CE01019662E374E07F
:10A6A0000E94AB52CE0101966EE274E00E94AB5262
:10A6B00086E590E3A5E3B0E08B839C83AD83BE8306
:10A6C00084E690E09A838983CE010196BE016D5F96
:10A6D0007F4F0E946752EAE6F9E007C09091C00000
:10A6E00095FFFCCF8093C600319684918823B1F703
:10A6F000EAE0FFE007C09091C00095FFFCCF809397
:10A70000C600319684918823B1F78091C00085FFFF
:10A71000FCCF8AE08093C6002A960FB6F894DEBF7D
:10A720000FBECDBFDF91CF911F910F910895EF9292
:10A73000FF920F931F93CF93DF937C018B01C0E1B6
:10A74000D0E0F701808191819C012F5F3F4F3183E1
:10A7500020830E94D5AAF80181938F01219789F760
:10A7600080E190E0DF91CF911F910F91FF90EF90EA
:10A770000895EF92FF920F931F93CF93DF937C0185
:10A780008B01C4E0D0E0F701808191819C012F5FB3
:10A790003F4F318320830E94D5AAF80181938F0116
:10A7A000219789F784E090E0DF91CF911F910F917D
:10A7B000FF90EF900895AF92BF92CF92DF92EF9209
:10A7C000FF920F931F93CF93DF93CDB7DEB7EA9736
:10A7D0000FB6F894DEBF0FBECDBFD82E84E690E052
:10A7E0009A83898386E590E3A5E3B0E08B839C831D
:10A7F000AD83BE831BE0E12EF12CEC0EFD1E8E011D
:10A80000095F1F4F89819A819C012F5F3F4F3A83D7
:10A8100029830E94D5AAF80181938F01EE15FF05C7
:10A8200089F7DD2009F097C0CE010396BE01695F6C
:10A830007F4F43E050E00E9467A8009709F08BC06B
:10A84000CE0101966FEF7FE00E949753CE010196F3
:10A850006FE070E10E9497530FEE1FE089819A81AB
:10A860009C012F5F3F4F3A8329830E94D5AAF801AC
:10A8700081938F01FFE00F3F1F0781F7CE01019603
:10A8800067EE7FE00E94B953CE01019663EE7FE050
:10A890000E94B953CE0101966BEE7FE00E94B9533E
:10A8A000CE01019663ED7FE00E94B9530FE110E104
:10A8B00089819A819C012F5F3F4F3A8329830E94AF
:10A8C000D5AAF80181938F01F0E103321F0781F7C8
:10A8D000CE0101966FED7FE00E94B953CE01019643
:10A8E0006BED7FE00E94B953CE01019667ED7FE0EA
:10A8F0000E94B953CE01019666E374E00E94B953F9
:10A90000CE01019662E374E00E94B953CE01019634
:10A910006EE274E00E94B953EAE6F9E007C0909154
:10A92000C00095FFFCCF8093C600319684918823A8
:10A93000B1F7E3E8FAE007C09091C00095FFFCCFC3
:10A940008093C600319684918823B1F78091C0002E
:10A9500085FFFCCFCEC0DE019B96E9EFF2E080E1FF
:10A9600001900D928150E1F7DE015B96E9E0F3E0A2
:10A9700080E101900D928150E1F7DE011B96E9E143
:10A98000F3E080E101900D928150E1F7FBE2AF2E00
:10A99000B12CAC0EBD1E4FEF5FE0BE01655E7F4F78
:10A9A0000FE010E1ABE0EA2EF12CEC0EFD1EBFEE45
:10A9B000CB2EBFE0DB2E24E030E0F50181919191B8
:10A9C000A191B1915F01FA0181939193A193B19308
:10A9D000AF01FB0181919191A191B191BF01F8016A
:10A9E00081939193A193B1938F01F70181919191FB
:10A9F000A191B1917F01F60181939193A193B193BC
:10AA00006F0121503040C9F680E090E8ABE3B5E437
:10AA10008093E70F9093E80FA093E90FB093EA0FAC
:10AA20008093E30F9093E40FA093E50FB093E60FAC
:10AA300080E090E0A0E0B0E08093EB0F9093EC0F0B
:10AA4000A093ED0FB093EE0F40E25EE460E070E0A3
:10AA500040931F1050932010609321107093221088
:10AA60008093D30F9093D40FA093D50FB093D60FAC
:10AA700080E090E0A0EAB1E48093DF0F9093E00FD4
:10AA8000A093E10FB093E20F8DEC9CECACECBEE335
:10AA90008093DB0F9093DC0FA093DD0FB093DE0F5C
:10AAA00080E090E0A0EAB0E48093D70F9093D80FB5
:10AAB000A093D90FB093DA0FEAE6F9E007C09091BE
:10AAC000C00095FFFCCF8093C60031968491882307
:10AAD000B1F7E1EEF2E006C09091C00095FFFCCF27
:10AAE0008093C60081918823B9F78091C00085FFCB
:10AAF000FCCF8AE08093C6000E94B624EA960FB687
:10AB0000F894DEBF0FBECDBFDF91CF911F910F91A3
:10AB1000FF90EF90DF90CF90BF90AF900895AF92ED
:10AB2000BF92CF92DF92EF92FF920F931F93CF933A
:10AB3000DF938C01FC0197818681981719F483813A
:10AB4000882339F081E0F801838382EE96E00E9449
:10AB5000619FF801D681EE24FF24AD2EBB24A7FC13
:10AB6000B09487E0D82E96E0C92E3FC1423009F458
:10AB700075C0433034F4442371F0413009F032C1E0
:10AB80003BC0443009F4CCC044300CF497C045308D
:10AB900009F028C1F6C0F8018381882351F082EEC4
:10ABA00096E060E04E2D0E94339F80EB91E10E9481
:10ABB000D62BF8012081332727FD30958C2F90E08C
:10ABC0002817390709F00EC18091FB0682FF0AC1E0
:10ABD0000E941E9DDC01CB018C509E4FAF4FBF4F9A
:10ABE0008093EC099093ED09A093EE09B093EF09DF
:10ABF00081E0F80181832FC0F8018381882351F01F
:10AC000082EE96E060E04E2D0E94339F8FEB91E143
:10AC10000E94D62BF8012081332727FD30958C2FF9
:10AC200090E02817390709F0DDC08091FB0682FF0C
:10AC3000D9C00E941E9DDC01CB018C509E4FAF4FAE
:10AC4000BF4F8093EC099093ED09A093EE09B09368
:10AC5000EF09F801C1820E945631C4C0F801838116
:10AC6000882351F082EE96E060E04E2D0E94339FE3
:10AC70008EEC91E10E94D62BF8012081332727FD2D
:10AC800030958C2F90E02817390709F0ABC08091E0
:10AC9000FB0682FFA7C00E941E9DDC01CB018C50E9
:10ACA0009E4FAF4FBF4F8093EC099093ED09A09357
:10ACB000EE09B093EF09F801D182CDCFF80183817D
:10ACC000882351F082EE96E060E04E2D0E94339F83
:10ACD0008DED91E10E94D62BF8012081332727FDCD
:10ACE00030958C2F90E02817390709F07BC08091B0
:10ACF000FB0682FF77C00E9456310E941E9DDC0138
:10AD0000CB018C509E4FAF4FBF4F8093EC09909377
:10AD1000ED09A093EE09B093EF090E94CD5262C0F5
:10AD2000F8018381882351F082EE96E060E04E2D99
:10AD30000E94339F8AEE91E10E94D62BF801208178
:10AD4000332727FD30958C2F90E02817390709F01D
:10AD500049C08091FB0682FF45C00E9456310E9487
:10AD60001E9DDC01CB018C509E4FAF4FBF4F809397
:10AD7000EC099093ED09A093EE09B093EF0980E000
:10AD80002FC0F8018381882351F082EE96E060E0C5
:10AD90004E2D0E94339F86EF91E10E94D62BF80141
:10ADA0002081332727FD30958C2F90E02817390715
:10ADB000C9F48091FB0682FF15C00E9456310E94A3
:10ADC0001E9DDC01CB018C509E4FAF4FBF4F809337
:10ADD000EC099093ED09A093EE09B093EF0981E09F
:10ADE0000E94DB530894E11CF11CCE2D4E2D4D0F1B
:10ADF000F8015681852F992787FD90950396970135
:10AE00002A0D3B1D821793070CF0B0CE8085882356
:10AE100009F06FC05783C091F906D091FA061382EA
:10AE2000848195819E01281B390BC90104968930C4
:10AE3000910508F05EC082EE96E060E040810E94DD
:10AE4000339F82EE96E060E20E94359EF801868193
:10AE5000D7FF06C08150868387FF48C0168246C050
:10AE6000C531D1054CF08F5FF8018683833014F033
:10AE700082E08683CFE0D0E0D093FA06C093F90653
:10AE8000F801D583C483CE0165E070E00E94FAA486
:10AE90006083643011F483E08083F8018081863020
:10AEA00014F085E08083F80197818681981711F06E
:10AEB00081E0838382EE96E060E0F80140810E94A9
:10AEC000339FF8018081992787FD9095268133274C
:10AED00027FD3095820F931F009711F06EE301C09C
:10AEE00063E082EE96E00E94359E03C0C4E0D0E0AD
:10AEF000C3CFDF91CF911F910F91FF90EF90DF9023
:10AF0000CF90BF90AF900895CF92DF92EF92FF92D3
:10AF1000CF93DF93EC0189B1992787FD90958095B8
:10AF200090958827990F881F99272091060A30E06D
:10AF300082179307C1F081E08B8389B18095881FC8
:10AF40008827881F8093060A82E297E04F9905C000
:10AF50000E94E07C80E792E104C00E94C37D8EE7FE
:10AF600092E10E94022C898190912904891749F06D
:10AF700091E09B831092FA061092F9061E8280934C
:10AF800029042091F9063091FA068C819D812817B9
:10AF9000390721F48091FB0682FF10C00E941E9D9C
:10AFA000DC01CB018856954CAF4FBF4F8093070A09
:10AFB0009093080AA093090AB0930A0A8981833002
:10AFC00009F44FC0843028F48130D9F18230F0F593
:10AFD0000DC0853009F455C0853008F446C0863070
:10AFE00009F44BC0873009F04FC043C0CE010E9426
:10AFF0003E508091FB0682FF47C018860E941E9D2E
:10B00000DC01CB018C509E4FAF4FBF4F8093EC09BA
:10B010009093ED09A093EE09B093EF0981E0898345
:10B020000E941E9DDC01CB018856954CAF4FBF4F4F
:10B030008093070A9093080AA093090AB0930A0A1A
:10B0400023C0CE010E946C3718861EC089858823D4
:10B0500021F0CE010E946F3917C0CE010E94083244
:10B0600013C0CE010E94904D0FC0CE010E948F559B
:10B070000BC0CE010E94FB4307C0CE010E940A3ED6
:10B0800003C0CE010E94E734C090070AD090080A9E
:10B09000E090090AF0900A0A0E941E9DDC01CB0193
:10B0A000C816D906EA06FB0608F419828091F9064B
:10B0B0009091FA069D838C83DF91CF91FF90EF9062
:10B0C000DF90CF900895CF92DF92EF92FF920E948F
:10B0D0001E9D6B017C014091EC095091ED0960913E
:10B0E000EE097091EF0980E090E0E1E0F0E0C41635
:10B0F000D506E606F7066CF4A091FB069F01082E24
:10B1000002C0220F331F0A94E2F720952A232093CE
:10B11000FB0601968830910551F79091FB068091CE
:10B12000F0099817A9F40E941E9DDC01CB01409103
:10B13000F1095091F2096091F3097091F409841BAF
:10B14000950BA60BB70B84369105A105B105A0F0B0
:10B150008091FB068093F0090E941E9DDC01CB01CB
:10B160008093F1099093F209A093F309B093F40945
:10B1700085EF99E00E948457FF90EF90DF90CF9089
:10B1800008952F923F924F925F926F927F928F928B
:10B190009F92AF92BF92CF92DF92EF92FF920F9366
:10B1A0001F93CF93DF93CDB7DEB7A2970FB6F89476
:10B1B000DEBF0FBECDBF87E40E944429882309F477
:10B1C000E7C50E9428290E949BA16430710509F4FB
:10B1D00041C06530710554F46230710541F163304E
:10B1E00071056CF577FF19C00C94876A6A35710593
:10B1F00009F464C56B35710534F46C31710511F0D7
:10B200000C94876A72C06B35710509F45BC56C35A7
:10B21000710511F00C94876A5AC58091FC06882349
:10B2200031F40E94BA290E94722A0C94B06A80916B
:10B23000FC06882321F40E94432A81E007C0809104
:10B24000FC06882339F40E94432A80E00E94142BD4
:10B250000C94B06A81E89DE00E94022C80E50E9477
:10B260004429882339F00E9428290E94A0A16B015B
:10B270007C0103C0CC24DD24760183E50E944429AF
:10B28000882361F00E94282920E030E04AE754E456
:10B290000E9401A40E94A0A16B017C010E942916BA
:10B2A0000E941E9D4B015C018C0C9D1CAE1CBF1CA2
:10B2B0000E941E9DDC01CB018093A6099093A709F3
:10B2C000A093A809B093A90905C00E94EF6D81E081
:10B2D0000E94882C0E941E9DDC01CB0188159905D7
:10B2E000AA05BB0590F30C94876A80911C04909189
:10B2F0001D04A0911E04B0911F048093AA0990938D
:10B30000AB09A093AC09B093AD0980910A04909168
:10B310000B0490931D0780931C0784E690E09093A4
:10B320000B0480930A040E941E9DDC01CB018093D4
:10B33000A6099093A709A093A809B093A90981E051
:10B340000E94EB0E80910B0790910C07A0910D07C6
:10B35000B0910E078093AE099093AF09A093B00906
:10B36000B093B10980910F0790911007A091110738
:10B37000B09112078093B2099093B309A093B409D6
:10B38000B093B5098091130790911407A091150708
:10B39000B09116078093B6099093B709A093B809A6
:10B3A000B093B9098091170790911807A0911907D8
:10B3B000B0911A078093BA099093BB09A093BC0976
:10B3C000B093BD0980E090E0A0E0B0E080931C0461
:10B3D00090931D04A0931E04B0931F0488E50E945F
:10B3E0004429882361F489E50E944429882339F49B
:10B3F0008AE50E944429882311F481E001C080E09D
:10B400008093200488E50E944429882309F4E8C039
:10B4100089E50E944429882309F4E2C080E090E095
:10B42000A0E0B0E080930B0790930C07A0930D076A
:10B43000B0930E0780930F0790931007A093110706
:10B44000B09312078BE097E06FE077E043E157E0BD
:10B4500027E137E00E94CC9880E090ECA9E9B3ECBA
:10B460008093AE099093AF09A093B009B093B1094E
:10B470008093B2099093B309A093B409B093B5092E
:10B4800020910C0430910D0440910E0450910F0452
:10B4900020931C0430931D0440931E0450931F04FA
:10B4A000C0901004D0901104E0901204F0901304A6
:10B4B000C701B6010E942CA187FF08C0C0921C04DE
:10B4C000D0921D04E0921E04F0921F0460911C04AF
:10B4D00070911D0480911E0490911F0420E030E0C3
:10B4E00040E752E40E9433A17B018C018EEA99E08F
:10B4F00062EB79E046EB59E02AEB39E0FEEFCF2E24
:10B50000F6E0DF2E0E946D8D0E9429160F2EF0E0CE
:10B510008F2EF0E09F2EF0E0AF2EF0E0BF2EF02D4A
:10B5200080920B0790920C07A0920D07B0920E0725
:10B5300080920F0790921007A0921107B092120705
:10B540008BE097E06FE077E043E157E027E137E0F9
:10B550000E94CC9880910B0790910C07A0910D0749
:10B56000B0910E078093AE099093AF09A093B009F4
:10B57000B093B10980910F0790911007A091110726
:10B58000B09112078093B2099093B309A093B409C4
:10B59000B093B50960911C0470911D0480911E0444
:10B5A00090911F0420E030E040E752E40E9433A174
:10B5B0007B018C018EEA99E062EB79E046EB59E081
:10B5C0002AEB39E00E946D8D80921C0490921D043C
:10B5D000A0921E04B0921F040E9429160E94E40E3D
:10B5E00080912004882331F488E50E94442988232F
:10B5F00009F4E7C00F2EF0E08F2EF0E09F2EF0E070
:10B60000AF2EF0E0BF2EF02D80920B0790920C072A
:10B61000A0920D07B0920E078BE097E06FE077E005
:10B6200043E157E027E137E00E94CC9880E090ECBE
:10B63000A9E9B3EC8093AE099093AF09A093B00948
:10B64000B093B10960910C0470910D0480910E04C7
:10B6500090910F0460931C0470931D0480931E044A
:10B6600090931F0420E030E040E752E40E9433A1B1
:10B670007B018C018EEA99E062EB79E046EB59E0C0
:10B680002AEB39E0EEEFCE2EE6E0DE2E0E946D8D45
:10B690000E94291680920B0790920C07A0920D072A
:10B6A000B0920E078BE097E06FE077E043E157E060
:10B6B00027E137E00E94CC9880E090E0A0EAB0E477
:10B6C0008093AE099093AF09A093B009B093B109EC
:10B6D00060911C0470911D0480911E0490911F04C0
:10B6E00020E030E040E752E40E9433A17B018C016E
:10B6F0008EEA99E062EB79E046EB59E02AEB39E01B
:10B700000E946D8D0E94291680E090E0A0E2B1ECCD
:10B710008093AE099093AF09A093B009B093B1099B
:10B7200060910C0470910D0480910E0490910F04AF
:10B7300020E030E040E05FE30E9401A49B01F82F8D
:10B74000E92F462F532F682F792F40931C045093D5
:10B750001D0460931E0470931F04822F932FAF2F3C
:10B76000BE2FBC01CD0120E030E040E752E40E9452
:10B7700033A17B018C018EEA99E062EB79E046EB24
:10B7800059E02AEB39E00E946D8D0E9429168092C3
:10B790000B0790920C07A0920D07B0920E078092B3
:10B7A000AE099092AF09A092B009B092B10980920F
:10B7B0001C0490921D04A0921E04B0921F040E94CB
:10B7C000E40E80912004882331F489E50E94442905
:10B7D000882309F4E7C00F2EF0E08F2EF0E09F2EB3
:10B7E000F0E0AF2EF0E0BF2EF02D80920F07909288
:10B7F0001007A0921107B09212078BE097E06FE05C
:10B8000077E043E157E027E137E00E94CC9880E001
:10B8100090ECA9E9B3EC8093B2099093B309A0939B
:10B82000B409B093B509609110047091110480912E
:10B8300012049091130460931C0470931D04809370
:10B840001E0490931F0420E030E040E752E40E9481
:10B8500033A17B018C018EEA99E062EB79E046EB43
:10B8600059E02AEB39E0FEEFCF2EF6E0DF2E0E9402
:10B870006D8D0E94291680920F0790921007A0925A
:10B880001107B09212078BE097E06FE077E043E199
:10B8900057E027E137E00E94CC9880E090E0A0EAF2
:10B8A000B0E48093B2099093B309A093B409B09324
:10B8B000B50960911C0470911D0480911E04909143
:10B8C0001F0420E030E040E752E40E9433A17B01F6
:10B8D0008C018EEA99E062EB79E046EB59E02AEBC5
:10B8E00039E00E946D8D0E94291680E090E0A0E270
:10B8F000B1EC8093B2099093B309A093B409B093CB
:10B90000B509609110047091110480911204909116
:10B91000130420E030E040E05FE30E9401A49B01BB
:10B92000F82FE92F462F532F682F792F40931C04AF
:10B9300050931D0460931E0470931F04822F932F55
:10B94000AF2FBE2FBC01CD0120E030E040E752E434
:10B950000E9433A17B018C018EEA99E062EB79E0D1
:10B9600046EB59E02AEB39E00E946D8D0E942916C2
:10B9700080920F0790921007A0921107B0921207C1
:10B980008092B2099092B309A092B409B092B5091D
:10B9900080921C0490921D04A0921E04B0921F0479
:10B9A0000E94E40E80912004882331F48AE50E94ED
:10B9B0004429882309F4E7C00F2EF0E08F2EF0E031
:10B9C0009F2EF0E0AF2EF0E0BF2EF02D80921307F7
:10B9D00090921407A0921507B09216078BE097E09B
:10B9E0006FE077E043E157E027E137E00E94CC9831
:10B9F00080E090E0A6E9B3EC8093B6099093B70994
:10BA0000A093B809B093B90960911404709115041A
:10BA1000809116049091170460931C0470931D0488
:10BA200080931E0490931F0420E030E040E752E42E
:10BA30000E9433A17B018C018EEA99E062EB79E0F0
:10BA400046EB59E02AEB39E0EEEFCE2EE6E0DE2EB3
:10BA50000E946D8D0E942916809213079092140700
:10BA6000A0921507B09216078BE097E06FE077E0A1
:10BA700043E157E027E137E00E94CC9880E090E076
:10BA8000A0E8BFE38093B6099093B709A093B809E3
:10BA9000B093B90960911C0470911D0480911E043B
:10BAA00090911F0420E030E040E752E40E9433A16F
:10BAB0007B018C018EEA99E062EB79E046EB59E07C
:10BAC0002AEB39E00E946D8D0E94291680E090E0FB
:10BAD000A0E0B0EC8093B6099093B709A093B809A1
:10BAE000B093B90960911404709115048091160403
:10BAF0009091170420E030E040E05FE30E9401A451
:10BB00009B01F82FE92F462F532F682F792F409351
:10BB10001C0450931D0460931E0470931F04822F15
:10BB2000932FAF2FBE2FBC01CD0120E030E040E7C6
:10BB300052E40E9433A17B018C018EEA99E062EB12
:10BB400079E046EB59E02AEB39E00E946D8D0E94C6
:10BB500029168092130790921407A0921507B092AD
:10BB600016078092B6099092B709A092B809B092D0
:10BB7000B90980921C0490921D04A0921E04B092F8
:10BB80001F040E94E40E88E50E9444298823F1F0F6
:10BB90000E943829DC01CB010097A105B105B1F065
:10BBA0000E9428292091FF0630910007409101074B
:10BBB000509102070E9453A0DC01CB0180930B0738
:10BBC00090930C07A0930D07B0930E0789E50E9490
:10BBD00044298823F1F00E943829DC01CB01009729
:10BBE000A105B105B1F00E942829209103073091E9
:10BBF000040740910507509106070E9453A0DC01FD
:10BC0000CB0180930F0790931007A0931107B09377
:10BC100012078AE50E9444298823F1F00E943829FE
:10BC2000DC01CB010097A105B105B1F00E942829E4
:10BC300020910707309108074091090750910A07A2
:10BC40000E9453A0DC01CB0180931307909314074B
:10BC5000A0931507B09316078BE097E06FE077E0AD
:10BC600043E157E027E137E00E94CC988091AA0990
:10BC70009091AB09A091AC09B091AD0980931C04DF
:10BC800090931D04A0931E04B0931F0480911C0781
:10BC900090911D0790930B0480930A040E941E9DAF
:10BCA000DC01CB018093A6099093A709A093A80972
:10BCB000B093A9090E94E40E0C94876A1092BE0901
:10BCC0000C94876A81E08093BE090C94876A85E4AE
:10BCD0000E944429882311F40E94291635E4832EFA
:10BCE00034E0932E4FEFC42E46E0D42E5BE0E52ED9
:10BCF00057E0F52E00E0F40181914F010E944429A4
:10BD00008823D1F10E942829F601208131814281C6
:10BD100053810E9453A0DC01CB01F7018083918302
:10BD2000A283B383033071F40E942829DC01CB0184
:10BD3000F70180839183A283B38387E197E00E9418
:10BD40007C991AC00E942829F60120813181428104
:10BD500053810E9453A0DC01CB01F70180839183C2
:10BD6000A283B3838BE097E06FE077E043E157E095
:10BD700027E137E00E94CC980F5F24E030E0C20E4C
:10BD8000D31EE20EF31E043009F0B5CF0C94876A7F
:10BD90008DE40E944429882311F40C94D9690E94EF
:10BDA00028290E949BA16A36710509F448C66B36A2
:10BDB00071050CF081C06E31710509F4ECC16F3171
:10BDC0007105ECF56731710509F458C168317105E9
:10BDD000DCF46431710509F41AC16531710554F45C
:10BDE0006131710509F409C16231710511F00C94DA
:10BDF000876A5FC66531710509F434C16631710522
:10BE000011F00C94876A34C16A31710509F463C179
:10BE10006B31710554F46831710509F444C169311D
:10BE2000710511F00C94876A50C16B31710509F4EA
:10BE300074C16C31710511F00C94876A74C163355B
:10BE4000710509F432C664357105DCF4603571059D
:10BE500009F420C66135710554F46F31710509F498
:10BE6000DBC16A32710511F00C94876A4AC26135F0
:10BE7000710509F412C66235710511F00C94876AD8
:10BE800011C66C35710509F479C66D35710554F428
:10BE90006435710509F40DC66535710511F00C9412
:10BEA000876A54C66836710509F473C2693671052C
:10BEB00011F00C94876AE4C26D3C710511F40C9486
:10BEC00012686E3C71050CF040C06737710509F4CB
:10BED0006FC768377105DCF46237710509F48CC6E9
:10BEE0006337710554F46B36710509F4D0C56D36AE
:10BEF000710511F00C94876A59C36337710509F411
:10BF00005BC66537710511F00C94876A63C6693C9E
:10BF1000710511F40C9492676A3C710554F46C3805
:10BF2000710509F498C26E3B710511F00C94876A93
:10BF3000DAC46B3C710511F40C94D0676C3C71054C
:10BF400011F00C94876A0C94EE6731E06F3273073E
:10BF500011F40C94A66981E06033780714F56D3D07
:10BF6000710511F40C94AE686E3D710564F46E3C7D
:10BF7000710511F40C947C686C3D710511F00C9402
:10BF8000876A0C949A6891E06D32790711F40C94E9
:10BF9000BF68E1E06E327E0711F00C94876A0C9462
:10BFA000A269F1E0653F7F0711F40C94BB6921E0C1
:10BFB000663F720774F431E06039730711F40C9432
:10BFC000B56981E0643F780711F00C94876A0C949E
:10BFD000B86991E0673F790711F40C94C169E1E019
:10BFE000673F7E0714F40C94BD69F3E0673E7F075A
:10BFF00011F00C94876A0C94C4698AE89DE00E9451
:10C00000022C159817984298A0980C94876AE3E937
:10C01000FDE007C09091C00095FFFCCF8093C60063
:10C02000319684918823B1F78091C00085FFFCCFC1
:10C030008AE08093C60082E297E00E949D7CE3EA5A
:10C04000FDE007C09091C00095FFFCCF8093C60033
:10C05000319684918823B1F78091C00085FFFCCF91
:10C060000C94846A82E297E00E94E07C0C94876AD8
:10C0700082E297E00E94C37D0C94876A0091940944
:10C08000109195090C5F1F4FC8016AE270E00E9491
:10C0900055A8009719F00197FC01108282E297E001
:10C0A000B80141E074C082E297E00E94C77D0E941F
:10C0B0001E9DDC01CB018093A2099093A309A0935C
:10C0C000A409B093A5090C94876A82E297E00E94C4
:10C0D000CE7D0C94876A80912407882311F40C94F8
:10C0E000876A83E50E944429882311F40C94876AA7
:10C0F0000E943829AB01382F292F6093FC075093F9
:10C10000FD078093FE079093FF0789ED97E0632F6B
:10C11000722F0E94351A0C94876A82E297E00E947F
:10C1200010810C94876A80919409909195090496E6
:10C130006AE270E00E9455A88C010097F9F0209106
:10C140008E0930918F0940E650E0249FC001259F61
:10C15000900D349F900D1124865F974F6EE470E030
:10C160000E9455A860E270E00E9455A80196909345
:10C17000950980939409F801319710826091940990
:10C18000709195096C5F7F4F82E297E040E00E94DA
:10C19000D37D0C94876A80912407882311F40C9432
:10C1A000876A82E297E00E94E882809194099091E8
:10C1B000950904966AE270E00E9455A88C010097E8
:10C1C000F9F020918E0930918F0940E650E0249FCC
:10C1D000C001259F900D349F900D1124865F974FCD
:10C1E0006EE470E00E9455A860E270E00E9455A8DD
:10C1F00001969093950980939409F80131971082E4
:10C2000060919409709195096C5F7F4F82E297E08D
:10C210000E94CC7F0C94876A0E941E9DDC01CB019A
:10C2200080939E0990939F09A093A009B093A109C0
:10C230004091A2095091A3096091A4097091A509A8
:10C24000841B950BA60BB70BBC01CD0128EE33E088
:10C2500040E050E00E940DA58DB79EB708970FB63D
:10C26000F8949EBF0FBE8DBF0DB71EB70F5F1F4F57
:10C27000CE010196EDB7FEB79283818389E192E00A
:10C28000F80193838283CA01B9012CE330E040E0D6
:10C2900050E00E940DA5DC01CB01F8013583248319
:10C2A000978386830E949EA8EAE6F9E084912DB7E1
:10C2B0003EB7285F3F4F0FB6F8943EBF0FBE2DBF6D
:10C2C00008C09091C00095FFFCCF8093C6003196C6
:10C2D00084918823B1F7FE01319606C09091C00089
:10C2E00095FFFCCF8093C60081918823B9F7809198
:10C2F000C00085FFFCCF8AE08093C600CE01019686
:10C3000078C483E50E944429882311F40C94876A39
:10C310000E9428296B017C0180E50E944429882322
:10C3200011F40C94876AC701B6010E949BA1DC013D
:10C33000CB017C0197FF02C00C94876A8F3F910567
:10C3400019F014F00C94876A0E9428290E949BA17E
:10C350008B019C01E9E4F4E020E081919191801748
:10C36000910711F40C94876A2F5F2A33B1F717FFF6
:10C3700002C00C94876A802F61E00E947C9C802F11
:10C380006E2D0E949D9C802FB7010E942C9B0C94C7
:10C39000876A8091FE068093BF0984E50E94442944
:10C3A000882379F10E9428290E94A0A16093BF09E7
:10C3B000662339F1EAE6F9E007C09091C00095FFE5
:10C3C000FCCF8093C600319684918823B1F7EFE2C9
:10C3D000F3E006C09091C00095FFFCCF8093C600AB
:10C3E00081918823B9F78BE59AE06091BF0940E01D
:10C3F00050E00E9456798091C00085FFFCCF0C94DC
:10C40000846A83E50E944429882309F10E9428292F
:10C410006B017C010091BF09802E99240E949BA191
:10C42000DC01CB01602F0E94536DF401EE0FFF1F62
:10C43000E25EF54F91838083F401EE0FFF1FEE0F54
:10C44000FF1FEC5EF54FC082D182E282F3820E9430
:10C4500070700C94876A83E50E944429882311F444
:10C460000C94876A0E9428290E949BA1DC01CB01C1
:10C470000E949B6D90931D0A80931C0A0C94876AFE
:10C480008091FE068093BF0984E50E944429882399
:10C4900079F10E9428290E94A0A16093BF09662318
:10C4A00039F1EAE6F9E007C09091C00095FFFCCFB2
:10C4B0008093C600319684918823B1F7E6E4F3E0D7
:10C4C00006C09091C00095FFFCCF8093C60081917B
:10C4D0008823B9F78BE59AE06091BF0940E050E00E
:10C4E0000E9456798091C00085FFFCCF0C94846A2D
:10C4F000E1EBFDE007C09091C00095FFFCCF809379
:10C50000C600319684918823B1F76091BF09E62F68
:10C51000F0E0EE0FFF1FE65EF54F808191810E94F3
:10C520009E6DAB01BC018BE59AE022E030E00E94F9
:10C530008F7AE7EBFDE007C09091C00095FFFCCF3C
:10C540008093C600319684918823B1F78091180AB0
:10C550009091190A0E940E70AB01BC018BE59AE024
:10C5600022E030E00E948F7AEBEBFDE007C0909173
:10C57000C00095FFFCCF8093C6003196849188233C
:10C58000B1F78091BF0990E00E944D6DBC018BE531
:10C590009AE04AE050E00E9493798091C00085FFC4
:10C5A000FCCF8AE08093C6000C94B06A8091FE06AE
:10C5B0008093BF0984E50E944429882371F10E9479
:10C5C00028290E94A0A16093BF09662331F1EAE601
:10C5D000F9E007C09091C00095FFFCCF8093C600A2
:10C5E000319684918823B1F7EDE5F3E006C0909190
:10C5F000C00095FFFCCF8093C60081918823B9F7D6
:10C600008BE59AE06091BF0940E050E00E945679C6
:10C610008091C00085FFFCCF77C78FEB9DE00E9423
:10C62000022C83E50E944429882309F10E942829CD
:10C630006B017C010091BF09802E99240E949BA16F
:10C64000DC01CB01602F0E94536DF401EE0FFF1F40
:10C65000E25EF54F91838083F401EE0FFF1FEE0F32
:10C66000FF1FEC5EF54FC082D182E282F3820E940E
:10C6700070700E941E9D2B013C018091BF0990E0CB
:10C68000880F991FFC01E25EF54F2081318138A3AC
:10C690002F8F865E954FFC010190F081E02DFAA36B
:10C6A000E9A388248A94982C5401EAECFDE03490A4
:10C6B000EDECFDE02490E1EDFDE004911AE001C114
:10C6C000832DEAECFDE008C09091C00095FFFCCFFF
:10C6D0008093C600319684918823B1F76091BF0999
:10C6E000E62FF0E0EE0FFF1FE65EF54F80819181AF
:10C6F0000E949E6DAB01BC018BE59AE022E030E028
:10C700000E948F7A822DEDECFDE008C09091C00070
:10C7100095FFFCCF8093C600319684918823B1F7B2
:10C720006091BF098BE59AE070E04AE050E00E941A
:10C730009379802FE1EDFDE008C09091C00095FF56
:10C74000FCCF8093C600319684918823B1F7B7FE61
:10C7500003C0E4E7F3E029C00E941E9DAB01BC01C9
:10C76000D501C40188579C4EAF4FBF4F841B950B1A
:10C77000A60BB70BBC01CD0128EE33E040E050E042
:10C780000E940DA58BE59AE0BA01A9012AE030E0EC
:10C790000E9449798091C00085FFFCCF0DC0909127
:10C7A000C00095FFFCCF8093C60081918823B9F724
:10C7B0008091C00085FFFCCF1093C6000E941E9D93
:10C7C0002B013C010E94EF6D81E00E94882C0E94A9
:10C7D0006358FFEF8F16FFEF9F06FFEFAF06FFEFE7
:10C7E000BF0619F5A091BF092F8D38A189A19AA183
:10C7F000B0E0AA0FBB1FFD01E25EF54FA65EB54F8C
:10C80000821793074CF4808191812D913C9111976F
:10C8100028173907F4F541C0808191812D913C9111
:10C82000119782179307ACF538C0B7FC36C06091FA
:10C83000BF09E62FF0E0EE0FFF1FE65EF54F8081A7
:10C8400091810E949E6D6B017C016091BF09E62F72
:10C85000F0E0EE0FFF1FE25EF54F808191810E94B4
:10C860009E6D9B01AC01C701B6010E9452A00E94BF
:10C870009BA1AB01BC0177FF07C0709560955095F7
:10C8800041955F4F6F4F7F4F4430510561057105F2
:10C8900024F00E941E9D4B015C019FEF89169FEFC3
:10C8A00099069FEFA9069FEFB90659F0B7FC32C66B
:10C8B0000E941E9D68197909E3E168387E0708F037
:10C8C00029C60E941E9DDC01CB0184199509A60989
:10C8D000B709893EF3E09F07F0E0AF07F0E0BF073C
:10C8E00008F0EECE6FCF83EE9DE00E94022C83E530
:10C8F0000E944429882361F00E9428290E949BA15C
:10C90000DC01CB010E949B6D90931D0A80931C0A51
:10C910000E941E9D6B017C01E0EFFDE0B490E3EF0F
:10C92000FDE08490E7EFFDE004911AE077C00E94FB
:10C930001E9DDC01CB018C199D09AE09BF09893E02
:10C9400023E0920720E0A20720E0B20708F45FC0CE
:10C950006091FE06E62FF0E0EE0FFF1FE65EF54F5A
:10C96000808191810E949E6DAB01BC018B2DE0EF17
:10C97000FDE008C09091C00095FFFCCF8093C600F9
:10C98000319684918823B1F78BE59AE022E030E07C
:10C990000E948F7A882DE3EFFDE008C09091C000DF
:10C9A00095FFFCCF8093C600319684918823B1F720
:10C9B0006091FE068BE59AE070E04AE050E00E944C
:10C9C0009379802FE7EFFDE008C09091C00095FFBC
:10C9D000FCCF8093C600319684918823B1F7809173
:10C9E000180A9091190A0E940E70AB01BC018BE5E8
:10C9F0009AE022E030E00E948F7A8091C00085FFAB
:10CA0000FCCF1093C6000E941E9D6B017C010E940A
:10CA1000EF6D81E00E94882C0E94635820911C0ACF
:10CA200030911D0A8091180A9091190A8217930774
:10CA30000CF47DCF8BEF9DE00E94022C7BC583E53B
:10CA40000E9444298823F9F00E94282920E030E040
:10CA500040E050E00E942CA187FD0FC00E942829D1
:10CA600020E030E04FE753E40E942FA318163CF07B
:10CA70000E9428290E94A0A103C060E001C06FEFBE
:10CA80006093FD0644C58FEF8093FD0640C510926C
:10CA9000FD063DC5269A2E983AC50E9429160E9489
:10CAA000252935C51092210732C581E080932107E1
:10CAB0002EC583E50E9444298823A9F00E942829D5
:10CAC00020E030E04AE754E40E9401A40E94A0A1C3
:10CAD000DC01CB018093210490932204A0932304D2
:10CAE000B093240414C588E50E944429882309F0E2
:10CAF0002EC589E50E944429882309F028C58AE5C6
:10CB00000E944429882309F022C585E40E94442913
:10CB1000882309F01CC50E942916A09A0E949B1622
:10CB2000F6C4159A89E50E9444298111179A8AE56D
:10CB30000E9444298111429A85E40E94442981116E
:10CB4000A09A85E09EE00E94022CE1C483E50E9449
:10CB500044290E94282920E030E04AE754E40E945A
:10CB600001A40E94A0A1DC01CB018093C009909395
:10CB7000C109A093C209B093C309C9C445E4C42E36
:10CB800044E0D42E0FEF1FE0EE24F60181916F01F7
:10CB90000E944429882349F00E942829DC01CB0106
:10CBA000F80180839183A283B383E3940C5F1F4FCA
:10CBB000F4E0EF1651F7ABC4E5E1FEE007C0909159
:10CBC000C00095FFFCCF8093C600319684918823E6
:10CBD000B1F79DC440918E0950918F0920E630E055
:10CBE000429FC001439F900D529F900D1124815F81
:10CBF000974F0E94E62B8BC4E0EBFEE007C09091BC
:10CC0000C00095FFFCCF8093C600319684918823A5
:10CC1000B1F740910B0750910C0760910D0770918F
:10CC20000E078BE59AE022E030E00E948F7AE3EB7A
:10CC3000FEE007C09091C00095FFFCCF8093C60036
:10CC4000319684918823B1F740910F0750911007D6
:10CC500060911107709112078BE59AE022E030E0B5
:10CC60000E948F7AE6EBFEE007C09091C00095FF2E
:10CC7000FCCF8093C600319684918823B1F7409110
:10CC800013075091140760911507709116078BE5F3
:10CC90009AE022E030E00E948F7AE9EBFEE007C0E4
:10CCA0009091C00095FFFCCF8093C600319684918F
:10CCB0008823B1F740911707509118076091190721
:10CCC00070911A078BE59AE022E030E00E948F7A9B
:10CCD000ECEBFEE007C09091C00095FFFCCF809385
:10CCE000C600319684918823B1F70E9485160E9470
:10CCF000CEA12091FF0F3091001040910110509172
:10CD000002100E9433A1AB01BC018BE59AE022E046
:10CD100030E00E948F7AE6ECFEE007C09091C00000
:10CD200095FFFCCF8093C600319684918823B1F79C
:10CD300081E00E9485160E94CEA1209103103091BF
:10CD4000041040910510509106100E9433A1AB01D0
:10CD5000BC018BE59AE022E030E00E948F7AE9EC9A
:10CD6000FEE007C09091C00095FFFCCF8093C60005
:10CD7000319684918823B1F782E00E9485160E9443
:10CD8000CEA12091071030910810409109105091C8
:10CD90000A100E9433A1AB01BC018BE59AE022E0AE
:10CDA00030E00E948F7A8091C00085FFFCCFACC339
:10CDB000ECECFEE007C09091C00095FFFCCF8093A3
:10CDC000C600319684918823B1F780B180FD03C0FD
:10CDD000E9E2F3E009C0ECE2F3E006C09091C000A4
:10CDE00095FFFCCF8093C60081918823B9F7E3EDCE
:10CDF000FEE007C09091C00095FFFCCF8093C60075
:10CE0000319684918823B1F7029903C0E9E2F3E0F7
:10CE100009C0ECE2F3E006C09091C00095FFFCCFA2
:10CE20008093C60081918823B9F7EAEDFEE007C040
:10CE30009091C00095FFFCCF8093C60031968491FD
:10CE40008823B1F7049903C0E9E2F3E009C0ECE2FA
:10CE5000F3E006C09091C00095FFFCCF8093C60020
:10CE600081918823B9F7E1EEFEE007C09091C00000
:10CE700095FFFCCF8093C600319684918823B1F74B
:10CE8000069903C0E9E2F3E009C0ECE2F3E006C072
:10CE90009091C00095FFFCCF8093C60081918823BC
:10CEA000B9F7E8EEFEE007C09091C00095FFFCCF17
:10CEB0008093C600319684918823B1F7379903C0D7
:10CEC000E9E2F3E009C0ECE2F3E006C09091C000B3
:10CED00095FFFCCF8093C60081918823B9F7EFEED0
:10CEE000FEE007C09091C00095FFFCCF8093C60084
:10CEF000319684918823B1F7359903C0E9E2F3E0D4
:10CF000009C0ECE2F3E006C09091C00095FFFCCFB1
:10CF10008093C60081918823B9F78091C00085FF76
:10CF2000FCCFF2C235E4C32E34E0D32E00E010E093
:10CF3000F60181916F010E944429882359F10E94D2
:10CF40002829EFEEEE2EEFE0FE2EE00EF11E0E94FD
:10CF5000A0A1DC01CB01F70180839183A283B3837D
:10CF60000E94282923ECE22E2FE0F22EE00EF11E83
:10CF7000F801E150F04F20813181428153810E94BC
:10CF800001A40E94A0A1DC01CB01F7018083918361
:10CF9000A283B3830C5F1F4F0031110549F6B7C25E
:10CFA00055E4C52E54E0D52E0FE010E164E0E62EE6
:10CFB000F60181916F010E944429882349F00E9463
:10CFC0002829DC01CB01F80180839183A283B383FC
:10CFD000EA940C5F1F4FEE2059F799C283E50E9437
:10CFE0004429882361F00E942829DC01CB01809329
:10CFF000E70F9093E80FA093E90FB093EA0F84E551
:10D000000E944429882309F482C20E942829DC0155
:10D01000CB018093E30F9093E40FA093E50FB093BF
:10D02000E60F75C283E50E944429882361F00E94BF
:10D030002829DC01CB018093EB0F9093EC0FA09398
:10D04000ED0FB093EE0F84E50E944429882361F030
:10D050000E942829DC01CB018093D30F9093D40F39
:10D06000A093D50FB093D60F82E40E944429882361
:10D0700071F00E9428290E94A0A1DC01CB018093BD
:10D080001F1090932010A0932110B093221088E5D8
:10D090000E944429882361F00E942829DC01CB01E9
:10D0A0008093DF0F9093E00FA093E10FB093E20F16
:10D0B0008AE50E944429882361F00E942829DC0126
:10D0C000CB018093DB0F9093DC0FA093DD0FB09327
:10D0D000DE0F85E40E944429882309F418C20E94C7
:10D0E0002829DC01CB018093D70F9093D80FA09310
:10D0F000D90FB093DA0F0BC235E4C32E34E0D32E30
:10D100000FEF16E043E0E42EF60181916F010E94DB
:10D110004429882349F00E942829DC01CB01F80129
:10D1200080839183A283B383EA940C5F1F4FEE2028
:10D1300059F7EDC183E50E944429882309F4E7C12A
:10D140000E9428290E949BA1DC01CB0190930B0433
:10D1500080930A0481E080931B07D9C183E50E9474
:10D160004429882309F4D3C10E9428290E949BA145
:10D17000DC01CB019093090480930804C8C180E5C9
:10D180000E944429882361F00E942829DC01CB01F8
:10D190008093360490933704A0933804B0933904F5
:10D1A00089E40E944429882391F00E9428292FE6CF
:10D1B00032E143E05EE30E9401A4DC01CB018093F5
:10D1C000320490933304A0933404B093350484E480
:10D1D0000E944429882391F00E9428292FE632E1F9
:10D1E00043E05EE30E9433A1DC01CB0180932E0477
:10D1F00090932F04A0933004B093310483E40E94F1
:10D200004429882361F00E942829DC01CB01809306
:10D210002A0490932B04A0932C04B0932D040E9415
:10D22000346DE6E7F3E006C09091C00095FFFCCFB7
:10D230008093C60081918823B9F7E9E7F3E006C03F
:10D240009091C00095FFFCCF8093C6008191882308
:10D25000B9F74091360450913704609138047091C9
:10D2600039048BE59AE022E030E00E948F7AEDE706
:10D27000F3E006C09091C00095FFFCCF8093C600FC
:10D2800081918823B9F760913204709133048091C1
:10D290003404909135042FE632E143E05EE30E94CE
:10D2A00033A1AB01BC018BE59AE022E030E00E94A3
:10D2B0008F7AE1E8F3E006C09091C00095FFFCCFC3
:10D2C0008093C60081918823B9F760912E047091F4
:10D2D0002F0480913004909131042FE632E143E035
:10D2E0005EE30E9401A4AB01BC018BE59AE022E061
:10D2F00030E00E948F7AE5E8F3E006C09091C0002C
:10D3000095FFFCCF8093C60081918823B9F7609187
:10D310002A0470912B0480912C0490912D042FE607
:10D3200032E143E05EE30E9401A4AB01BC018BE566
:10D330009AE022E030E00E948F7A8091C00085FF61
:10D34000FCCFE2C081E00E94A199E1C083E50E9488
:10D350004429882319F00E94282904C060E070E065
:10D3600086E193E40E94A370D2C00E942916CFC028
:10D370000E94CD52CCC080E001C081E00E94DB530E
:10D38000C6C00E94B624C3C01092FC068091C40996
:10D390009091C509A091C609B091C70980939A09D7
:10D3A00090939B09A0939C09B0939D090E948D299D
:10D3B000AEC084E50E944429882309F461C00E941C
:10D3C00028290E94A0A16093BF09EAE6F9E066233C
:10D3D00081F107C09091C00095FFFCCF8093C600FB
:10D3E000319684918823B1F7E9E8F3E006C0909183
:10D3F000C00095FFFCCF8093C60081918823B9F7C8
:10D400008BE59AE06091BF0940E050E00E945679B8
:10D41000EBE8F3E006C09091C00095FFFCCF80934D
:10D42000C60081918823B9F78091C00085FFFCCFA9
:10D430006BC01092FE0607C09091C00095FFFCCF14
:10D440008093C600319684918823B1F7ECE9F3E02C
:10D4500006C09091C00095FFFCCF8093C6008191DB
:10D460008823B9F76091FE068BE59AE070E04AE008
:10D4700050E00E9493798091C00085FFFCCF44C0AA
:10D48000EAE6F9E007C09091C00095FFFCCF8093D9
:10D49000C600319684918823B1F7E6EFFEE007C01D
:10D4A0009091C00095FFFCCF8093C6003196849187
:10D4B0008823B1F720918E0930918F0980E690E0A2
:10D4C000289FF001299FF00D389FF00D1124E65F91
:10D4D000F74F06C09091C00095FFFCCF8093C60027
:10D4E00081918823B9F7E8E0FFE007C09091C00080
:10D4F00095FFFCCF8093C600319684918823B1F7C5
:10D500008091C00085FFFCCF8AE08093C6000E9416
:10D51000632926C085ED9DE00E94022C0E941E9D7D
:10D52000DC01CB018093A2099093A309A093A409E5
:10D53000B093A5090E941E9DDC01CB018093A60932
:10D540009093A709A093A809B093A909E0CF0E94DE
:10D55000291688E50E944429882309F0E2CAE2CA14
:10D56000A2960FB6F894DEBF0FBECDBFDF91CF916C
:10D570001F910F91FF90EF90DF90CF90BF90AF90F1
:10D580009F908F907F906F905F904F903F902F90E3
:10D590000895CF93DF938091060890910708833018
:10D5A000910514F40E94E62C82E297E060E00E946C
:10D5B000D3818091060890910708009709F463C011
:10D5C00080912207882309F446C020918E0930916A
:10D5D0008F0980E690E0289FE001299FD00D389FB9
:10D5E000D00D1124C65FD74FCE016EEA73E00E94C2
:10D5F00084A80097B9F482E297E0BE010E94658199
:10D60000EBE2FCE007C09091C00095FFFCCF809357
:10D61000C600319684918823B1F78091C00085FFC0
:10D62000FCCF15C082E297E00E94E882EEE2FCE0C7
:10D6300007C09091C00095FFFCCF8093C600319643
:10D6400084918823B1F78091C00085FFFCCF8AE0E8
:10D650008093C60002C00E94C15880910608909134
:10D6600007080197909307088093060880918E0918
:10D6700090918F09019664E070E00E94FAA4909363
:10D680008F0980938E090E94EF6D81E00E94882CA3
:10D690000E94280E0E946358DF91CF9108958F92C7
:10D6A0009F92AF92BF92CF92DF92EF92FF920F9331
:10D6B0001F93CF930E9422298BE59AE040E950ED19
:10D6C00063E070E00E946878EDE7F9E007C09091B0
:10D6D000C00095FFFCCF8093C600319684918823CB
:10D6E000B1F78091C00085FFFCCF8AE08093C6002F
:10D6F0008AE699E0FC0107C03091C00035FFFCCFFD
:10D700002093C600319624912223B1F724B720FF3D
:10D7100014C0E3E8F9E007C04091C00045FFFCCF2A
:10D720003093C600319634913323B1F73091C00065
:10D7300035FFFCCF3AE03093C60021FF14C0EBE880
:10D74000F9E007C04091C00045FFFCCF3093C60010
:10D75000319634913323B1F73091C00035FFFCCFBF
:10D760003AE03093C60022FF14C0EBE9F9E007C0AD
:10D770004091C00045FFFCCF3093C60031963491F4
:10D780003323B1F73091C00035FFFCCF3AE030933E
:10D79000C60023FF14C0ECEAF9E007C04091C000C6
:10D7A00045FFFCCF3093C600319634913323B1F757
:10D7B0003091C00035FFFCCF3AE03093C60025FF22
:10D7C00014C0ECEBF9E007C03091C00035FFFCCF8E
:10D7D0002093C600319624912223B1F72091C000F6
:10D7E00025FFFCCF2AE02093C60014BEECECF9E044
:10D7F00007C03091C00035FFFCCF2093C6003196A2
:10D8000024912223B1F7E5EDF9E007C03091C00083
:10D8100035FFFCCF2093C600319624912223B1F727
:10D820002091C00025FFFCCF2AE02093C600FC0118
:10D830002491EAE6F9E008C03091C00035FFFCCF42
:10D840002093C600319624912223B1F7EFEDF9E041
:10D8500007C03091C00035FFFCCF2093C600319641
:10D8600024912223B1F7EFEEF9E007C03091C00018
:10D8700035FFFCCF2093C600319624912223B1F7C7
:10D88000E1E4FAE007C03091C00035FFFCCF2093FF
:10D89000C600319624912223B1F7EDE4FAE007C0E7
:10D8A0003091C00035FFFCCF2093C6003196249103
:10D8B0002223B1F72091C00025FFFCCF2AE020935E
:10D8C000C600FC018491EAE6F9E008C09091C0002E
:10D8D00095FFFCCF8093C600319684918823B1F7E1
:10D8E000EDE5FAE007C09091C00095FFFCCF809372
:10D8F000C600319684918823B1F70E948D28BC011F
:10D900008BE59AE04AE050E00E949379ECE6FAE079
:10D9100007C09091C00095FFFCCF8093C600319660
:10D9200084918823B1F78BE59AE060ED74E04AE0DA
:10D9300050E00E9493798091C00085FFFCCF8AE07F
:10D940008093C60010928A0910928B0910928C095C
:10D9500010928D0980E00E94DB530FEE1FE0AFEFC5
:10D96000AA2EAFE0BA2EB3EC8B2EBFE09B2EC0E008
:10D97000F80161917191819191918F01F501C190AF
:10D98000D190E190F1905F010E94CCA1A701960196
:10D990000E9401A40E94A0A1DC01CB01F4018193AB
:10D9A0009193A193B1934F01CF5FC43009F70E94C7
:10D9B00013700E94DE8C0E94CC15CF911F910F91A5
:10D9C000FF90EF90DF90CF90BF90AF909F908F909F
:10D9D000089521E434E0FC01318320832781222350
:10D9E00019F004960E94211B0895CF92EF920F9395
:10D9F00081309105A9F482E297E00E94927A82EE4A
:10DA000096E064E141E120E105E135E0E32E56E0F6
:10DA1000C52E0E941FA085EF99E00E94F73116C025
:10DA20000097A1F485ED97E00E94E96C83E997E007
:10DA30000E94E96C84E797E00E94E96C85E597E035
:10DA40000E94E96C84E397E00E94E96C0F91EF90EB
:10DA5000CF90089581E090E00E94F56C089580E0F9
:10DA600090E00E94F56C089560E070E08FE793E429
:10DA700020913204309133044091340450913504A4
:10DA80000E9433A1DC01CB018093210A9093220AEA
:10DA9000A093230AB093240A0895FC01E05EF54F99
:10DAA000808190E00895CF93DF93EC01662351F1DC
:10DAB000EAE4F3E107C09091C00095FFFCCF8093AA
:10DAC000C600319684918823B1F78BE59AE070E027
:10DAD0004AE050E00E949379E1E5F3E107C09091BC
:10DAE000C00095FFFCCF8093C600319684918823B7
:10DAF000B1F78091C00085FFFCCF8AE08093C6001B
:10DB00000E94552CBE01882777FD8095982F0E9492
:10DB1000CEA12FE632E143E050E40E9401A420E0D0
:10DB200030E040E851E40E9401A40E949BA1CB0197
:10DB3000DF91CF91089580E090E00895CF93DF9337
:10DB4000EC01662351F1EAE4F3E107C09091C000D3
:10DB500095FFFCCF8093C600319684918823B1F75E
:10DB60008BE59AE070E04AE050E00E949379EDE6A0
:10DB7000F3E107C09091C00095FFFCCF8093C600F1
:10DB8000319684918823B1F78091C00085FFFCCF46
:10DB90008AE08093C6000E94552CBE01882777FD3D
:10DBA0008095982F0E94CEA120E030E04AEF5EE3FE
:10DBB0000E9401A420E030E040E85DE30E9401A45F
:10DBC00020E030E040E050E00E9453A0462F572F65
:10DBD000682F792FCB01BA01DF91CF9108952F9251
:10DBE0003F924F925F926F927F928F929F92AF92ED
:10DBF000BF92CF92DF92EF92FF920F931F93CF933A
:10DC0000DF9300D00F92CDB7DEB78091130A88233F
:10DC100009F4EDC18FB7F8941092130A8FBF809169
:10DC20001A0A90911B0A60E00E949E6D2B013C0134
:10DC30006091140A7091150A8091160A9091170A42
:10DC4000A30192010E9452A0C62EB72E182F092FB1
:10DC50009801862F9B2DA32FB22F8093250A909396
:10DC6000260AA093270AB093280ABC01CD0120E020
:10DC700030E040E251E40E942FA318160CF450C18A
:10DC800098018C2D9B2DA32FB22FBC01CD0120E03C
:10DC900030E040E251EC0E942CA187FD3DC1809113
:10DCA000290A882309F029C198018C2D9B2DA32FC7
:10DCB000B02FBC01CD012091360430913704409142
:10DCC0003804509139040E9401A469837A831C01AD
:10DCD000472F862F942FA22DB32D80932E0A909339
:10DCE0002F0AA093300AB093310A98018C2D9B2DF6
:10DCF000A32FB02FBC01CD0120912A0A30912B0A0D
:10DD000040912C0A50912D0A0E9453A0B62EA72EA6
:10DD1000982E892E0091320A1091330A2091340AEC
:10DD20002C838091350A8B83A5019401852F942F34
:10DD3000A32FB22FBC01CD013C812B81C02ED12E4F
:10DD4000E32EF22EA70196010E942CA187FFB3C0FB
:10DD50003C812B81802F912FA32FB22F80932A0AF1
:10DD600090932B0AA0932C0AB0932D0ABC01CD01ED
:10DD700020913204309133044091340450913504A1
:10DD80000E9401A46B83872E182F092F9801862FDC
:10DD9000982DA32FB22F8093360A9093370AA09321
:10DDA000380AB093390AC301B20120913A0A30917E
:10DDB0003B0A40913C0A50913D0A0E9452A020919A
:10DDC0002E0430912F0440913004509131040E9470
:10DDD00001A420ED3CEC4CE45DE30E9401A46B0146
:10DDE0007C0160913E0A70913F0A8091400A9091B7
:10DDF000410A23E333E343E75FE30E9401A49B016D
:10DE0000AC01C701B6010E9453A0B62EC72EA82EA2
:10DE1000992E862F9C2DAA2DB92D80933E0A909382
:10DE20003F0AA093400AB093410A40923A0A5092A6
:10DE30003B0A60923C0A70923D0A59814A81852FC3
:10DE4000942FA22DB32DBC01CD01FB81A8010F2F72
:10DE5000182D252F342FA90198010E9453A00B2DB6
:10DE60001C2D2A2D392DA90198010E9452A0C62EE1
:10DE7000B72E182F092F9801862F9B2DA32FB22F75
:10DE8000BC01CD0120E030E040E050E00E942CA138
:10DE900087FD4EC098018C2D9B2DA32FB22FBC0166
:10DEA000CD0120E030E04FE753E40E942FA3181685
:10DEB0000CF042C038C00091210A1091220AE09172
:10DEC000230AEC83F091240AFB83A5019401852F9A
:10DED000942FA32FB22FBC01CD01C02ED12EEE2E38
:10DEE000FF2EA70196010E942FA318160CF430CF25
:10DEF0000B2D1A2D9C828B822BCF80E090E0A0E02E
:10DF0000B0E080932A0A90932B0AA0932C0AB09336
:10DF10002D0A1092290AC8CE81E08093290A08C0F0
:10DF200081E08093290ACC24BB241FE703E404C0CA
:10DF3000CC24BB2410E000E080911A0A90911B0AC7
:10DF40002091420A3091430A281739071CF0109299
:10DF5000200A14C020913A0430913B0482179307A1
:10DF6000B4F798018C2D9B2DA32FB02FBC01CD01B0
:10DF70000E949BA1759567956093200A0E941E9D43
:10DF8000DC01CB014091440A5091450A6091460A58
:10DF90007091470A841B950BA60BB70B883823E1B9
:10DFA000920720E0A20720E0B20708F10E941E9D20
:10DFB000DC01CB018093440A9093450AA093460A62
:10DFC000B093470A8091180A9091190A18161906F9
:10DFD0006CF4EFE38F3F9E074CF420911C0A3091C4
:10DFE0001D0A8217930714F4A59A01C0A5980F90F3
:10DFF0000F900F900F90DF91CF911F910F91FF9095
:10E00000EF90DF90CF90BF90AF909F908F907F90D8
:10E010006F905F904F903F902F90089560E070E078
:10E0200080E090E0089580E090E0A0E0B0E0809390
:10E03000320A9093330AA093340AB093350A60E011
:10E0400070E08FE793E420913204309133044091E3
:10E050003404509135040E9433A1DC01CB0180933C
:10E06000210A9093220AA093230AB093240A6C9A5F
:10E070006D9A9D9AE1E0F1E080818061808387ED77
:10E0800080937A0010927E00EDE7F0E010828081AC
:10E0900081608083808182608083808184608083CE
:10E0A00080E888BDEEE6F0E08081846080836AEFDE
:10E0B00070E080E090E00E945A9D85E090E060E092
:10E0C0000E94536D9093430A8093420A83E191E04A
:10E0D00060E00E94536D90933B0480933A0408954E
:10E0E000089580E090E060E00E94536D80E090E051
:10E0F000A0E0B0E08093140A9093150AA093160A4A
:10E10000B093170A10921D0A10921C0A10921F0A4F
:10E1100010921E0A1092200A82E060E00E949D9CEC
:10E120001092210A1092200A1092210A83E060E0E6
:10E130000E949D9C10921D0A10921C0A84E060E0CF
:10E140000E949D9C08952F923F924F925F926F92F2
:10E150007F928F929F92AF92BF92CF92DF92EF9277
:10E16000FF920F931F93CF93DF93CDB7DEB7E09766
:10E170000FB6F894DEBF0FBECDBF6D877E878F8749
:10E18000988B8FE78093200A0E941E9D6B8B7C8B5F
:10E190008D8B9E8BE2EBF3E006C09091C00095FF63
:10E1A000FCCF8093C60081918823B9F78091C0008D
:10E1B00085FFFCCF8AE08093C6000E9471702B8996
:10E1C0003C894D895E892B8F3C8F4D8F5E8F2F8BC5
:10E1D000388F498F5A8F8FE790E0A0E0B0E08D83B1
:10E1E0009E83AF83B8872FE730E040E050E029837B
:10E1F0003A834B835C8391E01A8A198AEBE8F2E157
:10E20000349139A7E3E9F2E144914AA7E8E9F2E160
:10E2100054915BA7EFE9F2E184918CA7E6EAF2E181
:10E22000A491ADA7ECEAF2E1B491BEA7F92E8091DA
:10E23000130A882309F4B5C48FB7F8941092130A0F
:10E240008FBF80911A0A90911B0A60E00E949E6D18
:10E2500069877A878B879C875F8D48A139A12AA11E
:10E26000852F942FA32FB22FBC01CD01F985EA850C
:10E270005B854C850F2F1E2F252F342FA901980168
:10E280000E942FA3181634F00F8F18A32B8529A3F3
:10E290003C853AA3892D9A2DAB2DB82DBC01CD011B
:10E2A000F985EA855B854C850F2F1E2F252F342F8E
:10E2B000A90198010E942CA187FD04C0902EA12ED7
:10E2C000BB848C84FF2009F45CC059854A853B855A
:10E2D0002C85852F942FA32FB22FBC01CD01FD8556
:10E2E000EE855F8548890F2F1E2F252F342FA9011A
:10E2F00098010E942FA318160CF053C40E941E9D73
:10E30000DC01CB012B8D3C8D4D8D5E8D821B930BE3
:10E31000A40BB50B893833E1930730E0A30730E055
:10E32000B30708F43EC489819A81AB81BC812D81F9
:10E330003E814F815885821B930BA40BB50BB5957D
:10E34000A795979587958093200A0E941E9D6F8BB5
:10E35000788F898F9A8FDC01CB012B8D3C8D4D8D71
:10E360005E8D821B930BA40BB50B8DA39EA3AFA355
:10E37000B8A73D853F8F4E8548A35F8559A38889FF
:10E380008AA359854A853B852C85852F942FA32FF9
:10E39000B22FBC01CD01FD85EE855F8548890F2F29
:10E3A0001E2F252F342FA90198010E942CA187FF31
:10E3B000F7C30E941E9DDC01CB012F89388D498D4A
:10E3C0005A8D821B930BA40BB50B893833E193074D
:10E3D00030E0A30730E0B30708F4E2C30E941E9DBB
:10E3E0006B8F7C8F8D8F9E8F49895A89411551057E
:10E3F00009F4B7C3DC01CB012F89388D498D5A8DC3
:10E40000821B930BA40BB50B4DA05EA06FA078A44C
:10E41000480E591E6A1E7B1E2DA13EA14FA158A574
:10E42000281B390B4A0B5B0B6D817E818F81988590
:10E430000E94C7A4A30192010E942FA589019A01FD
:10E4400089819A81AB81BC81080F191F2A1F3B1F4C
:10E4500004311105210531051CF109831A832B8331
:10E460003C830C3E11052105310544F02BEE30E0D4
:10E4700040E050E029833A834B835C8389819A8111
:10E48000AB81BC8180389105A105B105D4F02EEF98
:10E4900030E040E050E0281B390B4A0B5B0B0CC00E
:10E4A00084E190E0A0E0B0E089839A83AB83BC83F1
:10E4B00024E130E040E050E02D833E834F835887D5
:10E4C00008C089819A81AB81BC818D839E83AF8393
:10E4D000B88789A5EBE8F2E108C09091C00095FFEC
:10E4E000FCCF8093C600319684918823B1F78BE5E9
:10E4F0009AE049815A816B817C812AE030E00E9458
:10E500005E798AA5E3E9F2E108C09091C00095FF29
:10E51000FCCF8093C600319684918823B1F78BE5B8
:10E520009AE04D815E816F8178852AE030E00E941B
:10E530005E798BA5E8E9F2E108C09091C00095FFF3
:10E54000FCCF8093C600319684918823B1F78BE588
:10E550009AE0492D5A2D6B2D782D22E030E00E9453
:10E560008F7A8CA5EFE9F2E108C09091C00095FF89
:10E57000FCCF8093C600319684918823B1F78BE558
:10E580009AE0FF8DE8A139A12AA14F2F5E2F632FBA
:10E59000722F22E030E00E948F7A8091C00085FFC8
:10E5A000FCCF8AE08093C600A989BA89A330B1055F
:10E5B0000CF4D7C26D817E818F8198850E94CEA197
:10E5C00020E030E040E850E40E9401A46B017C01AF
:10E5D0005F8D48A139A12AA1852F942FA32FB22F97
:10E5E000BC01CD01092D1A2D2B2D382DA901980123
:10E5F0000E9452A020ED3FE049E450E40E9401A4B3
:10E6000020E030E040E05FE30E9401A49B01AC0108
:10E61000C701B6010E9433A1362E272E8BA39CA3DF
:10E62000C301B2010E94CEA120E030E04AE754E4E9
:10E630000E9433A1D62EC72EB82EA92E8DA5E6EAAC
:10E64000F2E108C09091C00095FFFCCF8093C60016
:10E65000319684918823B1F78BE59AE0F1013BA1D3
:10E660002CA14F2F522D632F722F22E030E00E94F9
:10E670008F7A8EA5ECEAF2E108C09091C00095FF78
:10E68000FCCF8093C600319684918823B1F78BE547
:10E690009AE0F60195014F2F5C2D632F7A2D22E031
:10E6A00030E00E948F7A8091C00085FFFCCF8AE025
:10E6B0008093C600A1013BA12CA1852F922DA32FF1
:10E6C000B22FBC01CD012AE939E949E15FE30E949B
:10E6D00001A46FA778ABF82EE92E562F472F97018C
:10E6E000862F942FA32FB22FBC01CD01FA01A701D1
:10E6F0000F2F1E2F252F342FA90198010E9453A000
:10E70000F601A5010F2F1C2D252F3A2DA9019801E7
:10E710000E9433A1962E872E782E692E5FA548A9D8
:10E720009701852F942FA32FB22FBC01CD01A501F6
:10E73000252F3A2DA90198010E9401A420E030E084
:10E7400040E05EE30E9401A4162F072F582E492EA9
:10E75000E2EBF2E184919FA538A90AC0292F90919C
:10E76000C00095FFFCCF922F8093C6003196849114
:10E770008823A1F78091C00085FFFCCF9FA738AB0D
:10E780008AE08093C600EFEBF2E184919FA538A95F
:10E790000AC0292F9091C00095FFFCCF922F809343
:10E7A000C600319684918823A1F79FA738AB8BE5EB
:10E7B0009AE0FFA5E32F97014F2F5E2F632F7E2D49
:10E7C00022E030E00E948F7A8091C00085FFFCCF6C
:10E7D0008AE08093C600E5ECF2E107C09091C000AA
:10E7E00095FFFCCF8093C600319684918823B1F7C2
:10E7F0008BE59AE0F40193014F2F582D632F762D6E
:10E8000022E030E00E948F7A8091C00085FFFCCF2B
:10E810008AE08093C600EBECF2E107C09091C00063
:10E8200095FFFCCF8093C600319684918823B1F781
:10E830008BE59AE0F80192014F2F502F632F742D32
:10E8400022E030E00E948F7A8091C00085FFFCCFEB
:10E850008AE08093C600A1013BA12CA1852F922DB7
:10E86000A32FB22FBC01CD0123EC35EF48EA5EE3C4
:10E870000E9401A46FA778ABF82EE92E472F9701CD
:10E88000862F942FA32FB22FBC01CD01F601A50135
:10E890000F2F1C2D252F3A2DA90198010E9433A17D
:10E8A000962E872E782E692E5FA548A99701852F71
:10E8B000942FA32FB22FBC01CD01A501252F3A2DF6
:10E8C000A90198010E9401A420E030E040E450E456
:10E8D0000E9433A1162F072F582E492EE1EDF2E1A9
:10E8E00084919FA538A90AC0292F9091C00095FF57
:10E8F000FCCF922F8093C600319684918823A1F794
:10E900008091C00085FFFCCF9FA738AB8AE0809341
:10E91000C600E2EEF2E184919FA538A90AC0292F32
:10E920009091C00095FFFCCF922F8093C600319646
:10E9300084918823A1F79FA738AB8BE59AE0FFA5C8
:10E94000E32F97014F2F5E2F632F7E2D22E030E0C3
:10E950000E948F7A8091C00085FFFCCF8AE080936F
:10E96000C600E8EEF2E107C09091C00095FFFCCF31
:10E970008093C600319684918823B1F78BE59AE0A5
:10E98000F40193014F2F582D632F762D22E030E0B4
:10E990000E948F7A8091C00085FFFCCF8AE080932F
:10E9A000C600EEEEF2E107C09091C00095FFFCCFEB
:10E9B0008093C600319684918823B1F78BE59AE065
:10E9C000F80192014F2F502F632F742D22E030E079
:10E9D0000E948F7A8091C00085FFFCCF8AE08093EF
:10E9E000C600A1013BA12CA1852F922DA32FB22FF0
:10E9F000BC01CD012DEC3CEC4CE45EE30E9401A493
:10EA0000562E472EF82EE92EA2019701852F942F1E
:10EA1000A32FB22FBC01CD01F201A7010F2F1E2F92
:10EA2000252F342FA90198010E9453A0F601A501BA
:10EA30000F2F1C2D252F3A2DA90198010E9433A1DB
:10EA4000962E872E782E692EA2019701852F942F5E
:10EA5000A32FB22FBC01CD01A501252F3A2DA9016D
:10EA600098010E9401A420E030E040E450E40E94BC
:10EA700033A1162F072FD82EC92EE4EFF2E107C0DD
:10EA80009091C00095FFFCCF8093C6003196849191
:10EA90008823B1F78091C00085FFFCCF8AE0809386
:10EAA000C600E3E0F3E107C09091C00095FFFCCF02
:10EAB0008093C600319684918823B1F78BE59AE064
:10EAC000F20197014F2F542D632F7E2D22E030E06D
:10EAD0000E948F7A8091C00085FFFCCF8AE08093EE
:10EAE000C600E9E0F3E107C09091C00095FFFCCFBC
:10EAF0008093C600319684918823B1F78BE59AE024
:10EB0000F40193014F2F582D632F762D22E030E032
:10EB10000E948F7A8091C00085FFFCCF8AE08093AD
:10EB2000C600EFE0F3E107C09091C00095FFFCCF75
:10EB30008093C600319684918823B1F78BE59AE0E3
:10EB4000F80196014F2F502F632F7C2D22E030E0EB
:10EB50000E948F7A8091C00085FFFCCF8AE080936D
:10EB6000C60089819A81AB81BC812D813E814F8114
:10EB70005885820F931FA41FB51FB595A79597952C
:10EB800087958093200A49895A894F5F5F4F5A8B36
:10EB9000498B9D84AE84BF848888FF24F39401C090
:10EBA000FF245D854E853F852889852F942FA32FCF
:10EBB000B22FBC01CD0120E030E040EA51E40E94D8
:10EBC00053A09B01AC01F985EA857B856C858F2F6D
:10EBD0009E2FA72FB62FBC01CD010E942FA3181680
:10EBE0006CF5E5E1F3E107C09091C00095FFFCCF23
:10EBF0008093C600319684918823B1F78091C0003C
:10EC000085FFFCCF8AE08093C600E0960FB6F894AB
:10EC1000DEBF0FBECDBFDF91CF911F910F91FF904F
:10EC2000EF90DF90CF90BF90AF909F908F907F90AC
:10EC30006F905F904F903F902F9008950E941E9D7F
:10EC4000DC01CB012B893C894D895E89821B930BAA
:10EC5000A40BB50B813D37E0930730E0A30730E00C
:10EC6000B30708F43FC00E941E9D6B8B7C8B8D8B7D
:10EC70009E8BE0E4F3E107C09091C00095FFFCCFCC
:10EC80008093C600319684918823B1F780911A0A47
:10EC900090911B0A60E00E949E6DAB01BC018BE568
:10ECA0009AE022E030E00E948F7AE6E4F3E107C0C8
:10ECB0009091C00095FFFCCF8093C600319684915F
:10ECC0008823B1F76091200A8BE59AE070E04AE072
:10ECD00050E00E9493798091C00085FFFCCF8AE0CC
:10ECE0008093C6000E946358A2CACF93C82F82E0C7
:10ECF00060E00E949D9C0E94D32B882379F5EAE472
:10ED0000F3E107C09091C00095FFFCCF8093C6004F
:10ED1000319684918823B1F78BE59AE06C2F40E01F
:10ED200050E00E9456798091C00085FFFCCF8AE0B8
:10ED30008093C600EAE8F3E107C09091C00095FF18
:10ED4000FCCF8093C600319684918823B1F78091DF
:10ED5000C00085FFFCCF8AE08093C600CF91089564
:10ED6000CF93C82F82E060E00E949D9C0E94D32B2D
:10ED7000882379F5EAE4F3E107C09091C00095FF9C
:10ED8000FCCF8093C600319684918823B1F78BE540
:10ED90009AE06C2F40E050E00E9456798091C000CC
:10EDA00085FFFCCF8AE08093C600E7EBF3E107C064
:10EDB0009091C00095FFFCCF8093C600319684915E
:10EDC0008823B1F78091C00085FFFCCF8AE0809353
:10EDD000C600CF9108951F920F920FB60F920BB6F7
:10EDE0000F9211242F933F934F935F936F937F93D1
:10EDF0008F939F93AF93BF93EF93FF9380913C04C6
:10EE0000882331F48091200A8093480A8111749AF2
:10EE10009091480A80913C04891708F074988F5F9C
:10EE20008F7780933C048091490A833009F450C065
:10EE3000843028F48130F9F08230D8F50DC0853067
:10EE400009F471C0853008F45FC0863009F487C0CA
:10EE5000873009F08FC087C088E080937B0080E412
:10EE600080937C0080917A00806480937A000E9475
:10EE70008A3181E01BC0409178005091790060E0B8
:10EE800070E080914A0A90914B0AA0914C0AB0918F
:10EE90004D0A840F951FA61FB71F80934A0A9093AF
:10EEA0004B0AA0934C0AB0934D0A82E08093490A22
:10EEB00061C088E080937B0082E480937C00809135
:10EEC0007A00806480937A000E948A3183E0EECFDA
:10EED000409178005091790060E070E080914E0A96
:10EEE00090914F0AA091500AB091510A840F951F3A
:10EEF000A61FB71F80934E0A90934F0AA093500A03
:10EF0000B093510A84E0D2CF88E080937B0081E403
:10EF100080937C0080917A00806480937A000E94C4
:10EF20008A3185E0C3CF409178005091790060E04C
:10EF300070E08091520A9091530AA091540AB091C6
:10EF4000550A840F951FA61FB71F8093520A9093EE
:10EF5000530AA093540AB093550A86E0A7CF0E94A3
:10EF60008A3187E0A3CF1092490A8091560A8F5FB9
:10EF70008093560A8091560A803108F45DC0209132
:10EF80004A0A30914B0A30931B0A20931A0A8FEFDA
:10EF90009FE340914E0A50914F0A841B950B90932A
:10EFA000190A8093180A81E08093130A1092560A76
:10EFB00010924A0A10924B0A10924C0A10924D0A73
:10EFC0001092520A1092530A1092540A1092550A43
:10EFD0001092570A1092580A1092590A10925A0A1F
:10EFE00010924E0A10924F0A1092500A1092510A33
:10EFF00080913A0490913B04281739074CF0109205
:10F000001F0A10921E0A80E00E9475760E94162C3C
:10F0100020911A0A30911B0A8091420A9091430A6A
:10F02000821793074CF010921F0A10921E0A80E07C
:10F030000E94B0760E94162CFF91EF91BF91AF9184
:10F040009F918F917F916F915F914F913F912F9100
:10F050000F900BBE0F900FBE0F901F9018951F9230
:10F060000F920FB60F920BB60F9211242F933F936E
:10F070004F935F936F938F939F93EF93FF93609161
:10F08000C6002091DC0A3091DD0AC90101968F7714
:10F0900090704091DE0A5091DF0A8417950741F085
:10F0A000245A354FF90160839093DD0A8093DC0A7E
:10F0B000FF91EF919F918F916F915F914F913F9150
:10F0C0002F910F900BBE0F900FBE0F901F901895B1
:10F0D0000F931F939A01AB01203081EE380780E037
:10F0E000480780E0580769F182E08093C00060E043
:10F0F00079E08DE390E00E942FA589019A010150EB
:10F10000104020403040C901B80122E030E040E02A
:10F1100050E00E942FA53093C5002093C400809139
:10F12000C10080618093C1008091C100886080939C
:10F13000C1008091C10080688093C1001F910F9130
:10F1400008951092C00020E130E0E5CF2091DE0A62
:10F150003091DF0A8091DC0A9091DD0A82179307D3
:10F1600071F0F901E45AF54F80812F5F3F4F2F77FF
:10F1700030703093DF0A2093DE0A90E008958FEF1D
:10F180009FEF08958091DE0A9091DF0A9093DD0A47
:10F190008093DC0A08956F927F928F929F92AF9234
:10F1A000BF92CF92DF92EF92FF920F931F93CF9374
:10F1B000DF93CDB7DEB7A0970FB6F894DEBF0FBED2
:10F1C000CDBF3C01DB01CA01411551056105710547
:10F1D00051F4C30140E350E060E070E020E030E033
:10F1E0000E945E7941C08E010F5F1F4FCC24DD2449
:10F1F0007601822E9924AA24BB24BC01CD01A5014D
:10F2000094010E940DA5F80161938F010894C11C1F
:10F21000D11CE11CF11CC901DA010097A105B1055F
:10F2200061F714C0E1E0F0E0EC0FFD1FEC0DFD1DF7
:10F2300040814A3010F4405D01C0495C50E060E01C
:10F2400070E0C30120E030E00E945E790894C108BC
:10F25000D108E108F108FFEFCF16FFEFDF06FFEF5F
:10F26000EF06FFEFFF06F1F6A0960FB6F894DEBFAB
:10F270000FBECDBFDF91CF911F910F91FF90EF9007
:10F28000DF90CF90BF90AF909F908F907F906F90C6
:10F2900008952115310539F48091C00085FFFCCF18
:10F2A0004093C60008950E94CB7808959A01462F96
:10F2B00050E060E070E00E9449790895CF92DF92BB
:10F2C000EF92FF92CF93DF93EC016A017B0121154E
:10F2D000310539F48091C00085FFFCCFC092C60093
:10F2E0001BC02A303105B1F477FF10C04DE250E069
:10F2F00060E070E020E030E00E945E79F094E094FD
:10F30000D094C094C11CD11CE11CF11CCE01B701EA
:10F31000A6012AE00E94CB78DF91CF91FF90EF9079
:10F32000DF90CF9008959A01FB01AF01662757FD4A
:10F330006095762F0E945E790895CF93DF93EC015C
:10F340004DE050E060E070E020E030E00E945E7947
:10F35000CE014AE050E060E070E020E030E00E9442
:10F360005E79DF91CF910895CF93DF93EC019A01FD
:10F37000AB0160E070E00E944979CE010E949D7966
:10F38000DF91CF9108958F929F92BF92CF92DF929B
:10F39000EF92FF920F931F93CF93DF934C016A017B
:10F3A0007B01B22ECB01BA0120E030E040E050E01A
:10F3B0000E942CA187FF0DC0C4014DE250E060E027
:10F3C00070E020E030E00E945E79F7FAF094F7F800
:10F3D000F094C0E050E040E030E02FE313C0FA01C9
:10F3E000B9018F2F942FA72FB22FBC01CD0120E0A0
:10F3F00030E040E251E40E9433A1562F472F382FCE
:10F40000292FCF5FCB1559F7C701B601DA01F901F2
:10F410000B2F142F2F2F3E2FA90198010E9453A0CC
:10F420006B01E82EC92F862F9D2DAE2DBC2FBC0160
:10F43000CD010E94A0A1D62F172F082FF92E0E94D0
:10F44000CCA19B01AC018C2D9D2DAE2DBC2FBC0100
:10F45000CD010E9452A0D62EE72EC82FC92EC4017E
:10F460004D2F512F602F7F2D2AE030E00E944979E7
:10F47000BB2009F446C0E5ECF3E006C09091C00063
:10F4800095FFFCCF8093C60081918823B9F739C0DE
:10F490008D2D9E2DAC2FBC2DBC01CD0120E030E088
:10F4A00040E251E40E9401A4EB01182F092F9801BA
:10F4B000862F9D2FA32FB22FBC01CD010E949BA1AF
:10F4C0006B017C01EE24D7FCE094FE2CC401B70153
:10F4D000A6012AE030E00E945E79C701B6010E94D1
:10F4E000CEA19B01AC01B8018C2F9D2FA72FB62F69
:10F4F000BC01CD010E9452A0D62EE72EC82FC92EE6
:10F50000BA94BB2029F6DF91CF911F910F91FF9004
:10F51000EF90DF90CF90BF909F908F9008950E94C2
:10F52000C3790895CF93DF93FC01168A118E158A53
:10F53000148A81E494E0938B828B17AA12AE16AAE8
:10F5400015AA94AB83ABDF01AA5ABF4F1C92139646
:10F550001C92DF01AE5ABF4F13961C921E92129757
:10F560008D939C93DF01AB58BF4F1C9213961C9256
:10F57000DF01AF58BF4F13961C921E9212978D93C6
:10F580009C93DF01A057BF4F29E111962C9311974F
:10F5900014961C92DF01A455BF4F1C92DF01A954A1
:10F5A000BF4F1C9213961C92DF01AD54BF4F1396B0
:10F5B0001C921E9212978D939C93DF01AE52BF4F07
:10F5C0001D921D921D921C921397DF01A652BF4FF0
:10F5D0001D921D921D921C9213971182128210820D
:10F5E000EF01CA52DF4F188219821A821B82DF0193
:10F5F000A252BF4F81E08C93118A108A0E941E9DF7
:10F60000DC01CB0188579C4EAF4FBF4F8883998355
:10F61000AA83BB83DF91CF910895DB01FC0120E039
:10F620003EE24C91403229F0283009F431934C915C
:10F6300041932F5F11962B30A1F7108208952F92DE
:10F640003F924F925F926F927F928F929F92AF9272
:10F65000BF92CF92DF92EF92FF920F931F93CF93BF
:10F66000DF93CDB7DEB7C758D0400FB6F894DEBFF2
:10F670000FBECDBF8C015B016A01FF2484E090E0E6
:10F68000C80ED91E23E0422E512C400E511E3FEDD4
:10F69000832E912C800E911EE0EE6E2E712C600E4A
:10F6A000711EF1E42F2EF4E03F2EE7E4F0E0EC0FC2
:10F6B000FD1F3496CA57DF4FF983E883C658D04000
:10F6C000EEE1F4E1E4900FC1E2968FADE29790E0B5
:10F6D0009C01287130702031310509F00EC1F40110
:10F6E0004081413009F409C1423009F406C1CE011C
:10F6F0000196BE016A597F4F0E940D7B1E86F5015F
:10F700008081882331F4CE010E9667EC73E00E946D
:10F710004AA8CE010E96B5010E944AA8CE010E96C7
:10F72000BE016F5F7F4F0E944AA8CE010E9667EC24
:10F7300073E00E944AA82C961FAE2C972F961FAEFE
:10F740002F972B961FAE1EAE2B9729963FAE2EAE4F
:10F750002997CA57DF4F88819981C658D040B60192
:10F76000AE014F5F5F4F21E00E94531D8823C1F51A
:10F77000F40180818823A1F58E2DEEE1F4E108C02B
:10F780009091C00095FFFCCF8093C6003196849184
:10F790008823B1F7E9ECF3E006C09091C00095FF33
:10F7A000FCCF8093C60081918823B9F78091C00077
:10F7B00085FFFCCF8AE08093C600FE01319606C02B
:10F7C0009091C00095FFFCCF8093C6008191882363
:10F7D000B9F78091C00085FFFCCF8AE08093C60016
:10F7E000FE01BC96CA57DF4FA881B981C658D040E8
:10F7F0008BE10D9001928150E1F72B968EAD9FAD7C
:10F800002B979BA78AA739A628A6C801BE01625FCD
:10F810007F4FAE01485D5F4F0E941F7BCE018896EF
:10F820000E94E96CCE01895B9F4F0E94E96C5BC02E
:10F83000453E09F458C04E3209F455C04F3509F41D
:10F8400052C083FD50C081E02031310509F080E0D5
:10F85000F8018787882359F4AF968FADAF97873427
:10F8600009F041C0E0968FADE0978E37E1F1C2011B
:10F87000BE016A597F4F0E940D7BF401808188236D
:10F88000F1F4F50106C09091C00095FFFCCF809384
:10F89000C60081918823B9F7F20106C09091C0009B
:10F8A00095FFFCCF8093C60081918823B9F78091A2
:10F8B000C00085FFFCCF8AE08093C60014C0813071
:10F8C00039F4F301808191810196918380830BC08B
:10F8D000823049F48F2D90E0F3012081318182172D
:10F8E000930789F0F394C601BE016A597F4F0E94C5
:10F8F000C51918160CF4E8CE06C0A7964FADA79709
:10F90000442309F095CFC957DF4F0FB6F894DEBFF7
:10F910000FBECDBFDF91CF911F910F91FF90EF9060
:10F92000DF90CF90BF90AF909F908F907F906F901F
:10F930005F904F903F902F900895EF92FF920F931A
:10F940001F93CF93DF93CDB7DEB76F970FB6F894C1
:10F95000DEBF0FBECDBF7C01FC01E152FF4F108224
:10F960008C010A5E1F4FC8010E94CF1AFE01359616
:10F97000D8018BE10D9001928150E1F7F701848964
:10F9800095899C838B8381E494E09A838983C70162
:10F990006CED73E0AE014F5F5F4F0E941F7BCE01A5
:10F9A00001960E94E96C6F960FB6F894DEBF0FBE09
:10F9B000CDBFDF91CF911F910F91FF90EF900895F0
:10F9C000EF92FF920F931F93CF93DF937C01FC0183
:10F9D0001282818D882321F0C70146960E94211B47
:10F9E000E701C057DF4FCE0160E045E30E94DE0C27
:10F9F0008823F9F4EEE1F4E107C09091C00095FF8F
:10FA0000FCCF8093C600319684918823B1F7E4E25D
:10FA1000F4E107C09091C00095FFFCCF8093C60031
:10FA2000319684918823B1F78091C00085FFFCCF87
:10FA300077C087010B561F4FC801BE0141E00E94ED
:10FA40004923882331F5C801BE0140E00E944923C3
:10FA50008823F9F4E1E3F4E107C09091C00095FF39
:10FA6000FCCF8093C600319684918823B1F7E8E3F8
:10FA7000F4E107C09091C00095FFFCCF8093C600D1
:10FA8000319684918823B1F78091C00085FFFCCF27
:10FA900047C0C7014696B8010E9424188823F9F48C
:10FAA000E1E3F4E107C09091C00095FFFCCF8093A3
:10FAB000C600319684918823B1F7EBE4F4E107C0E6
:10FAC0009091C00095FFFCCF8093C6003196849141
:10FAD0008823B1F78091C00085FFFCCF21C081E071
:10FAE000F7018283EEE1F4E107C09091C00095FF39
:10FAF000FCCF8093C600319684918823B1F7EBE563
:10FB0000F4E107C09091C00095FFFCCF8093C60040
:10FB1000319684918823B1F78091C00085FFFCCF96
:10FB20008AE08093C600D701D796F70176968BE1DD
:10FB300001900D928150E1F7F7018489958996AB88
:10FB400085ABC701429692AB81ABDF91CF911F91FC
:10FB50000F91FF90EF900895CF93DF93FC01EC019C
:10FB6000E796DC0156968BE10D9009928150E1F702
:10FB70008489958996AB85ABCF01C39692AB81AB57
:10FB8000DF91CF910895FC01118212820895FC014A
:10FB90008281882311F081E081830895FC018181B5
:10FBA0008111118208952F923F924F925F926F922E
:10FBB0007F928F929F92AF92BF92CF92DF92EF92FD
:10FBC000FF920F931F93CF93DF93CDB7DEB7AC9720
:10FBD0000FB6F894DEBF0FBECDBF6C014B01442EB3
:10FBE000FC018281882309F4BEC117EB612E712CC0
:10FBF0006C0C7D1CC3010E94211BF60111821A8A24
:10FC00001D8A198A188A81E494E09F878E87C6012D
:10FC1000429692AB81ABF40180818F3209F08EC0A5
:10FC2000C4016FE270E00E9455A87C010894E11CB9
:10FC3000F11CAAE05A2EBEE02B2E312C2C0E3D1EBC
:10FC400078C0C7016FE270E00E9455A85C01009780
:10FC500009F47CC0E816F90608F078C08C010E198A
:10FC60001F09CE010196B701A8010E9475A8E1E025
:10FC7000F0E0EC0FFD1FE00FF11F10828E010F5F0F
:10FC80001F4FF80106C09091C00095FFFCCF8093F4
:10FC9000C60081918823B9F78091C00085FFFCCF11
:10FCA0005092C600F60161A972A96115710519F09B
:10FCB0006C5F7F4F02C060E070E0CE014296AE0103
:10FCC0004F5F5F4F21E00E94531D882359F5E6E600
:10FCD000F4E107C09091C00095FFFCCF8093C6006F
:10FCE000319684918823B1F706C09091C00095FFAA
:10FCF000FCCF8093C600F80181918F018823A9F77A
:10FD0000EAE7F4E107C09091C00095FFFCCF809333
:10FD1000C600319684918823B1F78091C00085FF99
:10FD2000FCCFF3C0F60132AA21AA75010894E11CA8
:10FD3000F11CE114F10409F084CF05C0C601C3969B
:10FD4000F60192AB81ABE82C092D01C00F2DF60115
:10FD500061A972A9442009F49EC06115710519F0CA
:10FD60006C5F7F4F02C060E070E0C3014E2D502FEA
:10FD700021E00E94531D882309F462C096012E528F
:10FD80003F4FF601E954FF4F81899289A389B489D5
:10FD9000F90180839183A283B383ECE7F4E107C088
:10FDA0009091C00095FFFCCF8093C600319684915E
:10FDB0008823B1F7EE2DF02F06C09091C00095FF7B
:10FDC000FCCF8093C60081918823B9F7E9E8F4E17C
:10FDD00007C09091C00095FFFCCF8093C60031967C
:10FDE00084918823B1F7F601EE52FF4F4081518193
:10FDF000628173818BE59AE02AE030E00E944979C4
:10FE00008091C00085FFFCCF8AE08093C600F60198
:10FE1000E652FF4F1082118212821382E0E9F4E170
:10FE200007C09091C00095FFFCCF8093C60031962B
:10FE300084918823B1F78091C00085FFFCCF88C0F2
:10FE4000EEE9F4E107C09091C00095FFFCCF8093EC
:10FE5000C600319684918823B1F7EE2DF02F06C0AD
:10FE60009091C00095FFFCCF8093C60081918823BC
:10FE7000B9F7E2EBF4E107C09091C00095FFFCCF29
:10FE80008093C600319684918823B1F78091C00099
:10FE900085FFFCCF3AC06115710519F06C5F7F4F8B
:10FEA00002C060E070E0C3014E2D502F26E50E9495
:10FEB000531D882371F5E4EBF4E107C09091C00075
:10FEC00095FFFCCF8093C600319684918823B1F7CB
:10FED000EE2DF02F06C09091C00095FFFCCF8093CF
:10FEE000C60081918823B9F7E8ECF4E107C090914E
:10FEF000C00095FFFCCF8093C60031968491882383
:10FF0000B1F78091C00085FFFCCF8AE08093C600E6
:10FF100026C081E0F6018083EAECF4E107C090910D
:10FF2000C00095FFFCCF8093C60031968491882352
:10FF3000B1F7F40106C09091C00095FFFCCF80930B
:10FF4000C60081918823B9F78091C00085FFFCCF5E
:10FF50008AE08093C6008E2D902F0E94E62BCE0162
:10FF60000E960E94E96CAC960FB6F894DEBF0FBEF9
:10FF7000CDBFDF91CF911F910F91FF90EF90DF9058
:10FF8000CF90BF90AF909F908F907F906F905F9039
:10FF90004F903F902F9008954F925F927F928F9253
:10FFA0009F92AF92BF92CF92DF92EF92FF920F9308
:10FFB0001F93CF93DF93CDB7DEB7AC970FB6F8940E
:10FFC000DEBF0FBECDBF6C014B01FC0182818823D7
:10FFD00009F410C1C60189549F4F0E94211BF601EC
:10FFE00011821A8A1D8A198A188A81E494E09F87EF
:10FFF0008E87C601429692AB81ABF40180818F322D
:020000021000EC
:1000000009F08EC0C4016FE270E00E9455A87C0127
:100010000894E11CF11C0AE0702E2EE0422E512CB7
:100020004C0E5D1E78C0C7016FE270E00E9455A8BB
:100030005C01009709F47CC0E816F90608F078C066
:100040008C010E191F09CE010196B701A8010E946B
:1000500075A8E1E0F0E0EC0FFD1FE00FF11F10824A
:100060008E010F5F1F4FF80106C09091C00095FFF1
:10007000FCCF8093C60081918823B9F78091C0009E
:1000800085FFFCCF7092C600F60161A972A96115C7
:10009000710519F06C5F7F4F02C060E070E0CE0127
:1000A0004296AE014F5F5F4F21E00E94531D8823AF
:1000B00059F5ECEDF4E107C09091C00095FFFCCF3D
:1000C0008093C600319684918823B1F706C0909141
:1000D000C00095FFFCCF8093C600F80181918F018D
:1000E0008823A9F7E0EFF4E107C09091C00095FFE5
:1000F000FCCF8093C600319684918823B1F780911C
:10010000C00085FFFCCF6FC0F60152AA41AA75015D
:100110000894E11CF11CE114F10409F084CF05C03E
:10012000C601C396F60192AB81ABE82C092D01C044
:100130000F2DF60181A992A9009711F0049602C033
:1001400080E090E06E2D702F0E94151E882309F12B
:10015000E2EFF4E107C09091C00095FFFCCF8093DF
:10016000C600319684918823B1F7EE2DF02F06C09A
:100170009091C00095FFFCCF8093C60081918823A9
:10018000B9F7F601E652FF4F1082118212821382F4
:100190002DC0E0E0F5E107C09091C00095FFFCCFD5
:1001A0008093C600319684918823B1F7EE2DF02F0D
:1001B00006C09091C00095FFFCCF8093C60081914E
:1001C0008823B9F7E8E1F5E107C09091C00095FFF9
:1001D000FCCF8093C600319684918823B1F780913B
:1001E000C00085FFFCCF8AE08093C600CE010E964A
:1001F0000E94E96CAC960FB6F894DEBF0FBECDBF7F
:10020000DF91CF911F910F91FF90EF90DF90CF90F2
:10021000BF90AF909F908F907F905F904F90089588
:10022000CF93DF93EC018A818823C1F1EAE1F5E104
:1002300007C09091C00095FFFCCF8093C600319617
:1002400084918823B1F7FE01E652FF4F408151812E
:10025000628173818BE59AE02AE030E00E9449795F
:10026000ECE2F5E107C09091C00095FFFCCF8093D0
:10027000C600319684918823B1F7CE52DF4F488172
:1002800059816A817B818BE59AE02AE030E00E9407
:1002900049798091C00085FFFCCF11C0EEE2F5E105
:1002A00007C09091C00095FFFCCF8093C6003196A7
:1002B00084918823B1F78091C00085FFFCCF8AE04C
:1002C0008093C600DF91CF910895CF92DF92EF9295
:1002D000FF920F931F93CF93DF936C017B01DB01A0
:1002E0000D900020E9F78D0101501040061B170BFF
:1002F000FC01E954FF4F1082CB016EE470E00E94D4
:1003000055A8EC01009729F4F8013197EE0DFF1D77
:100310000FC060E270E00E9455A87C010894E11CC7
:10032000F11CCE016AE270E00E9455A8FC013197F1
:100330008DE081838AE082831382C6018D549F4FB2
:10034000B7010E94A924F601E954FF4F8081882358
:1003500009F1E1E3F4E107C09091C00095FFFCCF03
:100360008093C600319684918823B1F7EEE3F5E1DE
:1003700007C09091C00095FFFCCF8093C6003196D6
:1003800084918823B1F78091C00085FFFCCF8AE07B
:100390008093C600DF91CF911F910F91FF90EF9056
:1003A000DF90CF9008952F923F924F925F926F927D
:1003B0007F929F92AF92BF92CF92DF92EF92FF9285
:1003C0000F931F93CF93DF93CDB7DEB7CC55D040BB
:1003D0000FB6F894DEBF0FBECDBF5C016623C1F43B
:1003E000FC01E252FF4F8081882309F4D8C0F50157
:1003F000EA52FF4FC080D180E280F3800E941E9DB0
:10040000DC01CB01C816D906EA06FB0608F4C7C012
:10041000F501E252FF4F1082D50112968C9112978E
:10042000882341F4C5010E94E07CF5018281882384
:1004300009F4B5C000D000D0EDB7FEB731965FE14A
:10044000C52ED12CCC0EDD1EADB7BEB71296DC92F8
:10045000CE9211978DED93E093838283D5015096D0
:100460008D919C915197958384830E949EA8EDB7AE
:10047000FEB736960FB6F894FEBF0FBEEDBF8601ED
:1004800008C0D6018C9190E00E9414A8F6018193D7
:100490006F01F80101900020E9F73197E01BF10BA3
:1004A000C601801B910B8E179F075CF336E1432E2C
:1004B000512C4A0C5B1CC2010E94CF1A99248E0158
:1004C000035C1F4F4FE1242E312C2C0E3D1E3E01AC
:1004D0000894611C711C47C0D6018C9190E00E9469
:1004E00014A8F60181936F01C701F8010190002063
:1004F000E9F73197E01BF10B0894E11CF11C8E1712
:100500009F0754F327968FAD27978E3761F1C80167
:10051000B10145E050E00E9467A8009721F500D0A6
:1005200000D0EDB7FEB73196ADB7BEB712967C924C
:100530006E92119786EE93E09383828335822482B4
:100540000E949EA8ADB7BEB716960FB6F894BEBF70
:100550000FBEADBFC3010E94AA288DEE93E00E949A
:10056000AA2899249394C201B8010E94C5191816AB
:1005700024F46801EE24FF24B7CF992031F48FEFE3
:100580009FEFF501918B808B0AC0D50150968D911C
:100590009C915197019651969C938E935097C45A73
:1005A000DF4F0FB6F894DEBF0FBECDBFDF91CF9106
:1005B0001F910F91FF90EF90DF90CF90BF90AF9081
:1005C0009F907F906F905F904F903F902F900895F5
:1005D0000F931F93CF93DF938C01EC01C954DF4F2E
:1005E000CE010E94D61ACE010E94211BF801108272
:1005F000DF91CF911F910F9108950F931F93CF9388
:10060000DF93CDB7DEB76F970FB6F894DEBF0FBE9E
:10061000CDBF8C01C396F80192AB81ABE152FF4F85
:1006200082E08083F801E052FF4F60831182C801AD
:10063000C7960E94CF1AF80181A992A9DE011596EA
:10064000FC0134962BE101900D922150E1F7FC0161
:10065000828193819C838B8381E494E09A83898354
:10066000C8016CED73E0AE014F5F5F4F0E941F7BCE
:10067000CE0101960E94E96C6F960FB6F894DEBF2A
:100680000FBECDBFDF91CF911F910F9108950F93B2
:100690001F93CF93DF93CDB7DEB76F970FB6F89464
:1006A000DEBF0FBECDBF8C01C396F80192AB81AB0C
:1006B000E152FF4F81E08083F801E052FF4F118249
:1006C0001082C801C7960E94CF1AF80181A992A989
:1006D000DE011596FC0134962BE101900D9221501C
:1006E000E1F7FC01828193819C838B8381E494E018
:1006F0009A838983C8016CED73E0AE014F5F5F4F51
:100700000E941F7BCE0101960E94E96CF801E05225
:10071000FF4F808191816F960FB6F894DEBF0FBEB8
:10072000CDBFDF91CF911F910F910895CF92DF92AE
:10073000EF92FF920F931F93CF93DF93CDB7DEB766
:100740006F970FB6F894DEBF0FBECDBF8C01F62EAB
:10075000E72E1D8218861C821B8281E494E09A8316
:100760008983F80182AD882321F472E1C72ED12C50
:1007700003C063E3C62ED12CC00ED11EB6016C5F40
:100780007F4FCE0105964F2D5E2D21E00E94531D17
:10079000882371F5EEE1F4E107C09091C00095FF68
:1007A000FCCF8093C600319684918823B1F7E4E5AD
:1007B000F5E107C09091C00095FFFCCF8093C60083
:1007C000319684918823B1F7EF2DFE2D06C09091CC
:1007D000C00095FFFCCF8093C60081918823B9F7B4
:1007E0008091C00085FFFCCF8AE08093C60035C0B1
:1007F00098012F583F4FF9013496D801AA5ABF4F9C
:100800008BE10D9001928150E1F7F801EC5AFF4F16
:1008100080819181F90193838283D801AA5ABF4FC5
:10082000F60134968BE101900D928150E1F7F601CB
:1008300082819381F801EE5AFF4F93838283D8011E
:10084000D796FE0135968BE101900D928150E1F72C
:100850008B819C81F80196AB85ABCE0101960E94FD
:10086000E96C6F960FB6F894DEBF0FBECDBFDF9177
:10087000CF911F910F91FF90EF90DF90CF9008954F
:10088000CF93DF93EC018AAD8250823028F1DE01F4
:10089000D796FE01EA5AFF4F8BE101900D928150ED
:1008A000E1F7FE01EC5AFF4F808191819EAB8DAB49
:1008B000CE018E5A9F4FDC011496FE01EB58FF4F7C
:1008C0002BE101900D922150E1F7CD58DF4F2881A7
:1008D0003981FC0133832283DF91CF910895CF9337
:1008E000DF93EC010E9429160E94A616198281EF5F
:1008F00093E00E94AA28DF91CF9108952F923F9212
:100900004F925F926F927F928F929F92AF92BF921F
:10091000CF92DF92EF92FF920F931F93CF93DF93CB
:10092000CDB7DEB7C055D0400FB6F894DEBF0FBECE
:10093000CDBF2C017A8F698F4A012CA708AFE9AE91
:10094000AAAEBBAECCAEDDAE022F10E0000F111F81
:10095000000F111F9A01200F311F3DAB2CABD901A5
:100960008D919D910D90BC91A02D898B9A8BAB8B15
:10097000BC8BF201E00FF11FBC01CD012081318160
:10098000428153810E9453A06EAF7FAF21968FAFFB
:10099000219722969FAF2297B8ADEB2EFF24EE0C45
:1009A000FF1CEE0CFF1CF401EE0DFF1DFFABEEABC8
:1009B00080809180A280B380F201EE0DFF1DC50101
:1009C000B40120813181428153810E9453A023963A
:1009D0006FAF239724967FAF249725968FAF2597E7
:1009E00026969FAF2697F9AD8F2F90E0880F991F1D
:1009F000880F991FF201E80FF91F20813181428190
:100A000053812B8F3C8F4D8F5E8FE98DFA8DE80FD0
:100A1000F91F60817181828193810E9452A0462FCB
:100A2000572F682F792F4F8F58A369A37AA3A98DC9
:100A3000BA8D1C968D919D910D90BC91A02D88AB87
:100A400099ABAAABBBABD2011C962D913D914D91B8
:100A50005C911F972FA338A749A75AA729893A89DC
:100A60004B895C895058298B3A8B4B8B5C8BD50119
:100A7000C401B0588D8B9E8BAF8BB88FE98DFA8DEA
:100A8000E00FF11F6081718182819381FEADEFAD36
:100A900021965FAD219722964FAD22970F2F1E2FE3
:100AA000252F342FA90198010E9452A06B01482ED6
:100AB000792EE98DFA8DEE0DFF1D608171818281A5
:100AC00093812396FFAD23972496EFAD2497259627
:100AD0005FAD259726964FAD26970F2F1E2F252FFA
:100AE000342FA90198010E9452A0F62EE72E682EFD
:100AF000592E69897A898B899C89F7010F2F1E2FBE
:100B0000262D352DA90198010E9401A44B015C01FD
:100B10006D897E898F89988D0C2D1D2D242D372D63
:100B2000A90198010E9401A49B01AC01C501B40177
:100B30000E9452A06BA37CA38DA39EA369897A898E
:100B40008B899C89242D372DA90198010E9401A42D
:100B50004B015C016D897E898F89988DF7010F2F7C
:100B60001E2F262D352DA90198010E9401A49B015D
:100B7000AC01C501B4010E9453A09B01AC016BA163
:100B80007CA18DA19EA10E94C6A0162F072FF82E32
:100B9000E92EA8019701852F942FA32FB22FBC0116
:100BA000CD0120E030E040E050E00E942CA187FF22
:100BB00012C0A8019701852F942FA32FB22FBC013B
:100BC000CD012BED3FE049EC50E40E9453A0162FDD
:100BD000072FF82EE92EAB968FADAB97882391F0B7
:100BE000A8019701852F902FA32FBE2DBC01CD0109
:100BF0002BED3FE049EC50E40E9452A0162F072F46
:100C0000F82EE92EA8019701852F902FA32FBE2D36
:100C1000BC01CD01AA962CAD3DAD4EAD5FADAA97FE
:100C20000E9401A42F8D38A149A15AA15F770E948B
:100C30003CA34B015C012FE632E143E85AE30E94FA
:100C40002CA187FD6AC2C501B4010E9409A20E94BD
:100C5000A0A1DC01CB019FA78EA7009721F4A1E002
:100C6000B0E0BFA7AEA7EEA5FFA5BF0180E090E072
:100C70000E94CCA14B015C01A8019701852F902F08
:100C8000A32FBE2DBC01CD01A50194010E9433A16B
:100C9000362E272E8BA39BA76F8D78A189A19AA1B1
:100CA000A50194010E9433A12A966FAF2A972B9633
:100CB0007FAF2B972C968FAF2C972D969FAF2D97AC
:100CC00068A979A98AA99BA92FA138A549A55AA5E0
:100CD0000E9452A0A50194010E9433A12E966FAFED
:100CE0002E972F967FAF2F9760968FAF6097619664
:100CF0009FAF6197A1013BA12BA5852F942FA32F17
:100D0000B22FBC01CD0120E030E040E05FE30E9463
:100D100001A4F1015BA14BA50F2F1E2F252F342F0E
:100D2000A90198010E9401A49B01AC0160E070E060
:100D300080E89FE30E9452A068AB27967FAF279779
:100D400028968FAF289729969FAF299729ADE22F34
:100D5000F0E0EE0FFF1FEE0FFF1FCE010196E80F30
:100D6000F91F2B8D3C8D4D8D5E8D20833183428309
:100D700053832FA138A549A55AA52D873E874F87B4
:100D8000588B882441E050E058A74FA3BCA5AB2F57
:100D9000B0E0AA0FBB1FAA0FBB1F9C012A0F3B1F6D
:100DA0003C8F2B8F58AD452F50E0440F551F440FFB
:100DB000551F81E090E08C0F9D1F840F951F98A315
:100DC0008F8FFDA7ECA788C198E198150CF46FC030
:100DD00069897A898B899C89432D522DEBA1FBA5CA
:100DE0008A019F01A90198010E9401A46B017C0165
:100DF0006D897E898F89988D48A927965FAD279741
:100E00002896EFAD28972996FFAD29978A019F0173
:100E1000A90198010E9401A49B01AC01C701B60180
:100E20000E9453A0762E672E582E492E69897A8902
:100E30008B899C892896EFAD28972996FFAD299735
:100E40009F01A90198010E9401A4F62EE72ED82E39
:100E5000C92E6D897E898F89988D432D522DEBA1E6
:100E6000FBA58A019F01A90198010E9401A49B0191
:100E7000AC01F701B6018F2F9E2FA72FB62FBC0113
:100E8000CD010E9452A0462F572F682F792F498BF2
:100E90005A8B6B8B7C8B8394A3019201852F942FAB
:100EA000A32FB22F8D8B9E8BAF8BB88F81C0AFA13C
:100EB000B8A5BD0180E090E00E94CCA1432D522D49
:100EC000EBA1FBA58A019F01A90198010E9401A441
:100ED000162F072FF82EE92EA8019701852F942FA2
:100EE000A32FB22FBC01CD010E9430A16D8B7E8B50
:100EF0008F8B988FA8019701852F942FA32FB22F46
:100F0000BC01CD010E9464A42B013C01ECA9FDA908
:100F100080819181A281B3816C017D01F7FAF09407
:100F2000F7F8F094AEA9BFA98D909D90AD90BC90BC
:100F3000C701B6012D893E894F89588D0E9401A4B1
:100F4000698B7A8B8B8B9C8BC501B401A3019201B9
:100F50000E9401A49B01AC0169897A898B899C89D3
:100F60000E9453A0AB01682F792F498B5A8B6B8B52
:100F70007C8BC701B601A30192010E9401A46B0101
:100F80007C01C501B4012D893E894F89588D0E948D
:100F900001A49B01AC01C701B6010E9452A0462FDB
:100FA000572F682F792F4D8B5E8B6F8B788F88240E
:100FB0005EAD4FAD21963FAD219722962FAD229782
:100FC000852F942FA32FB22FBC01CD0129893A89F7
:100FD0004B895C890E9453A0DC01CB01EB8DFC8D19
:100FE00080839183A283B38323965FAD2397249656
:100FF0004FAD249725963FAD259726962FAD269782
:10100000852F942FA32FB22FBC01CD012D893E89AE
:101010004F89588D0E9453A0DC01CB01EF8DF8A1C0
:1010200080839183A283B383ACA5BDA56D917D918F
:101030008D919C912A964FAD2A972B965FAD2B9759
:101040002C96EFAD2C972D96FFAD2D978A019F0121
:10105000A90198010E9453A0DC01CB01ECA5FDA5DC
:1010600080839183A283B3836D857E858F859889E4
:101070002E964FAD2E972F965FAD2F976096EFADC2
:1010800060976196FFAD61978A019F01A901980160
:101090000E9453A0DC01CB018D879E87AF87B88B60
:1010A000CE010196BE016B5F7F4FAE01475F5F4F80
:1010B0009E01235F3F4FEAACFBAC0CAD1DADFBE6E0
:1010C000CF2ED12CCC0EDD1E0E946D8D2FA138A508
:1010D0002F5F3F4F38A72FA34FA158A58EA59FA5DF
:1010E0004817590708F470CE698D7A8D6C5F7F4F71
:1010F000498D5A8D485F5F4F298D3A8D245F3F4F50
:10110000898D9A8DEAACFBAC0CAD1DADEBE6CE2E15
:10111000D12CCC0EDD1E0E946D8DC05BDF4F0FB653
:10112000F894DEBF0FBECDBFDF91CF911F910F911D
:10113000FF90EF90DF90CF90BF90AF909F908F90F7
:101140007F906F905F904F903F902F9008952F92D7
:101150003F924F925F926F927F928F929F92AF9247
:10116000BF92CF92DF92EF92FF920F931F93CF9394
:10117000DF93CDB7DEB768970FB6F894DEBF0FBE2A
:10118000CDBF1C016A017B0128013901DC01D89621
:101190006D917D918D919C91DB970E94CCA14B012B
:1011A0005C01A70196010E9401A40E9419A10E945E
:1011B000A0A169837A838B839C83C501B401A301B9
:1011C00092010E9401A40E9419A10E94A0A16D8316
:1011D0007E838F83988729813A814B815C81283770
:1011E00031054105510540F488E790E0A0E0B0E00A
:1011F00089839A83AB83BC832D813E814F8158853F
:10120000283731054105510540F488E790E0A0E01A
:10121000B0E08D839E83AF83B887F101EC5BFF4F15
:101220004080518062807380D101DC966D917D9108
:101230008D919C91DF970E94CCA16D877E878F87CF
:10124000988BC301B2010E94CEA169877A878B87F0
:101250009C8720E030E040E050E00E942CA18823F1
:1012600039F1C501B401A50194010E9401A46B01EB
:101270007C016D857E858F8598899B01AC010E94DC
:1012800001A49B01AC01C701B6010E9452A06B01F1
:101290007C0169857A858B859C859B01AC010E94C8
:1012A00053A09B01AC01C701B6010E9433A104C049
:1012B00060E070E080E090E0382F292F862F972F94
:1012C000A32FB22FBC01CD010E9419A10E949BA1A6
:1012D0006B017C01F101E05CFF4F608171818281D3
:1012E00093810E94CCA1698B7A8B8B8B9C8B662718
:1012F0007727CB0164197509860997090E94CEA149
:101300002B013C0120E030E040E050E00E942CA1A5
:10131000882349F169897A898B899C899B01AC0171
:101320000E9401A46D8B7E8B8F8B988FC501B401B9
:10133000A50194010E9401A49B01AC016D897E89E5
:101340008F89988D0E9452A04B015C01C301B201AC
:10135000A30192010E9453A09B01AC01C501B401FD
:101360000E9433A104C060E070E080E090E0382F7C
:10137000292F862F972FA32FB22FBC01CD010E94BA
:1013800009A2F101408851886288738853014201A3
:101390008C189D08AE08BF080E949BA1DC01CB0100
:1013A000A5019401281B390B4A0B5B0BDA01C9011B
:1013B00057FF76C069857A858B859C8520E030E073
:1013C00040E050E00E942CA1882309F447C06985C1
:1013D0007A858B859C859B01AC010E9453A06B0193
:1013E0007C01C301B2010E94CCA19B01AC01C701E9
:1013F000B6010E9401A46B017C016D857E858F85FD
:1014000098899B01AC010E9401A49B01AC01C7011A
:10141000B6010E9452A06B017C0169897A898B898F
:101420009C899B01AC010E9401A49B01AC01C701F6
:10143000B6010E9453A06B017C0169857A858B857A
:101440009C8520E030E040E850E40E9401A49B012C
:10145000AC01C701B6010E9433A104C060E070E096
:1014600080E090E0382F292F862F972FA32FB22FBF
:10147000BC01CD010E9419A10E949BA16B017C01BE
:10148000F7FE03C0CC24DD247601C414D504E604A1
:10149000F70410F07301620180E090E0A0E0B0E09A
:1014A0002FB7F894F101E45BFF4F3081332309F546
:1014B000F101C48AD58AE68AF78A8C0D9D1DAE1D7E
:1014C000BF1D808F918FA28FB38F89819A81AB814D
:1014D000BC8184AF95AFA6AFB7AFA101405C5F4FB1
:1014E0008D819E81AF81B885FA0180839183A2832B
:1014F000B3832FBF68960FB6F894DEBF0FBECDBF83
:10150000DF91CF911F910F91FF90EF90DF90CF90DF
:10151000BF90AF909F908F907F906F905F904F9013
:101520003F902F9008954F925F926F927F928F928B
:101530009F92AF92BF92CF92DF92EF92FF920F9362
:101540001F93CF93DF93EB016A01209709F47DC0CD
:101550004115510509F479C07AA46BA45CA44DA48B
:101560006EA17FA188A599A5F301A2010F2F1E2FBF
:10157000252F342FA90198010E942CA1882309F45A
:1015800064C08FA9882309F054C0F601C6A0D7A073
:10159000E0A4F1A4A3019201852F942FA32FB22FD1
:1015A000BC01CD01A70196010E942FA318160CF0D3
:1015B00040C0C701B601A70196010E9401A46B01BA
:1015C0007C018AA99BA9ACA9BDA99C01AD01505879
:1015D000CA01B9010E9453A02EA53FA548A959A947
:1015E0000E9401A49B01AC01C701B6010E9452A058
:1015F0000E946EA4162FC72E082FF92EA301920168
:10160000852F942FA32FB22FBC01CD01812E9C2CAE
:10161000A02EBF2CA50194010E942CA187FF04C01D
:10162000172DC62C052DF42C512F4C2D302F2F2D7E
:1016300002C0A3019201852F942FA32FB22F8EA356
:101640009FA3A8A7B9A781E08EABDF91CF911F918F
:101650000F91FF90EF90DF90CF90BF90AF909F9051
:101660008F907F906F905F904F900895CF92DF9210
:10167000EF92FF920F931F93CF938091E20A809194
:10168000E20A2091E10A90E0821B91098F7090702C
:10169000843091052CF1C091E20AC350CF7040E034
:1016A00050E0EE24FF248DE4C82ED12C15C0CC23AD
:1016B00009F4C0E1C1508C2F90E08C9D80018D9D7C
:1016C000100D9C9D100D11240D51154FC801B7012F
:1016D0000E94938AA70178018091E10AC81739F71F
:1016E000CF911F910F91FF90EF90DF90CF900895D1
:1016F0006F927F928F929F92AF92BF92CF92DF9222
:10170000EF92FF920F931F93CF93DF93EC013B0176
:10171000009709F473C08FA9882309F06FC0CEA089
:10172000DFA0E8A4F9A4FB01B6A0A7A090A481A41F
:10173000C701B601F501A4010F2F1E2F252F342F4D
:10174000A90198010E942CA187FF58C0C701B601CA
:10175000A70196010E9401A46B017C018AA99BA9A3
:10176000ACA9BDA99C01AD015058CA01B9010E94A4
:1017700053A02EA53FA548A959A90E9401A49B01E9
:10178000AC01C701B6010E9452A00E946EA4C62EF1
:10179000C72FD82FF92EA5019401852F942FA32FA1
:1017A000B22FBC01CD010C2D1C2F2D2F3F2DA901D7
:1017B00098010E942CA187FF04C0CB2CCA2DD92DE3
:1017C000F82CA5019401852F9A2DA32FB82DBC01CB
:1017D000CD010C2D1C2F2D2F3F2DA90198010E940A
:1017E0002CA1882359F0802F9C2FAD2FBF2DF30102
:1017F00086A397A3A0A7B1A781E086ABDF91CF9185
:101800001F910F91FF90EF90DF90CF90BF90AF901E
:101810009F908F907F906F900895CF92DF92EF927C
:10182000FF920F931F93CF93C091E10AEE24FF2400
:1018300020E030E09DE4C92ED12C16C08C2F90E022
:101840008C9D80018D9D100D9C9D100D11240D51BE
:10185000154FC901B701A8010E94788BCF5FC03135
:1018600009F4C0E0970178018091E20AC81731F7C6
:10187000C901B70140E050E00E94788BCF911F91E1
:101880000F91FF90EF90DF90CF9008952F923F92AD
:101890004F925F926F927F928F929F92AF92BF9280
:1018A000CF92DF92EF92FF920F931F93CF93DF932C
:1018B000F090E10AC0E0D0E02DE4222E312C39C0B6
:1018C000229D6001239DD00C329DD00C112483EE0B
:1018D0009AE0C80ED91E209731F18EA9882321F4F1
:1018E000F60186A98823F9F08AA09BA0ACA0BDA030
:1018F0006EA17FA188A599A5A50194010E9433A19D
:101900002B013C01F60166A177A180A591A5A50157
:1019100094010E9433A18B019C01CE01B301A2016D
:101920000E94A7881EAAF394F0E1FF1609F4FF2491
:10193000E6012F2D332727FD30958091E20A90E0B4
:101940002817390709F0BCCF2097F1F0CAA0DBA017
:10195000ECA0FDA06EA17FA188A599A5A701960185
:101960000E9433A14B015C016DEC7CEC8CE49DE3A7
:10197000A70196010E9433A18B019C01CE01B50104
:10198000A4010E94A7881EAADF91CF911F910F91F9
:10199000FF90EF90DF90CF90BF90AF909F908F908F
:1019A0007F906F905F904F903F902F9008950E948E
:1019B000368B0E940D8C0E94468C08951092E20A8C
:1019C0001092E10A80E1E3EBFFE0DF011D928A95CE
:1019D000E9F780E090E0A0E0B0E0809323109093DE
:1019E0002410A0932510B093261080932710909375
:1019F0002810A0932910B0932A1080932B10909355
:101A00002C10A0932D10B0932E1080932F10909334
:101A10003010A0933110B093321080933310909314
:101A20003410A0933510B09336100895CF93909151
:101A3000E10A8091E20A981771F1A091E10A2A2F38
:101A400030E08DE490E0289FF001299FF00D389F51
:101A5000F00D1124E55DF44FC081B0E017C02A2FCE
:101A600030E0289FF001299FF00D389FF00D1124E0
:101A7000E55DF44F408151816281738141155105CB
:101A80006105710509F0BF5FAF5FAF702091E20A99
:101A9000A21729F70AC06091FD06662321F087E0AE
:101AA00070E00E942C9BC0E0B0E08091FD0688238E
:101AB00039F4BB2329F487E060E070E00E942C9B9E
:101AC0008091FD06882339F0CC2329F087E06C2F24
:101AD00070E00E942C9BCF9108952F923F924F92DD
:101AE0005F926F927F928F929F92AF92BF92CF92AE
:101AF000DF92EF92FF920F931F93CF93DF93CDB7B7
:101B0000DEB7C156D0400FB6F894DEBF0FBECDBFD2
:101B10005C014B015CA34BA33AAB29AB1701602ED0
:101B2000412EDEAACDAA8091E20A8F5F803109F4AE
:101B300080E0282F332727FD30956F963FAF2EAFDB
:101B40006F9707C00E94EF6D81E00E94882C0E9471
:101B500063588091E10A90E06F964EAD5FAD6F974C
:101B60008417950779F3D5016D917D918D919C91A5
:101B70002091FF0F30910010409101105091021000
:101B80000E9401A40E94D1A32A966FAF2A972B9698
:101B90007FAF2B972C968FAF2C972D969FAF2D97BD
:101BA000F4016081718182819381209103103091D1
:101BB000041040910510509106100E9401A40E944B
:101BC000D1A32E966FAF2E972F967FAF2F9760964B
:101BD0008FAF609761969FAF6197ABA1BCA16D91EC
:101BE0007D918D919C91209107103091081040912A
:101BF000091050910A100E9401A40E94D1A362967C
:101C00006FAF629763967FAF639764968FAF649769
